:100000000C94F6130C9420140C9420140C942014CB
:100010000C9420140C9420140C9420140C94201490
:100020000C9420140C9420140C9420140C94201480
:100030000C9420140C94EC730C9420140C94201445
:100040000C9420140C94A6710C9421C20C942014CE
:100050000C94103B0C94063B0C9420140C9420142C
:100060000C9420140C9420140C9420140C94201440
:100070000C9420140C9420140C9420140C94201430
:100080000C9420140C9420140C9420144E414E49CE
:100090004E495459494E46CDCCCC3D0AD7233C1746
:1000A000B7D13877CC2B329595E6241FB14F0A0093
:1000B0000020410000C84200401C4620BCBE4CCA83
:1000C0001B0E5AAEC59D7400407A10F35A00A07200
:1000D0004E18090010A5D4E80000E8764817000083
:1000E000E40B54020000CA9A3B000000E1F5050051
:1000F0000080969800000040420F000000A086019A
:10010000000000102700000000E803000000006469
:1001100000000000000A00000000000100000000D4
:10012000002C76D888DC674F0823DFC1DFAE59E1A9
:10013000B1B796E5E3E453C63AE651997696E8E618
:10014000C28426EB898C9B62ED407C6FFCEFBC9CEB
:100150009F40F2BAA56FA5F490055A2AF75C936BFD
:100160006CF9676DC11BFCE0E40D47FEF520E6B5B8
:1001700000D0ED902E0300943577050080841E0892
:100180000000204E0A000000C80C333333330F98B0
:100190006E12831141EF8D2114893BE65516CFFE77
:1001A000E6DB18D1844B381BF77C1D901DA4BBE403
:1001B00024203284725E228100C9F124ECA1E53D45
:1001C00027434F4D4D554E49434154494F4E0044EE
:1001D000525952554E004552524F525300494E46C5
:1001E0004F004543484F00486F74656E6420496472
:1001F0006C652054696D656F757400486F74656E29
:10020000642049646C652054696D656F75740A00DB
:100210002121204B494C4C20636175736564206239
:100220007920746F6F206D75636820696E616374E7
:100230006976652074696D65202D2063757272651D
:100240006E7420636F6D6D616E643A200053544F7D
:10025000505045442E20005072696E7465722073B0
:10026000746F707065642064756520746F206572AA
:10027000726F72732E2046697820746865206572EB
:10028000726F7220616E6420757365204D39393943
:1002900020746F20726573746172742E2028546507
:1002A0006D70657261747572652069732072657313
:1002B00065742E20536574206974206166746572BC
:1002C0002072657374617274696E67290A004E6FDB
:1002D00020436865636B73756D2077697468206C63
:1002E000696E65206E756D6265722C204C61737449
:1002F000204C696E653A20004E6F20436865636B41
:1003000073756D2077697468206C696E65206E75F1
:100310006D6265722C204C617374204C696E653A75
:100320002000636865636B73756D206D69736D6123
:100330007463682C204C617374204C696E653A209C
:10034000004C696E65204E756D6265722069732080
:100350006E6F74204C617374204C696E65204E750D
:100360006D6265722B312C204C617374204C696E68
:10037000653A20004D3131300053657269616C205F
:10038000737461747573206D69736D617463680A49
:100390000053442072656164206572726F720A00B6
:1003A0004D6564696120496E7365727465640050BF
:1003B0006C65617365205265736574005052494ED7
:1003C0005445522048414C5445440025533A202579
:1003D0005300706F7765726F6666004B494C4C45F1
:1003E000442E20005072696E7465722068616C74CE
:1003F00065642E206B696C6C28292063616C6C65C8
:1004000064210A006563686F3A004572726F723A40
:10041000000A4D6561737572656420706F696E7452
:10042000733A0A00357835206D6573682E205A209E
:100430006F66667365743A2000206E6F7420656E77
:1004400074657265642E0A0050726F62696E67206F
:10045000506F696E740025532025692F256900208F
:100460006F6620004D424C2047323920706F696E14
:10047000742000290A004A206F7574206F6620726C
:10048000616E67652028302D00290A0049206F75AC
:1004900074206F662072616E67652028302D0047DA
:1004A00032384C30004D6573682070726F62696E2F
:1004B0006720646F6E65004D6573682070726F62AF
:1004C000696E6720646F6E652E0A005374617274E2
:1004D000206D6573682070726F62696E672077693E
:1004E00074682022473239205331222066697273A2
:1004F000742E0A004732395332004732384C300AE2
:10050000473239533200686173206E6F2064617422
:10051000612E0A004D65736820426564204C657643
:10052000656C696E67200053206F7574206F6620BC
:1005300072616E67652028302D35292E0A0020490A
:100540006E76616C6964206578747275646572207A
:1005500000536C6565702E2E2E004D6573682070FB
:100560006F696E74206F7574206F662072616E679C
:10057000650A00436C69636B20746F205265737564
:100580006D652E2E2E004E6F204D6F76652E004528
:100590006E642066696C65206C6973740A0042653C
:1005A00067696E2066696C65206C6973740A004E19
:1005B0006F206D656469610A00706175736500285C
:1005C0006E6F2066696C65290043757272656E7482
:1005D0002066696C653A20005344207072696E741D
:1005E000696E67206279746520004E6F74205344F1
:1005F000207072696E74696E670A002E0A00446585
:100600006C6574696F6E206661696C65642C204648
:10061000696C653A200046696C652064656C657498
:1006200065643A002569730025696D2025697300AA
:100630002569682025696D20256973002569642076
:100640002569682025696D20256973002569792051
:10065000256964202569682025696D202569730056
:100660005072696E742074696D653A20006F6B007A
:100670006F666600E201DD01D601CF01C10144458C
:100680004255473A0020573A0042656420436F6F55
:100690006C696E672E2E2E00426564204865617479
:1006A000696E672E2E2E004D696E69205375506558
:1006B00052204F46462E004649524D574152455F03
:1006C0004E414D453A4D61726C696E20322E302E8E
:1006D000375F4457372E3320544D3344204D454D1A
:1006E000444E4E2028417072203234203230323154
:1006F0002032323A30313A33332920534F55524366
:10070000455F434F44455F55524C3A68747470736B
:100710003A2F2F6769746875622E636F6D2F496E6B
:1007200073616E6974794175746F6D6174696F6E10
:100730002F4D61726C696E2F747265652F437265FF
:10074000616C6974794477696E5F322E3020505243
:100750004F544F434F4C5F56455253494F4E3A31D9
:100760002E30204D414348494E455F545950453A3B
:100770004D696E6920537550655220455854525545
:100780004445525F434F554E543A312055554944E4
:100790003A63656465326132662D343161322D34DD
:1007A0003734382D396231322D6335356336326650
:1007B00033363766660A002F2F004D31343520530B
:1007C0003C696E6465783E206F7574206F66207298
:1007D000616E67652028302D31290A0020520041C2
:1007E0006363656C65726174696F6E3A205000577F
:1007F00041524E494E4721204C6F77205A204A657E
:10080000726B206D6179206C65616420746F207556
:100810006E77616E746564207061757365732E0AFE
:10082000004D32303620580020204D61783A2000AB
:10083000200020204D696E3A2000536F66742065B9
:100840006E6473746F70733A200046523A0020460B
:100850006C6F773A20004D424C2041646A75737486
:10086000205A0020643A0020693A0020703A00497A
:100870006E76616C69642065787472756465720A5D
:100880000064697300656E0043290A0061626C654B
:100890006420286D696E2074656D702000436F6C54
:1008A00064206578747275646573206172652000D8
:1008B0004F4646004F4E00426564204C6576656C9D
:1008C000696E6720004661696C656420746F2065FD
:1008D0006E61626C6520426564204C6576656C696A
:1008E0006E670A004D65736820426564204C65762A
:1008F000656C20646174613A0A00496E76616C69C6
:1009000064206D6573682E0A004D65736820706FF2
:10091000696E74206F7574206F662072616E6765F2
:100920000A004D34323120696E636F7272656374F0
:1009300020706172616D65746572207573616765A1
:100940000A004F666673657473204170706C696548
:1009500064004572723A20546F6F20666172210004
:10096000546F6F206661722066726F6D20726566CB
:100970006572656E636520706F696E740A00454527
:1009800050524F4D204F4B0A004D383400446F6E8B
:1009900065207072696E74696E672066696C650A9D
:1009A000004D3737004D333100496E76616C696414
:1009B0002065787472756465720A0020573A0043A6
:1009C0006F6F6C696E672E2E2E0048656174696EBC
:1009D000672E2E2E00452025530023646566696E20
:1009E000652044454641554C545F004B6420004B04
:1009F0006920004B702000504944204175746F7489
:100A0000756E652066696E6973686564212050752E
:100A10007420746865206C617374204B702C204BBB
:100A20006920616E64204B6420636F6E7374616E25
:100A300074732066726F6D2062656C6F7720696ECB
:100A4000746F20436F6E66696775726174696F6E4B
:100A50002E680A00504944204175746F74756E65A4
:100A6000206661696C6564212074696D656F7574B9
:100A70000A00504944204175746F74756E65206694
:100A800061696C6564212054656D7065726174756F
:100A9000726520746F6F20686967680A00204B6474
:100AA0003A2000204B693A2000204B703A20002069
:100AB000436C617373696320504944200A002054D9
:100AC000753A2000204B753A2000206D61783A205D
:100AD00000206D696E3A200020643A20002062698F
:100AE00061733A2000504944204175746F74756EEB
:100AF000652073746172740A005049442041757412
:100B00006F74756E65206661696C6564212054653B
:100B10006D706572617475726520746F6F2068699D
:100B200067680A00504944204175746F74756E659A
:100B3000206661696C65642120426164206865619A
:100B40007465722069640A00504944204175746FCD
:100B500074756E65004572723A2075746638206649
:100B60006F6E74206E6F7420696E697469616C6950
:100B70007A65642E004572723A2075746638206674
:100B80006F6E74206E6F7420696E697469616C6930
:100B90007A65642E004572723A2075746638206654
:100BA0006F6E74206E6F7420696E697469616C6910
:100BB0007A65642E0042656400456E636C6F7375E0
:100BC0007265002568753A25303268750025303227
:100BD00068753A25303268750020202020202020BA
:100BE0000020202020003FFFF038007030FC302033
:100BF000FC102078102030102C00D02E31D02F7B0C
:100C0000D02F7BD02E31D02C00D020301020781067
:100C100020FC1030FC303800703FFFF03FFFF03810
:100C200000703186302387102787902F87D02F03BD
:100C3000D02030102078102078102030102F03D0D2
:100C40002F87D02787902387103186303800703F58
:100C5000FFF0041040020820020820041040082081
:100C60008010410010410008208004104000000066
:100C70001FFFF81FFFF863616E63656C00507269B7
:100C80006E742041626F72746564004D323500509D
:100C9000617573696E672E2E2E00726573756D65B2
:100CA000004D32340046696C2E204469612E004F9D
:100CB0006666004F6E004520696E206D6D5E3300E4
:100CC0005654726176204D696E00566D696E0056FD
:100CD0006D6178204500566D6178205A00566D612F
:100CE00078205900566D6178205800416D61782058
:100CF0004500416D6178205A00416D6178205900AE
:100D0000416D6178205800412D54726176656C0008
:100D1000412D5265747261637400416363656C00B8
:100D200056652D4A65726B00565A2D4A65726B00E6
:100D300056592D4A65726B0056582D4A65726B00E4
:100D4000452073746570732F6D6D005A2053746560
:100D500070732F6D6D00592053746570732F6D6D16
:100D600000582053746570732F6D6D004164766177
:100D70006E6365642053657474696E6773003F0029
:100D800043616E63656C00496E6974004D3432389E
:100D900000496E697469616C697A652045455052F5
:100DA0004F4D0046696C616D656E740053746570DB
:100DB000732F6D6D004A65726B00416363656C65EE
:100DC000726174696F6E0056656C6F636974790047
:100DD00053657420486F6D65204F66667365747344
:100DE00000436F6E66696775726174696F6E004C5F
:100DF0006576656C696E6720446F6E6521004D6F86
:100E00007665205A00473239533200000C0F00FE3D
:100E100007022503BB017FFE08FE08FE0508080641
:100E2000000040F0C888889878100508080600007F
:100E3000C0F88888888888F80505050600012030F4
:100E4000F830200508080600002070F82020202037
:100E5000E00509090600FF2070A8A8B8888870205E
:100E6000070505070001D86C366CD805090906008E
:100E7000FFF8A88888888888A8F8050A0A0600FE6E
:100E8000205050505088A8A8887003030306000320
:100E900040A040FFFFFFFFFFFFFFFFFFFFFFFFFF3F
:100EA000FFFFFFFFFFFFFFFFFF0000000605FF0140
:100EB000070706020080808080800080030303060D
:100EC0000105A0A0A005060606000050F85050F845
:100ED000500509090600FF2070A8A07028A87020FE
:100EE000050707060000C8C81020409898050707A6
:100EF00006000040A0A040A8906801030306020578
:100F00008080800309090601FF20404080808040E6
:100F100040200309090601FF804040202020404076
:100F20008005070706000020A8702070A82005058E
:100F3000050600012020F820200203030601FFC05F
:100F40004080050101060003F8020202060100C00C
:100F5000C005070706000008101020404080050764
:100F600007060000708898A8C88870030707060164
:100F70000040C040404040E0050707060000708880
:100F800008102040F8050707060000F80810300890
:100F9000887005070706000010305090F810100503
:100FA0000707060000F880F00808887005070706A4
:100FB0000000304080F0888870050707060000F8C0
:100FC0000810102020200507070600007088887090
:100FD0008888700507070600007088887808106008
:100FE000020505060100C0C000C0C00206060601D9
:100FF000FFC0C000C04080030505060101204080FD
:101000004020050303060002F800F8030505060169
:1010100001804020408005070706000070881020EE
:101020002000200507070600007088B8A8B8807067
:10103000050707060000708888F888888805070774
:10104000060000F04848704848F005070706000011
:1010500070888080808870050707060000F0484887
:10106000484848F0050707060000F88080F08080B7
:10107000F8050707060000F88080F08080800507EB
:1010800007060000708880809888700507070600B2
:1010900000888888F8888888030707060100E040F0
:1010A00040404040E00507070600003810101010CF
:1010B00090600507070600008890A0C0A0908805F2
:1010C0000707060000808080808080F805070706FB
:1010D000000088D8A8888888880507070600008847
:1010E00088C8A8988888050707060000708888883F
:1010F000888870050707060000F08888F0808080E7
:1011000005070706000070888888A890680507070B
:10111000060000F08888F0A0908805070706000008
:1011200070888070088870050707060000F8202086
:1011300020202020050707060000888888888888E6
:10114000700507070600008888888850502005072A
:101150000706000088888888A8A8500507070600A9
:101160000088885020508888050707060000888876
:101170005020202020050707060000F80810204016
:1011800080F80309090601FFE0808080808080806C
:10119000E005070706000080404020101008030902
:1011A000090601FFE020202020202020E005030385
:1011B0000600052050880501010600FEF803030320
:1011C00006010580402005050506000070087888A6
:1011D000780507070600008080F0888888F00505FC
:1011E000050600007080808870050707060000086B
:1011F0000878888888780505050600007088F080E2
:1012000070050707060000304840E04040400507F1
:10121000070600FE708888887808700507070600B2
:10122000008080F088888888030707060100400056
:10123000C0404040E00409090601FE1000301010D3
:101240001010906005070706000080808890E090ED
:1012500088030707060100C04040404040E0050504
:1012600005060000D0A8A8A8A8050505060000B03E
:10127000C88888880505050600007088888870057C
:1012800007070600FEF0888888F0808005070706BB
:1012900000FE78888888780808050505060000B0F3
:1012A000C880808005050506000078807008F0057C
:1012B00007070600002020F8202020180505050655
:1012C00000008888889868050505060000888888D9
:1012D00050200505050600008888A8A850050505CA
:1012E00006000088502050880507070600FE888801
:1012F0008850204080050505060000F8102040F8C1
:101300000309090601FF2040404080404040200181
:1013100009090602FF808080808080808080030928
:10132000090601FF80404040204040408005030303
:1013300006000248A890FF41425300504C41004E25
:1013400065787420506F696E74002569202F202500
:101350007500473239533100473239533200436CFC
:1013600069636B20746F20426567696E00486F6D1A
:10137000696E672058595A0053746F72652053651F
:101380007474696E6773004C6F6164205365747484
:10139000696E677300426564205A004F6666004FAD
:1013A0006E00426564204C6576656C696E67004C22
:1013B0006576656C20426564004D6F74696F6E00E0
:1013C000426564004E6F7A7A6C650046616E205308
:1013D0007065656400436F6E6669677572617469F4
:1013E0006F6E00526573746F726520446566617537
:1013F0006C7473004C6F61642053657474696E671C
:10140000730053746F72652053657474696E6773EB
:101410000050726568656174202420436F6E660019
:10142000416476616E6365642053657474696E67A8
:1014300073004D61696E003F004261636B0053743D
:101440006F70004D3231005072696E742066726F99
:101450006D204D656469610052656C65617365203E
:101460004D65646961004D323200436F6E66696795
:1014700075726174696F6E0054656D706572617428
:10148000757265004D6F74696F6E00526573756D8E
:1014900065205072696E7400417474616368204DF8
:1014A000656469610054756E650053746F702050F7
:1014B00072696E74005061757365205072696E7444
:1014C00000496E666F2053637265656E0043616EFE
:1014D0006E6F7420656E74657220737562646972D4
:1014E0003A2000022E2E0001526566726573680074
:1014F0004D61696E002100486F74656E6420746FE1
:101500006F20636F6C64004261636B0050726F63A5
:10151000656564004D6F74696F6E00446973616244
:101520006C65205374657070657273004D383400BB
:10153000426564204C6576656C696E670041757420
:101540006F20486F6D6500473238004D61696E004D
:1015500050726568656174202420456E6400507285
:1015600065686561742024204265640054656D706F
:1015700065726174757265003B133713436F6F6C4E
:10158000646F776E00507265686561742024004650
:10159000616E20537065656400426564004E6F7A29
:1015A0007A6C65004D61696E0042616279737465A1
:1015B00070205A00466C6F770046616E205370654C
:1015C000656400426564004E6F7A7A6C650042651E
:1015D00064205A005370656564004D61696E00486F
:1015E0006F6D696E67204661696C6564006F706538
:1015F0006E00545249474745524544003A20007A0C
:101600005F6D696E00795F6D696E00785F6D696E00
:10161000005265706F7274696E6720656E647374D2
:101620006F70207374617475730A0020746F6F207B
:101630006C6F6E6720657874727573696F6E207059
:10164000726576656E7465640A0020636F6C642051
:10165000657874727573696F6E2070726576656EE9
:101660007465640A00000000000000000000000033
:10167000005761726E696E673A20486F6D696E67D8
:101680002042756D702044697669736F72203C202A
:10169000310A000202040000964300005C4300008F
:1016A000964300000041000000410000004000009F
:1016B000964300005C4300009643000000000000D9
:1016C00000000000000053657474696E6773205356
:1016D000746F72656400454550524F4D20496E69E4
:1016E0007469616C697A65640A003B2000204400DB
:1016F00020490020204D33303120500050494420F3
:1017000073657474696E67733A0020460020420066
:1017100020480020204D3134352053004D61746540
:101720007269616C206865617475702070617261A6
:101730006D65746572733A00202047323920533446
:10174000205A00204A0020204732392053332049B4
:101750000020204D3432302053004D657368204204
:101760006564204C6576656C696E673A0020204D93
:10177000323036205800486F6D65206F666673659D
:10178000743A0020580020530020204D323035207C
:101790004200416476616E6365643A20423C6D6943
:1017A0006E5F7365676D656E745F74696D655F7597
:1017B000733E20533C6D696E5F666565647261744B
:1017C000653E20543C6D696E5F74726176656C5F36
:1017D00066656564726174653E20583C6D61785F32
:1017E000785F6A65726B3E20593C6D61785F795F06
:1017F0006A65726B3E205A3C6D61785F7A5F6A65FC
:10180000726B3E20453C6D61785F655F6A65726B07
:101810003E0020540020520020204D323034205011
:1018200000416363656C65726174696F6E20287531
:101830006E6974732F7332293A20503C7072696E4E
:10184000745F616363656C3E20523C7265747261C3
:1018500063745F616363656C3E20543C74726176AF
:10186000656C5F616363656C3E0020204D323031F2
:101870002058004D6178696D756D20416363656C1A
:1018800065726174696F6E2028756E6974732F7349
:1018900032293A0020204D3230332058004D6178F3
:1018A000696D756D20666565647261746573202865
:1018B000756E6974732F73293A00537465707320C1
:1018C00070657220756E69743A0020440020204DC6
:1018D0003230302053002044697361626C65640AC1
:1018E0000046696C616D656E742073657474696E11
:1018F00067733A0020204D3134392043203B205576
:101900006E69747320696E2043656C736975730A20
:101910000020286D6D290020204732312020202012
:101920003B20556E69747320696E206D6D000080D8
:101930003B4400803B4400002041000096420000F0
:10194000A0420000A0420000C8430000BE42D007F1
:101950000000D0070000640000004B00000024F4E9
:10196000D43050C38E20C2A24017828B7011127ADD
:10197000910D816CD90AA861E108C75866076151C9
:1019800043061E4B5D05C145A7041A411104093DDC
:101990009803713931034036DB0265339102D4304C
:1019A0005402802E1D02632CEE01752AC501B02859
:1019B000A001102781018F2564012B244B01E02217
:1019C0003401AC211F018D200D01801FFC00841EFD
:1019D000ED00971DDF00B81CD200E61BC600201BDF
:1019E000BC00641AB200B219A8000A19A0006A1853
:1019F0009900D117910040178B00B516840031165D
:101A00007E00B31579003A157300C7146F0058149F
:101A10006A00EE1366008813630025135E00C71288
:101A20005B006C12570015125400C1115100701167
:101A30004F0021114B00D61049008D104700461071
:101A4000440002104200C00F4000800F3E00420FD1
:101A50003C00060F3B00CB0E3800930E37005C0EA7
:101A60003500270E3400F30D3200C10D3100900D0A
:101A70003000600D2E00320D2D00050D2C00D90C0C
:101A80002B00AE0C2900850C29005C0C2700350CBE
:101A900027000E0C2600E80B2400C40B2400A00B2A
:101AA00023007D0B23005A0B2100390B2100180B5A
:101AB0002000F80A1F00D90A1E00BB0A1E009D0A5A
:101AC0001D00800A1D00630A1C00470A1B002C0A27
:101AD0001B00110A1A00F7091A00DD091900C409D0
:101AE0001900AB091900920917007B091800630956
:101AF00017004C09160036091600200916000A09BD
:101B00001500F5081500E0081400CC081400B8080A
:101B10001400A4081400900813007D0812006B083C
:101B20001300580812004608120034081100230858
:101B300011001208110001081100F0071000E00761
:101B40001000D0071000C0071000B0070F00A10759
:101B5000100091070E0083070F0074070F00650740
:101B60000E0057070E0049070E003B070D002E0719
:101B70000E0020070D0013070D0006070D00F906E3
:101B80000C00ED060D00E0060C00D4060C00C806A3
:101B90000C00BC060C00B0060C00A4060B00990655
:101BA0000C008D060B0082060B0077060B006C06FE
:101BB0000B0061060A0057060B004C060A0042069D
:101BC0000A0038060A002E060A0024060A001A0631
:101BD0000A001006090007060A00FD050900F405C1
:101BE0000900EB050900E2050900D9050900D00547
:101BF0000900C7050900BE050900B5050800AD05C7
:101C00000800A50509009C050800940508008C053E
:101C10000800840508007C050800740508006C05B0
:101C20000700650508005D050700560508004E051C
:101C30000700470507004005080038050700310583
:101C400007002A050700230507001C0506001605E6
:101C500007000F0507000805060002050700FB0442
:101C60000600F5040700EE040600E8040600E2049E
:101C70000700DB040600D5040600CF040600C904F3
:101C80000600C3040600BD040600B7040600B10444
:101C90000500AC040600A6040600A00405009B0491
:101CA000060095040500900406008A0405008504DA
:101CB0000500800406007A04050075040500700420
:101CC00005006B04050066040500610405005C0462
:101CD000050057040500520405004D0405004804A2
:101CE0000500430405003E0404003A0405003504E1
:101CF0000500300404002C0405002704040023041C
:101D000005001E0404001A04040016040500110452
:101D100004000D0404000904050004040400000488
:101D20000400FC030400F8030400F4030400F003BF
:101D30000400EC030400E8030400E4030400E003EF
:101D40000400DC030400D8030400D4030400D0031F
:101D50000400CC030400C8030300C503030024F4FB
:101D600004D9201BC40C5C0E9804C4095F026507EB
:101D70007101F405F900FB04B30048048700C103B6
:101D800069005803550003034500BE023A0084026F
:101D9000310053022A002902250004022000E40138
:101DA0001C00C8011900AF0117009801140084013C
:101DB0001300710110006101100051010E00430178
:101DC0000D0036010B002B010B0020010B0015014B
:101DD00009000C01090003010800FB000800F300E2
:101DE0000800EB000700E4000600DE000600D80053
:101DF0000600D2000600CC000500C7000500C200A6
:101E00000500BD000400B9000400B5000400B100E5
:101E10000400AD000400A9000400A5000300A20016
:101E200003009F0004009B0003009800030095003E
:101E3000020093000300900003008D0002008B005D
:101E40000300880002008600020084000300810075
:101E500002007F0002007D0002007B00020079008A
:101E60000200770001007600020074000200720098
:101E70000100710002006F0002006D0001006C00A3
:101E800002006A00010069000200670001006600AC
:101E900001006500010064000200620001006100B1
:101EA0000100600001005F0002005D0001005C00B5
:101EB00001005B0001005A000100590001005800B8
:101EC00001005700010056000100550001005400B8
:101ED00001005300000053000100520001005100B6
:101EE0000100500001004F0001004E0000004E00B4
:101EF00001004D0001004C0001004B0000004B00B0
:101F000001004A00010049000100480000004800AB
:101F100001004700010046000000460001004500A6
:101F200000004500010044000100430000004300A0
:101F30000100420000004200010041000000410099
:101F40000100400001003F0000003F0001003E0092
:101F500000003E0001003D0000003D0001003C008B
:101F600000003C0000003C0001003B0000003B0082
:101F700001003A0000003A00010039000000390079
:101F80000100380000003800000038000100370070
:101F90000000370001003600000036000000360067
:101FA000010035000000350000003500010034005C
:101FB0000000340000003400010033000000330052
:101FC0000000330001003200000032000000320047
:101FD000010031000000310000003100010030003C
:101FE000000030000000300001002F0000002F0032
:101FF00000002F0000002F0001002E0000002E0026
:1020000000002E0001002D0000002D0000002D001A
:1020100000002D0001002C0000002C0000002C000E
:1020200000002C0001002B0000002B0000002B0002
:1020300000002B0001002A0000002A0000002A00F6
:1020400000002A00010029000000290000002900EA
:1020500000002900000029000100280000002800DD
:1020600000002800000028000000280001002700D0
:1020700000002700000027000000270000002700C4
:1020800001002600000026000000260000002600B7
:1020900000002600010025000000250000002500AA
:1020A000000025000000250000002500010024009C
:1020B0000000240000002400000024000000240090
:1020C0000100230000002300000023000000230083
:1020D0000000230000002300000023000100220074
:1020E0000000220000002200000022000000220068
:1020F000000022000100210000002100000021005A
:10210000000021000000210000002100000021004B
:10211000010020000000200000002000000020003E
:10212000000020000000200000002000000020002F
:1021300001001F0000001F0000001F0000001F0022
:1021400000001F0000001F0000001F0001001E0013
:1021500000001E0000001E0000001E0000000437EA
:1021600000001E290000511B00005810000010093B
:102170000000CC0400007802000041010000204370
:102180006F756E7420583A004265640045310062F4
:102190006564002C2073797374656D2073746F709F
:1021A00070656421204865617465725F49443A2016
:1021B0000048656174696E67204661696C656400FA
:1021C00048656174696E67206661696C6564004D7D
:1021D0003131322053687574646F776E001000C916
:1021E0000210012C014001220170011801B0010E02
:1021F00001F00104015002FA00B002F0003003E6E1
:1022000000D003DC009004D2007005C800A006BE18
:10221000000008B400B009AA00D00BA000600E9620
:102220000060118C000015820020197800C01D6E1E
:1022300000A0226400B0275A00902C5000003146C4
:1022400000E0343C0010383200903A2800603C1E18
:1022500000A03D1400803E0A00203F000054484585
:10226000524D414C2052554E4157415900546865DA
:10227000726D616C2052756E617761790045727282
:102280003A204D415854454D50004D415854454D0C
:102290005020747269676765726564004572723AAE
:1022A000204D494E54454D50004D494E54454D50DA
:1022B0002074726967676572656400202F00204290
:1022C000403A0020403A007C3C3E5E2B3D3F2F5B75
:1022D0005D3B2C2A225C0043616E6E6F74206F7030
:1022E000656E2073756264697220005344206361D7
:1022F0007264206F6B0A006F70656E526F6F74208E
:102300006661696C65640A00766F6C756D652E692F
:102310006E6974206661696C65640A004E6F2053B3
:102320004420636172640A000A4D3234004D323336
:10233000202573002E0A006F70656E206661696C3F
:1023400065642C2046696C653A200046696C6520FE
:1023500073656C65637465640A002053697A653A35
:10236000200046696C65206F70656E65643A2000D8
:10237000454E4420535542524F5554494E450A004C
:102380002220706F73002220706172656E743A2291
:1023900000535542524F5554494E452043414C4CF1
:1023A000207461726765743A220053756263616CD0
:1023B0006C204F766572666C6F7700457863656553
:1023C000646564206D617820535542524F555449DD
:1023D0004E452064657074683A0057726974696E7E
:1023E0006720746F2066696C653A200066726573B9
:1023F0006800646F696E67002066696C653A20004A
:102400004E6F7720002F6175746F25632E67006013
:1024100001F4017001EA019001E001B001D601D0A0
:1024200001CC010002C2013002B8016002AE01908D
:1024300002A401D0029A012003900170038601C01A
:10244000037C0130047201A004680120055E01B024
:1024500005540160064A0120074001F0073601F0EB
:10246000082C01100A2201500B1801C00C0E01505B
:102470000E04013010FA002012F0005014E600C0E3
:1024800016DC007019D200501CC800501FBE00702E
:1024900022B400B025AA00F028A000202C9600301D
:1024A0002F8C0010328200A0347800F0366E00E0ED
:1024B000386400803A5A00403B5500E03B5000F041
:1024C0003C4600C03D3C00603E3200E03E2800300B
:1024D0003F1E00503F1900703F1400A03F0A00C08B
:1024E0003F0000D03FF6FFE03FECFF2020506C6142
:1024F0006E6E657242756666657242797465733A8E
:1025000020002046726565204D656D6F72793A2016
:1025100000436F6D70696C65643A204170722032BF
:102520003420323032310A00204C617374205570EF
:1025300064617465643A20323032312D30342D318B
:1025400038207C20417574686F723A2054696E7926
:102550004D616368696E657333440A00322E302E14
:10256000375F4457372E330A004D61726C696E0035
:1025700020536F6674776172652052657365740AC3
:1025800000205761746368646F67205265736574D7
:102590000A002042726F776E206F75742052657347
:1025A00065740A002045787465726E616C2052650E
:1025B0007365740A00506F77657255700A00737402
:1025C0006172740A004732385859004D3130303149
:1025D000006F6B006572726F722077726974696E3A
:1025E0006720746F2066696C650A00446F6E652011
:1025F000736176696E672066696C652E0A004D32DC
:102600003900456E6473746F707300255320256321
:1026100020256320256320256300205A3A00205995
:102620003A0020583A00656E6473746F70732068C6
:1026300069743A2000000000010200090A0000004D
:102640000004030807000000000000000000000074
:102650000000000000004D6F76652025736D6D0051
:102660004D6F766520302E316D6D004D6F76652093
:10267000316D6D004D6F76652031306D6D004D6FA1
:102680007665204178697300457874727564657267
:10269000004D6F7665205A004D6F76652059004DCC
:1026A0006F76652058005072696E742066726F6D87
:1026B000204D6564696100FFFFFF486F6D6520254F
:1026C000732573257320466972737400220A0055BE
:1026D0006E6B6E6F776E20636F6D6D616E643A2006
:1026E00022004D696E692053755065522052656114
:1026F00064792E005072696E74696E672E2E2E00FA
:102700005072696E742050617573656400204500D5
:10271000205A00205900204D393220580020453AD7
:1027200000205A3A0020593A00583A004572726F18
:10273000722077726974696E6720746F2045455006
:10274000524F4D210A0020746F6F206C6F6E67200E
:10275000657874727573696F6E2070726576656ED8
:102760007465640A0020636F6C6420657874727508
:1027700073696F6E2070726576656E7465640A00A9
:10278000526573656E643A2000000022002500281F
:10279000002B0000002100240027002A0002020272
:1027A00002020202020404040404040404030303F6
:1027B00003030303030101010101010101010204FB
:1027C000081020408001020408102040800102040B
:1027D000081020408080402010080402012F2F6143
:1027E0006374696F6E3A000085D658DD11241FBEF0
:1027F000CFEFD0E4DEBFCDBF12E0A0E0B1E0E0E17A
:10280000F7ED01E00BBF02C007900D92AE31B107AA
:10281000D9F727E1AEE1B2E001C01D92A93BB207B2
:10282000E1F713E1C5EFD3E104C02197FE010E9457
:10283000DFE8C43FD107C9F70E94A9D70C947BEB0E
:102840000C9400008F929F92AF92BF92CF92DF9232
:10285000EF92FF92CF936B017C0120E030E0A90161
:102860000E94FAE187FD9FC06DEB77E386E095E378
:10287000A70196010E94F1E86B017C0120E030E0A5
:1028800040E251E40E9460E220E030E048EC52E493
:102890000E9460E24B015C0120E030E0A901C70129
:1028A000B6010E94FAE120E030E040EA50E487FF00
:1028B00004C020E030E040EA50ECC501B4010E94C1
:1028C000F1E820E030E040E251E40E9474E90E9427
:1028D000E6E96B017C018BE2F7FE09C0F094E0941D
:1028E000D094C094C11CD11CE11CF11C8DE28093DA
:1028F000D503C701B60120E137E240E050E00E9475
:10290000C0E88AE0882E912CA12CB12CCA01B90113
:10291000A50194010E94C0E8605D6093D603C701E1
:10292000B60128EE33E040E050E00E94C0E8CA0162
:10293000B901A50194010E94C0E8605D6093D703CE
:10294000C701B60124E630E040E050E00E94C0E854
:10295000CA01B901A50194010E94C0E8605D6093BD
:10296000D8038EE28093D903C701B601A501940173
:102970000E94C0E8C62FCA01B901A50194010E94B6
:10298000C0E8605D6093DA03C05DC093DB0385ED52
:1029900093E0CF91FF90EF90DF90CF90BF90AF90FA
:1029A0009F908F9008956DEB77E386E095EB60CF75
:1029B0008F929F92AF92BF92CF92DF92EF92FF924F
:1029C000CF936B017C0120E030E0A9010E94FAE185
:1029D00087FDAAC06DEB77E386E095E3A70196013A
:1029E0000E94F1E86B017C0120E030E0A9010E9427
:1029F000FAE187FF9EC0C701B601905820E030E0A1
:102A000040E251E40E9460E220E030E040E251E424
:102A10000E9460E220E030E040EA50E40E94F1E8E9
:102A200020E030E040E251E40E9474E90E94E6E9CF
:102A30006B017C0180E28093D50360E280E1C816DF
:102A400087E2D806E104F1048CF0C701B60120E169
:102A500037E240E050E00E94C0E8CA01B9012AE034
:102A600030E040E050E00E94C0E8605D6093D60333
:102A700060E288EEC81683E0D806E104F1048CF029
:102A8000C701B60128EE33E040E050E00E94C0E804
:102A9000CA01B9012AE030E040E050E00E94C0E8FD
:102AA000605D6093D70360E284E6C816D104E10458
:102AB000F1048CF0C701B60124E630E040E050E0BC
:102AC0000E94C0E8CA01B9012AE030E040E050E0CD
:102AD0000E94C0E8605D6093D8038AE0882E912C44
:102AE000A12CB12CC701B601A50194010E94C0E838
:102AF000C62FCA01B901A50194010E94C0E8605D1A
:102B00006093D9038EE28093DA03C05DC093DB0348
:102B100085ED93E0CF91FF90EF90DF90CF90BF9045
:102B2000AF909F908F9008956DEB77E386E095EBE3
:102B300055CF20E030E040E251E4C701B60162CF5A
:102B4000CF93DF93EC01CB01BA010E9401E220E0B8
:102B500030E040E251E40E9474E920E030E0A90155
:102B60000E94F1E8688379838A839B83DF91CF9108
:102B700008950E9401E220E030E040E251E40E942A
:102B800074E920E030E0A9010E94F1E80C94D81427
:102B9000CF93DF93EC01CB01BA010E9401E220E068
:102BA00030E048EC52E40E9474E920E030E0A901F2
:102BB0000E94F1E8688379838A839B83DF91CF91B8
:102BC00008950E9401E220E030E048EC52E40E94C7
:102BD00074E920E030E0A9010E94F1E80C9422148D
:102BE000CF93DF93EC01CB01BA010E9401E220E018
:102BF00030E0A9010E94F1E8688379838A839B838E
:102C0000DF91CF910895CF93DF93EC01CB01BA010F
:102C10000E9401E220E030E0A9010E94F1E868830F
:102C200079838A839B83DF91CF910895CF93DF933C
:102C3000EC01CB01BA010E9401E22AE037ED43E248
:102C40005DE30E9474E920E030E0A9010E94F1E810
:102C50000E94EDE9688379838A839B83DF91CF911A
:102C60000895CF93DF93EC01CB01BA010E9401E2FA
:102C70002AE037ED43E25DE30E9474E920E030E0B2
:102C8000A9010E94F1E8688379838A839B83DF919D
:102C9000CF910895CF93DF93EC01CB01BA010E944D
:102CA00001E220E030E04AE754E40E9474E920E0C9
:102CB00030E0A9010E94F1E8688379838A839B83CD
:102CC000DF91CF910895FC0184910895FC018081EA
:102CD0000895FC0180E09191992329F0907C90382F
:102CE000D1F38F5FF8CF089511980000000087FDA1
:102CF00052C0419800000000119A00000000119895
:102D00000000000086FD53C0419800000000119AA9
:102D10000000000011980000000085FD46C04198A9
:102D200000000000119A000000001198000000004F
:102D300084FD39C0419800000000119A0000000095
:102D400011980000000083FD2CC041980000000095
:102D5000119A0000000011980000000082FD1FC0C1
:102D6000419800000000119A000000001198000036
:102D7000000081FD12C0419800000000119A00007F
:102D80000000119800000000419800000000119A16
:102D9000000000000895419AADCF419AEDCF419ACD
:102DA000E0CF419AD3CF419AC6CF419AB9CF419A49
:102DB000ACCF90E080E00895CF93DF93DB01F90181
:102DC0009C919130C1F0943080F094509C93883065
:102DD000D1F480819181009771F001979183808374
:102DE000480F591FEA01188206C08C3539F49C5FE0
:102DF0009C93943041F4DF91CF9108958B3339F750
:102E000081E08C93F8CF20813181B9016F5F7F4FD2
:102E100071836083420F531FEA018883808191810F
:102E20008F3591056CF7E7CF0F931F9381E00091E9
:102E3000C2161091C3162091C4163091C516409148
:102E4000BE165091BF166091C0167091C11604173E
:102E500015072607370708F480E01F910F910895A2
:102E6000282F90914003833021F495FD0FC094FDED
:102E70000FC0892F90E0B0E0A0E004C0B695A79500
:102E8000979587952A95D2F78170089581E00895E6
:102E900080E0089580915301882341F06091D00330
:102EA0007091D10341E081E00C940ABC089563E97C
:102EB00072E084E690E00E9498946AEB72E084E607
:102EC00090E00C94989481110C94571768EB71E082
:102ED00084E190E00C949894CF93DF9300D000D0DD
:102EE000CDB7DEB70E94EDE90E94FFE169837A83E6
:102EF0008B839C83CE0101960E94BE900F900F9011
:102F00000F900F90DF91CF9108950E9401E22AE087
:102F100037ED43E25DE30E9474E920E030E0A9016F
:102F20000E94F1E80C946C17CF92DF92EF92FF921F
:102F3000CF93DF9300D000D0CDB7DEB76B017C011B
:102F400020E030E0A9010E94FAE187FD1BC06DEB93
:102F500077E386E095E3A70196010E94F1E8698393
:102F60007A838B839C83CE0101960E94BE900F9042
:102F70000F900F900F90DF91CF91FF90EF90DF9027
:102F8000CF9008956DEB77E386E095EBE4CF0E9458
:102F900001E22AE037ED43E25DE30E9474E920E0BC
:102FA00030E0A9010E94F1E80C9494170E9401E21C
:102FB00020E030E0A9010E94F1E80C949417CF9230
:102FC000DF92EF92FF926B017C0120E030E0A901DB
:102FD0000E94FAE187FD26C06DEB77E386E095E37A
:102FE000A70196010E94F1E86B017C0120E030E02E
:102FF000A9010E94FAE120E030E040E05FE387FFB2
:1030000004C020E030E040E05FEBC701B6010E9461
:10301000F1E80E94E6E9CB01FF90EF90DF90CF90BE
:103020000C945C926DEB77E386E095EBD9CF0E9430
:1030300001E220E030E0A9010E94F1E80C94DF17E2
:103040000E9401E220E030E04AE754E40E9474E983
:1030500020E030E0A9010E94F1E80C94C594EF92C1
:10306000FF920F931F938EE7E82E8DE0F82E01E973
:103070001DE030E020E043E75DE160E87DE087E8C7
:103080009DE00E949EC41F910F91FF90EF900895C4
:103090000E9467740C9463170E941A8F0C94571740
:1030A0000C9478770C9478770C9478770C947877E4
:1030B0000C942A770C942A770C942A770C942A770C
:1030C0000E9456A60C946317AF92BF92CF92DF92E4
:1030D000EF92FF920F931F93CF93DF936B01E90160
:1030E0004A3009F4B8C0453109F06AC0DB011296D4
:1030F000ED91FC91F280C681D781139A88E28A957E
:103100000000E9F7BF2CB29420EFB22230E1A32EE9
:10311000AF0C48E2E42E88EF0E9474168E2D8A953B
:103120000000E9F7BFE1BF1508F481C08F2D80775B
:1031300080680E9474168B2D0E9474168E2D8A95BD
:103140000000E9F780E80E94741680E00E9474167F
:103150008E2D8A950000E9F78AEF0E9474168E2D55
:103160008A950000E9F78E01005F1F4F8881807FFC
:103170000E94741689918295807F0E947416C017F0
:10318000D107A1F78E2D8A950000E9F7F394E0E1CD
:10319000BE0EFA10C0CF1398D6011296CD91DC91D5
:1031A000CE010E946BC28111EEC1DF91CF911F91C0
:1031B0000F91FF90EF90DF90CF90BF90AF90089568
:1031C000FB0102811381423309F498C108F49CC1C8
:1031D000463409F489C1473409F48CC14B3329F5CD
:1031E00089812B81D80112966C91129713964C917C
:1031F000213009F4DFC1233009F0A9C138EF380FBD
:10320000582F91E0431708F490E041E0531708F07D
:1032100040E031E0561708F430E0592F542B3523A5
:1032200009F0BDC1942309F0BAC181E0BECF80EEA0
:103230008F0D8068807F0E9474168F2D8295807F0D
:103240000E9474168E2D8A950000E9F780E80E948E
:10325000741680E87BCF0B9A1398399A4198099A93
:10326000119A139A88E28A950000E9F788E790E0BE
:10327000CEE9DFE0FE013197F1F70197D9F788EF4A
:103280000E94741618E2812F8A950000E9F780E207
:103290000E94741680E00E947416812F8A950000A7
:1032A000E9F780E00E94741680E80E947416812F6E
:1032B0008A950000E9F780E00E94741680E10E9480
:1032C0007416812F8A950000E9F7CE010197F1F776
:1032D000CE010197F1F7CE010197F1F7CE010197E9
:1032E000F1F7CE010197F1F7CE010197F1F7CE0189
:1032F0000197F1F7CE010197F1F7CE010197F1F7B0
:10330000CE010197F1F7CE010197F1F7CE010197B8
:10331000F1F7CE010197F1F7CE010197F1F721976F
:10332000F1F780E20E94741680E40E947416812FE7
:103330008A950000E9F780E20E94741680E60E94F8
:1033400074161A950000E9F710E0D0E0C8E28D2F5E
:10335000807780680E947416812F0E9474168C2FCB
:103360008A950000E9F780E80E94741680E00E94C8
:1033700074168C2F8A950000E9F78AEF0E94741664
:103380008C2F8A950000E9F780E211980000000078
:10339000419800000000119A000000001198000000
:1033A0000000419800000000119A000000001198F0
:1033B00000000000419800000000119A0000000089
:1033C000119800000000419800000000119A0000D0
:1033D0000000119800000000419800000000119AC0
:1033E000000000001198000000004198000000005B
:1033F000119A0000000011980000000041980000A0
:103400000000119A0000000011980000000041988F
:1034100000000000119A0000000011980000000058
:10342000419800000000119A00000000119800006F
:103430000000419800000000119A0000000011985F
:1034400000000000419800000000119A00000000F8
:10345000119800000000419800000000119A00003F
:103460000000119800000000419800000000119A2F
:1034700000000000119800000000419800000000CA
:10348000119A00000000119800000000419800000F
:103490000000119A000000001198000000004198FF
:1034A00000000000119A000000009C2F9A95000077
:1034B000E9F7815009F069CF88EF0E9474168C2FCC
:1034C0008A950000E9F7DF5F105FD03209F03FCF47
:1034D00080E00E94741680EC0E947416CA95000069
:1034E000E9F7139881E061CED80115968C91888315
:1034F00081E05BCEF80181818883FACFB901C801F0
:103500000E9488C281E051CE443171F0473109F008
:103510008CCE1882F80182818983858181508A83CB
:1035200083818B8381E041CED80115964C9115970C
:1035300050E0440F551F70E060E016968D919C910D
:103540000E941CEBC8010E9481C281E02ECE481768
:1035500008F46BCE861708F468CEFA80E12CD12CE3
:10356000243070F41DC0BE01C8010E9488C2898148
:1035700098819D0D98838E0D8983FF0C09F455CE9B
:10358000F7FEF6CFF0CF4D8150E0440F551F70E0AD
:1035900060E08E819F810E941CEB81E006CEFA8064
:1035A00030E0F901EE58FE4FD08022593E4FF9012C
:1035B000E080E6CF58E0580F382F23CE2091480303
:1035C000022E000C330B8217130641F08093480340
:1035D0006BE07EE08AE495E10C9440C60895EF929A
:1035E000FF920F931F93CF93DF93EC018B017A012E
:1035F0008A859B858617970731F0888199810E947B
:1036000040C61B870A87B701888199810E94E0BC68
:103610002E813F81820F932F911D9F838E8390E097
:1036200080E0DF91CF911F910F91FF90EF9008956F
:103630009F92AF92BF92CF92DF92EF92FF920F9341
:103640001F93CF93DF93EC018B01942EA52E8A85D7
:103650009B858617970731F0888199810E9440C623
:103660001B870A8788859985019649F5BC800A8160
:103670008E81080FC880D980D6015596ED91FC91B6
:10368000C6010995B80EE92CFA2C10E0F70121913A
:103690007F01211127C08E819F81810F911D9F8302
:1036A0008E8390E080E0DF91CF911F910F91FF908A
:1036B000EF90DF90CF90BF90AF909F9008950E81D4
:1036C0001F81692D7A2D888199810E94E0BC800F2D
:1036D000912F911D288539852817390738F681E003
:1036E00090E0E1CF4B2D602FC6010E9498C6080FD5
:1036F000180FCCCFDF92EF92FF920F931F93CF93CF
:10370000DF93EC01D62E1CAD0BAD7C0184E0E80EFE
:10371000F11CE98DFA8DC7010995412F480F2D2D18
:10372000602FC7010E9498C69BAD890F8BAF81E0C7
:1037300090E0DF91CF911F910F91FF90EF90DF907C
:103740000895CF92DF92EF92FF920F931F93CF9342
:10375000DF93CDB7DEB72C970FB6F894DEBF0FBE60
:10376000CDBFF0908115E090821520914A03211180
:103770001DC045E75BE06E2D8F2D0E9404C790E0D1
:1037800080E0F80EF0928115E092821599272C9630
:103790000FB6F894DEBF0FBECDBFDF91CF911F9162
:1037A0000F91FF90EF90DF90CF900895C0904E154D
:1037B000D0904F152AE435E13A8329832F2D30E04C
:1037C0003C832B832E2D30E03E832D8318861F8271
:1037D0007A8769871C861B8608E11BE19E012F5FA3
:1037E0003F4F43E656E1BC01C6010E9451B6B60107
:1037F0008AE495E10E9440C68F819885C2CFEF92FE
:10380000FF920F931F93CF937C010091430310917C
:103810004403C0E0F701EC0FF11D6081662351F015
:10382000062E000C770BC8010E9441EB892B49F44E
:10383000CF5FF0CF80E0CF911F910F91FF90EF907D
:10384000089581E0F8CF682F880F770B80914303AC
:10385000909144030E9441EBFC0181E0309709F410
:1038600080E0309781F0918120ED290F2A3030F0EF
:103870009E3251F4928190539A3098F43196F0939D
:103880003503E093340308959D3211F09B3249F4DF
:10389000928120ED290F2A3088F39E3211F4938112
:1038A000EACFF0E0E0E0EBCF809134039091350374
:1038B000009731F04AE050E070E060E00C941CE0CA
:1038C00060E070E0CB01089580913403909135035E
:1038D000009731F04AE050E070E060E00C94EEDEDA
:1038E00060E070E0CB0108950E94641CCB01089554
:1038F0000F931F93CF9380913403909135030097DA
:10390000E9F0FC018F01C1912C2F2F7D81F0C5348E
:1039100011F0C536B9F7F801108270E060E00E943E
:1039200090DDF801C083CF911F910F91089570E051
:1039300060E0CF911F910F910C9490DD60E070E0FA
:10394000CB01F1CFCF93DF93CDB7DEB720E24F812C
:1039500058856E818D810E9467BCDF91CF9108955B
:103960008F929F92AF92BF92EF92FF920F931F930D
:10397000CF93DF93EC018B01E42EF22E809144155E
:10398000909145158C179D0709F43EC02091CA03FC
:1039900027FD1092CA032AE9C039D20709F03FC0B7
:1039A0008250944371F40E9480C16E517B4F8F4FBF
:1039B0009F4F6093CC037093CD038093CE0390937D
:1039C000CF03D0934515C093441530E020E0009319
:1039D000CE051093CF052093D0053093D105E0920A
:1039E000C705F092C805C250D44321F41092C60511
:1039F0001092CB0382E08093530181E08093DE0537
:103A00001092D4031092C505DF91CF911F910F91B1
:103A1000FF90EF90BF90AF909F908F90089524E318
:103A2000C230D20771F680599A4919F0C2E0D4E346
:103A3000C8CF0E9480C18090CC039090CD03A0900D
:103A4000CE03B090CF03681979098A099B0997FFC3
:103A5000EDCF809194058770873041F7CEE6D6E6AA
:103A6000B0CF80911E1590911F15891B8F7051F456
:103A700080910006813031F08091C61682FB882744
:103A800080F9089581E00895E091CB03E63010F5C8
:103A900081E08E0F8093CB034091CE055091CF05EE
:103AA0006091D0057091D1059091C7058091C805AE
:103AB00028E0E29FF0011124E656FC4F20914415C6
:103AC000309145153183208342835383648375830A
:103AD00096838783089520E040E070E060E082E014
:103AE00094E30C94B01CCF930E941A8F0E946774C9
:103AF000C82F882319F080E00E9482A08C2F0E949A
:103B00006317CF910C946B1DE091CB03EE2389F0EA
:103B1000E150E093CB0388E0E89FF0011124E656E2
:103B2000FC4F6281738127814681808191810C9451
:103B3000B01C0C946B1D8091D203811106C01092B1
:103B4000C6050E94841D0E94571780915301882347
:103B500031F041E06FEE7DE081E00E940ABC82E03E
:103B60008093530108954F925F926F927F928F924C
:103B70009F92AF92BF92CF92DF92EF92FF920F93FC
:103B80001F93CF93DF930E94311D782E0E9493BD27
:103B9000C091C70515E0711001C016E06C2E85E0DC
:103BA000582E5C0E05E00C1B84E0F82EFC1A83E016
:103BB000E82EEC1A82E0982E9C1A9CE8A92E9DE033
:103BC000B92E20EDC22E2DE0D22E81E0882E8C1A47
:103BD0004C2E4194C11132C08091C905882389F0CF
:103BE00080915301882309F447C081E09091C90571
:103BF000911180E024E041EE5DE0642D0E9467BCFD
:103C00003BC08091C4051092C405882349F30E94EB
:103C1000841D8091DE05882319F3DF91CF911F91D8
:103C20000F91FF90EF90DF90CF90BF90AF909F905B
:103C30008F907F906F905F904F900895C13009F002
:103C40005BC08091C905813009F443C08091530164
:103C5000882391F01F92DF92CF928F9281E0909112
:103C6000C905913009F080E08F930E94A21C0F904B
:103C70000F900F900F900F90711079C0C53009F020
:103C800076C08091C905853009F49EC080915301AA
:103C90008111ABC0D6E081E08D0F8C1313C09091E1
:103CA000C9059C1709F4CCC080915301882351F0B9
:103CB0006C2F661981E09C1380E023E041E95DE010
:103CC0000E9467BCCF5FC51185CFDE5FD093C8056A
:103CD000A4CF8091C4051092C405882309F4B6CFFF
:103CE000B092A205A092A1050E946B1D8091DE05F5
:103CF000882309F4ABCF91CFC23009F0C2C08091C4
:103D0000C905823081F080915301882309F4B4CF32
:103D100081E09091C905923009F080E023E047EC02
:103D20005DE0692D6BCF8091C4051092C405882396
:103D300051F38CE496E20E94F9948091DE05882389
:103D400011F36BCF8091C9058330F1F0809153015D
:103D5000882309F491CF81E09091C905933009F04F
:103D600080E023E04AEB5DE06E2D0E9467BC1C13EF
:103D700009C08091C905811709F444C0809153019D
:103D8000811151C0D12F87CF8091C4051092C405F5
:103D90008823E1F28CE198E20E94F9948091DE059B
:103DA0008823A1F23ACF8091C4051092C4058823DC
:103DB00009F472C085E19BE20E94F9948091DE05CE
:103DC000882309F469C029CF8091C4051092C405E5
:103DD000882309F45BCF83EF9CE20E94F9948091E1
:103DE000DE05882309F452CF18CF81E09091C905F0
:103DF000953009F080E023E04CEA5DE0602F0E94FE
:103E000067BC48CF8091C4051092C405882309F48B
:103E1000B5CF82E29EE20E94F9948091DE0588236C
:103E200009F4ACCFFACE6C2F661981E09091C905E8
:103E30009C1380E023E043EA5DE00E9467BCA2CFD0
:103E40008091C4051092C405882309F42DCF0E94E7
:103E5000441D20E040E070E060E08FE298E1DF91F7
:103E6000CF911F910F91FF90EF90DF90CF90BF9077
:103E7000AF909F908F907F906F905F904F900C9439
:103E8000B01CC33009F45ECFC43009F0F5CE809188
:103E9000C905843009F487CF80915301882309F440
:103EA000EBCE81E09091C905943009F080E023E0E9
:103EB00045EB5DE06F2D59CFCF93DF93CDB7DEB7E4
:103EC0008D8190919612891768F0809396129E01C9
:103ED000285F3F4F4E815F816AE270E08BE692E19E
:103EE0000E94C1E1DF91CF9108950F931F93CF936B
:103EF000DF938C016F3F19F41092961260E02091CD
:103F00009612862F062E000C990B2817190609F019
:103F1000F4F460939612C8010E9447E1800F911F4C
:103F2000EC01C01BD10BCB32D1053CF00197FC0159
:103F30002491207C2038D1F3F3CFDD27AE01B801E6
:103F40008BE692E10E9468E1C559DD4E1882DF914F
:103F5000CF911F910F910895CF938091920381117A
:103F600009C08FE89CE09093D1038093D00381E057
:103F7000809392030E94441D20E040E070E060E0E6
:103F80008AE497E10E94B01CC1E0C093C6050E947C
:103F90009C771092C6050E94841DC093C60560E000
:103FA00080E097E20E94751F8BE89CE09093A20549
:103FB0008093A105CF910895109291031092520120
:103FC0008091C61680648093C61686E79CE00E94A6
:103FD0007EB560E08DE79CE00E94751F0C946B1D20
:103FE0000F931F930E9480C100918D0310918E0347
:103FF00020918F0330919003601B710B820B930B08
:1040000097FD0CC089B183FB882780F991E089274F
:104010004A9B8260309B846080938C0380918C03E8
:10402000817090918C0391FD826090918B03981721
:1040300049F0813009F148F0823079F0833091F015
:1040400080938B031F910F910895913079F09230F6
:10405000B9F790918A0391500CC0992339F09330AD
:10406000C1F3EECF9130A9F3923051F790918A03CA
:104070009F5F90938A03E4CF992359F3933001F71C
:10408000F5CFCF92DF92EF92FF92CF93C82F0E948D
:1040900080C16B017C0124EA30E74DE75FE360916A
:1040A0001B0170911C0180911D0190911E010E94C5
:1040B000FAE187FD18C08AEF90E0A0E0B0E08C0D37
:1040C0009D1DAE1DBF1D80937A0390937B03A0932B
:1040D0007C03B0937D03C0931901CF91FF90EF90C3
:1040E000DF90CF90089580E090E0DC01E8CFCF939F
:1040F00080914B03811154C010928115109282154A
:104100001092831510924F1510924E151092511562
:10411000109250151092531581E08093521582E24F
:10412000809354151092591510925815EDE6F5E14B
:104130002BE735E18FEF81932E173F07E1F7C1E0C1
:10414000C0936A152CE037EA3093601520935F1511
:10415000C0936115109262151092631590E49093CC
:104160006415109265152AED36EA30937C1520937C
:104170007B1521E131E030934D1520934C159EE1E4
:104180009093711591E1909372159CE190936F1546
:1041900080936E1580936D150E94C9C2C0934B0326
:1041A00081E080934A0383EC9BE090939814809382
:1041B000971410929A141092991453985B9A5298EB
:1041C0005A9A3898409A0E94F01F10928A03CF9111
:1041D0000895FC01A081B1811C92A281B3818C91D0
:1041E0008F5F8C930280F381E02D90818CE0989F0B
:1041F000800D1124E6E4F5E113AE84AF0895FC01CF
:1042000080E09491992331F0907C903809F08F5F91
:104210003196F7CF0895AF92BF92CF92DF92EF928F
:10422000FF920F931F93CF93DF93EC015B018A0101
:10423000FB01099587FD16C0C82ED12CF12CE12C6D
:104240002196F801C082D182E282F382CE01DF9111
:10425000CF911F910F91FF90EF90DF90CF90BF9083
:10426000AF900895982F907E903CA9F48F7190E0C4
:10427000B0E0A0E06C017D0156E0CC0CDD1CEE1C32
:10428000FF1C5A95D1F7CE010196F50109958F7360
:10429000C82A2296D6CF982F907F903E11F58F7026
:1042A00090E0B0E0A0E06C017D0136E0CC0CDD1CBC
:1042B000EE1CFF1C3A95D1F7CE010196F501099548
:1042C0008F73C82A46E0CC0CDD1CEE1CFF1C4A95FF
:1042D000D1F7CE010296F50109958F73C82A23966E
:1042E000B0CF982F987F903F79F5877090E0B0E03D
:1042F000A0E06C017D0186E0CC0CDD1CEE1CFF1CF7
:104300008A95D1F7CE010196F50109958F73C82AD8
:1043100096E0CC0CDD1CEE1CFF1C9A95D1F7CE016B
:104320000296F50109958F73C82A26E0CC0CDD1C96
:10433000EE1CFF1C2A95D1F7CE010396F5010995D5
:104340008F73C82A24967DCF982F907C903841F4A3
:10435000807C803869F42196CE01F5010995F8CF6B
:104360008E7F8D3F28F02196CE01F5010995F8CF7B
:10437000C12CD12C760165CF9CE0899F802D112422
:1043800091E0980F909349032CE0280F2093E405C7
:1043900030E02E5F3F4F40917E154217130619F013
:1043A00014F080E00895209180159217D0F76623CD
:1043B00041F08E5F0E94EAC38091E4058E5F0E9407
:1043C000EAC38091E40590917E15891750F32091FE
:1043D000801590914903291720F31092811580933D
:1043E000821581E00895CF92DF92EF92FF920F93B2
:1043F0001F93CF93DF93CDB7DEB72C970FB6F8940A
:10440000DEBF0FBECDBF6F3F71058105910509F07D
:10441000D0F486E495E10E947A1BE0914E15F0916C
:104420004F153196849190E02C960FB6F894DEBF2C
:104430000FBECDBFDF91CF911F910F91FF90EF90F5
:10444000DF90CF900895F0908115E0908215209133
:104450004A0321110FC045E95BE06E2D8F2D0E94AC
:1044600004C790E080E0F80EF0928115E09282158A
:104470009927DACFC0904E15D0904F152AE435E138
:104480003A8329832F2D30E03C832B832E2D30E07F
:104490003E832D8318861F822FEF3FEF3A872987AF
:1044A0001C861B8608E11BE19E012F5F3F4FAB017D
:1044B000BC01C6010E948DB5B6018AE495E10E9457
:1044C00040C68F819885CFCFAF92BF92CF92DF92B7
:1044D000EF92FF920F931F93CF93DF9300D000D002
:1044E000CDB7DEB77C01062F6A01122F86E0A82E19
:1044F000B12C11160CF040C0AE014F5F5F4F63E668
:1045000076E1C7010E940B217C0169817A818B8150
:104510009C81611571058105910571F16D337105FE
:104520008105910509F450C06E377105810591052B
:1045300009F44AC06A3271058105910569F507FFE2
:1045400012C089EB9BE00E3F11F085EB9BE026E06B
:104550001202B00111240E94A11B66E070E00E94CB
:10456000ACE8161B61C065E470E080E090E00E945A
:10457000F321115059F510E0812F0F900F900F90FB
:104580000F90DF91CF911F910F91FF90EF90DF90EF
:10459000CF90BF90AF900895643271058105910569
:1045A00079F4C114D10461F026E01202B0011124A3
:1045B000C6010E94A11BB5010E94ACE8161B99CF51
:1045C0000E94F321115095CF07FDBBCF61E0898197
:1045D0009A81AB81BC81CD97A105B10509F460E05A
:1045E000600F6A30ACF01150862F6AE00E948AE8B2
:1045F000092F682F880F770B605D7F4F072E000C07
:10460000880B990B0E94F321112309F4B4CF602F7A
:10461000062E000C770B605D7F4F072E000C880B79
:10462000990B0E94F3211150112309F4A4CF86E0C5
:104630001802B0011124C7010E94A11B66E070E0BE
:104640000E94ACE8161B98CF6FEF7FEF0C94A11B74
:10465000CF92DF92EF92FF920F931F93CF93DF934E
:10466000CDB7DEB72C970FB6F894DEBF0FBECDBF27
:10467000F0908115E090821520914A0321111DC010
:1046800045E55BE06E2D8F2D0E9404C790E080E031
:10469000F80EF0928115E092821599272C960FB6AC
:1046A000F894DEBF0FBECDBFDF91CF911F910F9168
:1046B000FF90EF90DF90CF900895C0904E15D0906E
:1046C0004F152AE435E13A8329832F2D30E03C83CE
:1046D0002B832E2D30E03E832D8318861F827A8710
:1046E00069871C861B8608E11BE19E012F5F3F4FF7
:1046F00046E656E1BC01C6010E9451B6B6018AE405
:1047000095E10E9440C68F819885C2CF6FEF7FEF01
:104710000C942823AF92BF92CF92DF92EF92FF9238
:104720000F931F93CF93DF935C016B010E94FF20D7
:10473000E82EC6010E946916F12C03E110E0081B67
:104740001109C5E20E151F050CF4CFE18C2F90E086
:104750009C012E5F3F4F40917E154217130609F0D2
:10476000CCF5099720918015281719069CF14091E6
:10477000E6055091E7056091E50510928115C0931B
:10478000821525E1C5010E946422D1E0C114D10443
:10479000B1F06AE370E080E090E00E94F3210E1532
:1047A0001F05D4F4C45F80917E15C81740F0209196
:1047B00080154C2F4950550B241715067CF4DF91BA
:1047C000CF911F910F91FF90EF90DF90CF90BF900E
:1047D000AF900895D0E0DACFDD2389F3802F880FE2
:1047E000080F000F00938115C093821560E270E0FE
:1047F00080E090E00E94F321C601DF91CF911F91EC
:104800000F91FF90EF90DF90CF90BF90AF900C94FE
:104810008623CF92DF92EF92FF92CF93DF9300D067
:1048200000D0CDB7DEB78091C4051092C4058823AF
:1048300031F18091D3038F5F8093D3038931E0F00E
:1048400081E08093D20320E040E070E060E08BE9FB
:104850009DE10E94B01C85E09EE09093A2058093AC
:10486000A1050F900F900F900F90DF91CF91FF90C7
:10487000EF90DF90CF9008950E9454A0F2CF609106
:10488000CE057091CF058091D0059091D10561152D
:1048900071058105910509F43EC00E9401E22DECED
:1048A0003CEC4CEC5CE30E9460E220914C0B3091BC
:1048B0004D0B40914E0B50914F0B0E94F1E86B0154
:1048C0007C0120E030E040E850EC0E94FAE187FDF6
:1048D00053C020E030E040E850E4C701B6010E9438
:1048E00074EA18160CF44FC0C0924C0BD0924D0BCA
:1048F000E0924E0BF0924F0B8EE891E00E945F85A4
:1049000082E0809353011092CE051092CF05109251
:10491000D0051092D10580915301882309F4A1CFCD
:10492000C0904C0BD0904D0BE0904E0BF0904F0B85
:1049300020E030E0A901C701B6010E94FAE127E1B9
:1049400037EB41ED58E387FF04C027E137EB41ED3A
:1049500058EBC701B6010E94F1E869837A838B8323
:104960009C836BE2CE0101960E944191BC018EEFC7
:104970009DE00E948A2375CFC12CD12C90E8E92EAE
:1049800090ECF92EB1CFC12CD12C80E8E82E80E438
:10499000F82EAACF0F931F93CF93DF93FC01EB0167
:1049A0008091CE059091CF05A091D005B091D10511
:1049B000B7FF08C01092CE051092CF051092D00517
:1049C0001092D1058091D2059091D305A091D40584
:1049D000B091D5054091CE055091CF056091D0059D
:1049E0007091D10584179507A607B70744F4809303
:1049F000CE059093CF05A093D005B093D1058091BB
:104A000053018823E1F06091CE057091CF0580912C
:104A1000D0059091D1050091D6051091D705209130
:104A2000D8053091D905600F711F821F931F09951A
:104A3000BC018091DC059091DD050E948A23809164
:104A4000C405811108C08091CB058823D1F18091E4
:104A500053018823B1F18091DA059091DB0500972D
:104A6000B1F04091CE055091CF056091D005709185
:104A7000D1050091D6051091D7052091D805309128
:104A8000D905400F511F621F731FFE010995E09168
:104A9000CC05F091CD05309741F08091CB05811187
:104AA00003C08091C405811109958091C4051092BD
:104AB000C405882331F0DF91CF911F910F910C94A1
:104AC000841DDF91CF911F910F91089560EA75E1E8
:104AD00089EB95E10C94CA2468EC75E181EE95E1CF
:104AE0000C94CA2463E076E187E198E10C94CA242F
:104AF00066E176E185E897E10C94CA2461E376E10A
:104B000087EC97E10C94CA2460EF75E186ED97E19C
:104B10000C94CA246AE476E180E298E10C94CA24F9
:104B20008F929F92AF92BF92CF92DF92EF92FF92BD
:104B30000F931F93CF93DF93CDB7DEB72C970FB6AC
:104B4000F894DEBF0FBECDBF982F862F5A01790192
:104B5000D02E692F0E94BC21882309F487C01091B0
:104B60004A03C701002381F10E94FF20C82E8090D4
:104B70004E1590904F15111143C01FEF23E12C19D2
:104B80004091E6055091E7056091E505C5010E9459
:104B90006422CC2009F46AC0B6E08B9F5001112436
:104BA0006AE370E080E090E00E94F32157E0A516F0
:104BB000B10408F442C060E270E080E090E00E943E
:104BC000F321A81AB90AF2CF0E946916C82E809064
:104BD0004E1590904F15112381F2FE0133968AE015
:104BE000DF011D928A95E9F78AE495E19A8389832A
:104BF0000FEE1AE19E012F5F3F4F46E656E112C0CD
:104C0000FE0133968AE0DF011D928A95E9F78AE476
:104C100095E19A8389830FEE1AE19E012F5F3F4F42
:104C200043E656E1B701C4010E9451B6B4018AE4DB
:104C300095E10E9440C61F81A1CF4091E405212F3C
:104C400030E0A6E0CA9EC00111242E5F3F4F281716
:104C500039070CF49C0180E8821B809381154093F6
:104C60008215C701DD20A9F00E9424232C960FB6DF
:104C7000F894DEBF0FBECDBFDF91CF911F910F9192
:104C8000FF90EF90DF90CF90BF90AF909F908F906C
:104C900008950E948623EACF7F928F929F92AF92CF
:104CA000BF92CF92DF92EF92FF920F931F93CF9319
:104CB000DF930E9493BDC091C70565E0862E8C0EE0
:104CC000D6E0DC1B85E0D82EDC1A84E0C82ECC1A96
:104CD00083E0B82EBC1A82E0A82EAC1A81E0982E90
:104CE0009C1A7C2E7194C11134C08091C90588230F
:104CF000B1F080915301882359F081E09091C9056A
:104D0000911180E024E04CE65DE0672D0E9467BCD5
:104D1000CF5FC811E8CF87E08093C8050CC08091B1
:104D2000C4051092C405882321F30E94841D80913C
:104D3000DE058823F1F2DF91CF911F910F91FF9053
:104D4000EF90DF90CF90BF90AF909F908F907F902B
:104D50000895C130E9F58091C9058130E9F080916D
:104D600053018823A9F211E08091C905813009F02F
:104D700010E06091200B7091210B8091220B90919B
:104D8000230B0E94941700E09C0144EE5CE0692D27
:104D9000812F0E949025BCCF8091C4051092C4053C
:104DA0008823E9F20E9414BDE12C1CE3F12E0CE1F2
:104DB00016E420E030E040E85FE360E27BE084EE70
:104DC0009CE00E94E9BD8091DE05882341F2B3CFCB
:104DD000C23009F006C18091C9058230D9F08091B6
:104DE0005301882309F494CF11E08091C9058230E2
:104DF00009F010E06091240B7091250B8091260B37
:104E00009091270B0E94941700E09C014DED5CE00F
:104E10006A2DBECF8091C4051092C4058823F9F293
:104E20000E9414BDE12C1CE3F12E0CE116E420E0FD
:104E300030E040E85FE364E27BE08DED9CE00E94BF
:104E4000E9BD8091DE05882351F275CF8091C905B7
:104E50008330D9F080915301882309F459CF11E0B0
:104E60008091C905833009F010E06091280B7091A2
:104E7000290B80912A0B90912B0B0E94941700E034
:104E80009C0146ED5CE06B2D83CF8091C4051092B0
:104E9000C4058823F9F20E9414BDE12C1CE3F12E15
:104EA0000CE116E420E030E040E85FE368E27BE0FC
:104EB00086ED9CE00E94E9BD8091DE05882351F2D9
:104EC0003ACF8091C9058430D9F08091530188236D
:104ED00009F41ECF11E08091C905843009F010E07B
:104EE00060912C0B70912D0B80912E0B90912F0BBC
:104EF0000E94941700E09C014FEC5CE06C2D48CFC1
:104F00008091C4051092C4058823F9F20E9414BD53
:104F1000E12C1CE3F12E0CE116E420E030E040E847
:104F20005FE36CE27BE08FEC9CE00E94E9BD809146
:104F3000DE05882351F2FFCE8091C9058530D9F076
:104F400080915301882309F4E3CE11E08091C905D3
:104F5000853009F010E060913C0B70913D0B809121
:104F60003E0B90913F0B0E94941700E09C014AEC8D
:104F70005CE06D2D0DCF8091C4051092C40588238F
:104F8000F9F20E9414BDE12C1CE3F12E0CE116E4B1
:104F900020E030E0A9016CE37BE08AEC9CE00E9419
:104FA000E9BD8091DE05882359F2C5CE8091C40504
:104FB0001092C405882329F10E9414BDE12C1CE342
:104FC000F12E0CE116E420E030E0A90160E47BE082
:104FD00080EC9CE00E94E9BD8091DE05882389F089
:104FE000AACEC33009F432CFC43009F46ACFC53039
:104FF00009F4A2CFC63009F08BCE8091C905863066
:10500000A9F280915301882309F482CE11E08091A6
:10501000C905863009F010E06091400B7091410B9A
:105020008091420B9091430B0E94941700E09C01E9
:1050300040EC5CE06D2FACCE2F923F924F925F928E
:105040006F927F928F929F92AF92BF92CF92DF9298
:10505000EF92FF920F931F93CF93DF93CDB7DEB7FD
:105060002C970FB6F894DEBF0FBECDBFC090000BDB
:10507000D090010BE090020BF090030B8091040B99
:105080009091050BA091060BB091070B8C159D0517
:10509000AE05BF0510F4D701C601C090FC0AD09040
:1050A000FD0AE090FE0AF090FF0ABC01CD016C15EC
:1050B0007D058E059F0510F4C701B6010E94FFE132
:1050C0002B013C010E9493BD2091C7052B872E83A5
:1050D000822F8B5F8D8387E0922F821B8F8386E0E8
:1050E000821B888785E0821B898784E0821B8A87F0
:1050F00083E0282E221A82E0382E321A91959C875E
:105100002B85211142C08091C9058823C9F0809167
:105110005301882359F081E09091C905911180E0F5
:1051200024E04CE65DE06C850E9467BC8B858F5F58
:105130008B879D819813E4CF88E08093C8050CC0CD
:105140008091C4051092C405882309F30E94841D30
:105150008091DE058823D9F22C960FB6F894DEBF35
:105160000FBECDBFDF91CF911F910F91FF90EF90B8
:10517000DF90CF90BF90AF909F908F907F906F9077
:105180005F904F903F902F9008958B85813009F06C
:1051900089C08091C9058130F9F08091530188233D
:1051A00029F211E08091C905813009F010E0609189
:1051B000300B7091310B8091320B9091330B0E9428
:1051C000941761E02E81621B00E09C014AE15DE0E2
:1051D000812F0E949025AACF8091C4051092C4050A
:1051E0008823D9F20E9414BD2AE037ED43E25DE343
:1051F000C301B2010E9460E220E030E0A9010E94F8
:10520000F1E84B015C0120E030E040E05FE40E9407
:10521000FAE187FD05C0812C912CA12C3FE4B32E2F
:105220002AE037ED43E25DE36091300B7091310B82
:105230008091320B9091330B0E9460E220E030E0CD
:10524000A9010E94F1E820E030E040E85FE30E941D
:10525000F0E80E94EDE969837A838B839C83C50122
:10526000B4010E94E6E97B018C0121E0E21AF10819
:1052700001091109912C812C2EE7A22E25E2B22ED4
:10528000C980DA8021E030E040E050E060E37BE07C
:105290008AE19DE00E9420BD8091DE05882309F40B
:1052A0007CCF5ACF8B85823009F08EC18091C905A1
:1052B0008230D9F080915301882309F437CF11E06F
:1052C0008091C905823009F010E06091340B709133
:1052D000350B8091360B9091370B0E94941700E0AC
:1052E0009C0140E15DE0632D73CF8091C405109275
:1052F000C4058823F9F20E9414BD6091080B7091D7
:10530000090B80910A0B90910B0B0E94FFE17B012E
:105310008C0120E030E048EC52E464E37BE080E183
:105320009DE00E94E9BD8091DE05882319F214CF2B
:105330008091C9058330D9F080915301882309F405
:10534000F5CE11E08091C905833009F010E060913D
:10535000380B7091390B80913A0B90913B0B0E9466
:10536000941700E09C0147E05DE0622D31CF809111
:10537000C4051092C4058823F9F20E9414BD2AE0E6
:1053800037ED43E25DE3C301B2010E9460E220E039
:1053900030E0A9010E94F1E84B015C0120E030E01F
:1053A00040E05FE40E94FAE187FD05C0812C912C6A
:1053B000A12C9FE4B92E2AE037ED43E25DE3609132
:1053C000380B7091390B80913A0B90913B0B0E94F6
:1053D00060E220E030E0A9010E94F1E820E030E046
:1053E00040E85FE30E94F0E80E94EDE969837A8378
:1053F0008B839C83C501B4010E94E6E97B018C018B
:1054000021E0E21AF10801091109912C812C8EE7A3
:10541000A82E85E2B82EC980DA8021E030E040E095
:1054200050E068E37BE087E09DE00E9420BD809132
:10543000DE05882309F480CF8FCE8091C9058430A2
:10544000E9F080915301882309F470CE11E0809136
:10545000C905843009F010E06091FC0A7091FD0AE2
:105460008091FE0A9091FF0A0E94FFE10E946C1752
:1054700000E09C0140E05DE06A85AACE8091C40511
:105480001092C4058823E9F20E9414BD0EE518E1CC
:1054900024E630E040E050E06CEF7AE080E09DE010
:1054A0000E9486BE8091DE05882359F255CE8091F8
:1054B000C9058530E9F080915301882309F436CE7F
:1054C00011E08091C905853009F010E06091000B72
:1054D0007091010B8091020B9091030B0E94FFE1F0
:1054E0000E946C1700E09C0149EF5CE0698570CE7A
:1054F0008091C4051092C4058823E9F20E9414BD6E
:105500000CE518E124E630E040E050E060E07BE0AC
:1055100089EF9CE00E9486BE8091DE05882359F2C7
:105520001BCE8091C9058630E9F080915301882314
:1055300009F4FCCD11E08091C905863009F010E036
:105540006091040B7091050B8091060B9091070BF5
:105550000E94FFE10E946C1700E09C0142EF5CE0BA
:10556000688536CE8091C4051092C4058823E9F27F
:105570000E9414BD0AE518E12AE030E040E050E066
:1055800064E07BE082EF9CE00E9486BE8091DE05B5
:10559000882359F2E1CD8091C4051092C405882377
:1055A00039F10E9414BD08E518E124E630E040E03E
:1055B00050E068E07BE08BEE9CE00E9486BE80912C
:1055C000DE058823A9F0C8CD2B85233009F4B0CEA1
:1055D000243009F432CF253009F469CF263009F49C
:1055E000A0CF273009F0A2CD8091C905873099F26C
:1055F00080915301882309F499CD11E08091C90568
:10560000873009F010E06091080B7091090B8091D0
:105610000A0B90910B0B0E94FFE10E946C1700E0B7
:105620009C014BEE5CE06F81D3CD3F924F925F9235
:105630006F927F928F929F92AF92BF92CF92DF92A2
:10564000EF92FF920F931F93CF93DF930E9493BD2E
:10565000C091C705A5E04A2E4C0ED4E0DC1B83E0C8
:10566000782E7C1A82E0682E6C1A81E0582E5C1A23
:105670003C2E3194C11138C08091C9058823B1F006
:1056800080915301882359F081E09091C9059111CF
:1056900080E024E04CE65DE0632D0E9467BCCF5FB4
:1056A000C411E8CF85E08093C8050CC08091C40583
:1056B0001092C405882321F30E94841D8091DE0589
:1056C0008823F1F2DF91CF911F910F91FF90EF901E
:1056D000DF90CF90BF90AF909F908F907F906F9012
:1056E0005F904F903F900895C13009F05BC080916A
:1056F000C9058130E9F080915301882381F211E0DE
:105700008091C905813009F010E060910F06709119
:10571000100680911106909112060E94DF1700E09A
:105720009C0148E35DE0652D812F0E949025B7CF55
:105730008091C4051092C4058823E9F20E9414BD2B
:1057400020E030E0A90160910F0670911006809171
:105750001106909112060E94F1E820E030E040E846
:105760005FE30E94F0E80E94EDE9912C812CE2E7D2
:10577000AE2EE5E2BE2E6B011DEDE12E13E0F12E03
:1057800000E010E021E030E040E050E06FE076E043
:1057900088E39DE00E9420BD8091DE05882309F406
:1057A000AACF90CFC23009F0F8C08091C9058230ED
:1057B000D9F080915301882309F471CF11E08091D1
:1057C000C905823009F010E060911306709114064B
:1057D00080911506909116060E94DF1700E09C014B
:1057E00040E35DE0662DA0CF8091C4051092C40512
:1057F0008823F9F20E9414BD20E030E0A9016091F5
:1058000013067091140680911506909116060E9459
:10581000F1E820E030E040E85FE30E94F0E80E9419
:10582000EDE9912C812C42E7A42E45E2B42E6B01C8
:105830001DEDE12E13E0F12E00E010E021E030E05C
:1058400040E050E063E176E080E39DE00E9420BD0F
:105850008091DE05882309F4ACCF34CF8091C9054F
:105860008330D9F080915301882309F418CF11E0D7
:105870008091C905833009F010E06091170670919E
:1058800018068091190690911A060E94221400E0D1
:105890009C0148E25DE0672D47CF8091C4051092DE
:1058A000C4058823F9F20E9414BD20E030E048ECE2
:1058B00052E4609117067091180680911906909134
:1058C0001A060E9460E220E030E0A9010E94F1E89F
:1058D00020E030E040E251E40E94F0E80E94EDE96F
:1058E000912C812C2CE6A22E25E2B22E6B011EEA11
:1058F000E12E12E8F12E01E010E02AE030E040E075
:1059000050E067E176E088E29DE00E9420BD809152
:10591000DE05882309F4A6CFD5CE8091C405109268
:10592000C405882309F444C00E9414BD20E030E07F
:1059300048EC52E460911B0670911C0680911D0694
:1059400090911E060E9460E220E030E0A9010E94D2
:10595000F1E820E030E040E251E40E94F0E80E94EB
:10596000EDE9912C812C8CE6A82E85E2B82E6B01F6
:105970001EEAE12E12E8F12E01E010E02AE030E00C
:1059800040E050E06BE176E080E29DE00E9420BDC7
:105990008091DE05882361F095CEC33009F45ECF97
:1059A000C43009F07CCE8091C905843009F4B5CFAC
:1059B00080915301882309F472CE11E08091C905CA
:1059C000843009F010E060911B0670911C068091F4
:1059D0001D0690911E060E94221400E09C0140E2E8
:1059E0005DE06D2FA1CEBF92CF92DF92EF92FF923A
:1059F0000F931F93CF93DF930E9493BDC091C70570
:105A000085E0C82ECC0ED4E0DC1B13E01C1B82E02A
:105A1000F82EFC1A81E0E82EEC1ABC2EB194C111CC
:105A200030C08091C9058823B1F08091530188234B
:105A300059F081E09091C905911180E024E04CE695
:105A40005DE06B2D0E9467BCCF5FCC11E8CF85E095
:105A50008093C8050CC08091C4051092C4058823AA
:105A600021F30E94841D8091DE058823F1F2DF91ED
:105A7000CF911F910F91FF90EF90DF90CF90BF904B
:105A80000895C130B9F58091C9058130F1F0809158
:105A900053018823C9F2DD24D3948091C905813054
:105AA00009F0D12C6091100B7091110B8091120BA9
:105AB0009091130B0E94D81400E09C0141E65DE038
:105AC0006E2D8D2D0E949025BFCF8091C405109220
:105AD000C4058823E1F20E9414BD46E558E160E167
:105AE0007BE081E69DE00E9406BF8091DE05882371
:105AF00071F2BDCFC23009F07FC08091C9058230FC
:105B0000E1F080915301882309F49ECFDD24D394E2
:105B10008091C905823009F0D12C6091140B7091ED
:105B2000150B8091160B9091170B0E94D81400E072
:105B30009C0146E55DE06F2DC4CF8091C4051092B5
:105B4000C4058823F1F20E9414BD44E558E164E1E4
:105B50007BE086E59DE00E9406BF8091DE058823FC
:105B600081F285CF8091C9058330E1F080915301A6
:105B7000882309F469CFDD24D3948091C90583304B
:105B800009F0D12C6091180B7091190B80911A0BB0
:105B900090911B0B0E94D81400E09C014BE45DE047
:105BA000612F8FCF8091C4051092C4058823F1F234
:105BB0000E9414BD42E558E168E17BE08BE49DE082
:105BC0000E9406BF8091DE05882381F250CF80912C
:105BD000C4051092C4058823C9F00E9414BD40E595
:105BE00058E16CE17BE080E49DE00E9406BF80917B
:105BF000DE05882359F03BCFC33009F4B3CFC4305E
:105C000009F022CF8091C905843009F380915301B6
:105C1000882309F419CFDD24D3948091C9058430F9
:105C200009F0D12C60911C0B70911D0B80911E0B03
:105C300090911F0B0E94D81400E09C0140E45DE0AD
:105C40006D2F3FCF2F923F924F925F926F927F9234
:105C50008F929F92AF92BF92CF92DF92EF92FF927C
:105C60000F931F93CF93DF930E9493BDC091C705FD
:105C700035E0432E4C0E43E0342E55E3652E5FE5B0
:105C8000752ED1E0DC1B2C2E219482E0582E5C1A5C
:105C9000C11141C08091C9058823F1F08091530161
:105CA000882359F081E09091C905911180E024E0AA
:105CB0004CE65DE0622D0E9467BC8091060488235B
:105CC00009F4C3C0C23009F45CC083E0CF5FC411E3
:105CD000DFCF8093C8050CC08091C4051092C40525
:105CE0008823E1F20E94841D8091DE058823B1F2B1
:105CF000DF91CF911F910F91FF90EF90DF90CF90A8
:105D0000BF90AF909F908F907F906F905F904F90DB
:105D10003F902F900895C13081F68091C905813060
:105D2000C9F080915301882341F281E09091C90527
:105D3000913009F080E09091060423EB3CE0911152
:105D400002C02FEA3CE001E046EB5CE06D2F0E94D0
:105D50009025B3CF809106049091C4051092C4059C
:105D60009923F9F28C278093060430925301611431
:105D7000710411F00E94355F8091DE05882389F25D
:105D8000B7CF8091C9058230F1F08091530188230B
:105D900009F49BCF11E08091C905823009F010E031
:105DA00060910204709103048091040490910504B1
:105DB0000E94C59400E09C0145EA5CE0652D812FBE
:105DC0000E94902582CF8091C4051092C40588233B
:105DD000E1F20E9414BD20E030E04AE754E4609113
:105DE00002047091030480910404909105040E94C0
:105DF00060E220E030E0A9010E94F1E820E030E814
:105E00004BEB54E40E94F0E80E94EDE985E3882E14
:105E10008FE5982E9AE8A92E95E2B92E6B0116ED22
:105E2000E12E16E0F12E00E010E02CED35E040E030
:105E300050E062E074E085EA9CE00E9420BD809121
:105E4000DE05882309F4A1CF53CF82E03FCFE6E4FB
:105E5000F5E183AF64AFCA010C9486230F931F93BF
:105E6000CF9310924203109241032FE320934703F4
:105E700010924603109245039C01F90190812F5F17
:105E80003F4F9032D1F39E34C9F4818190ED980F49
:105E90009A3020F08D3211F08B3281F432969F01CE
:105EA0002F5F3F4F808180538A3008F468C09F0184
:105EB0002F5F3F4F8081803209F463C0F093F20579
:105EC000E093F1058F010F5F1F4FC0816AE270E020
:105ED000C8010E9441EB009731F0FC0131978081AD
:105EE0008032E1F31182CD3429F0C43519F0C73482
:105EF00009F041C0F80180810F5F1F4F8032D1F35C
:105F000080538A30C0F5C093470330E020E06AE058
:105F1000AF014F5F5F4F629FC001639F900D1124DF
:105F20009C01205331098081280F311D87FD3A954E
:105F3000FA01808180538A3058F3309346032093CE
:105F40004503CA01FC01019640814032D9F3F09328
:105F50004403E0934303CD3401F52E31310539F08C
:105F600090F42731310519F02C313105B1F4F0935B
:105F70004203E0934103CF911F910F910895F901DE
:105F80008ECFF90194CF2537310538F02737310509
:105F900070F3203A83E0380751F350E040E0CF013E
:105FA00001966081662309F45AC0613291F4CD34C0
:105FB00081F42032310569F49093420380934103C8
:105FC00063E270E00E9441EB0097A9F2FC011082AD
:105FD000D2CFFC01DF018D91803271F090ED980FEE
:105FE0009A3008F18E3251F4918190539A30D8F062
:105FF00041155105E1F414C0FD01ECCF8D3211F0D3
:106000008B3259F4918160ED690F6A3060F09E32F5
:1060100021F4928190539A3030F04115510519F4D2
:10602000AF014150510981548A3108F4B8CFDF01E2
:10603000FD018D91882309F4B2CF90ED980F9A302D
:10604000B8F393ED980F923098F38B3289F3CF0128
:1060500001966081603209F0A2CFFC01F8CF509325
:1060600042034093410387CF0E94641C97FD0CC0FC
:106070000E94641C6F3F71058105910509F034F49D
:106080000E94641C862F089580E008958FEF089584
:106090008091340390913503892B41F00E94343074
:1060A00091E0811101C090E0892F089591E0FCCF2B
:1060B0000E94231C882341F081E020913403309119
:1060C0003503232B09F480E00895CF93DF93EB0190
:1060D0000E945830882319F00E94641CEB01CE0105
:1060E000DF91CF910895CF93DF93C82FD62F0E94D1
:1060F0005830882321F0DF91CF910C9448308C2FB9
:106100000E94231C811101C08D2FDF91CF91089532
:1061100010926B0410926C0410926D0410926E0435
:10612000E7E0F4E084E6DF011D928A95E9F708953F
:10613000909101049817B1F00E949C77809101041E
:10614000882341F084E49BE00E94D57710920104FB
:106150000C94518681E08093010484E49BE00E94CA
:10616000BD77F6CF08959091010481E089270C94C2
:106170009830EF92FF920F931F93CF93DF9307E036
:1061800014E0C5E07801D5E0F7016191719181914A
:1061900091917F0120E030E0A9010E94FAE1811194
:1061A0000EC0D15089F7C1500C5E1F4FC111EACF0C
:1061B000DF91CF911F910F91FF90EF90089581E0B3
:1061C000F7CFEFE6F0E080818260808308954F9200
:1061D0005F926F927F928F929F92AF92BF92CF9277
:1061E000DF92EF92FF920F931F93CF93DF9300D034
:1061F00000D0CDB7DEB70E9480C14B015C01809119
:1062000019018F3F09F441C00E9480C1C0907A03F8
:10621000D0907B03E0907C03F0907D036C197D09A6
:106220008E099F0997FD31C080911E1590911F1511
:106230008F5F8F70891749F1E091190180E090E03C
:10624000A8E4B3E4E43050F424E0E29FF001112428
:10625000EA58FE4F80819181A281B38189839A831C
:10626000AB83BC83C12CD12C76018E010F5F1F4FF5
:1062700020E53BE04CE45BE068E47BE084E49BE009
:106280000E9437B98FEF809319010E94F01F80910F
:106290008C0382FF33C080918903811131C091E06A
:1062A000909389038091910389278093C40510926C
:1062B000910383E08093530110928C030E9480C16C
:1062C0006C507E4F8F4F9F4F60938D0370938E0362
:1062D00080938F039093900368E873E182E090E0ED
:1062E0000E94989416E0115059F00E943C9462E08C
:1062F00070E080E090E00E94E5C0F5CF1092890345
:106300008091850390918603A0918703B0918803C3
:10631000A5019401281B390B4A0B5B0BDA01C9015B
:10632000B7FF05C08091D403882309F4C6C1D50105
:10633000C4018C599F4FAF4FBF4F809385039093FB
:106340008603A0938703B093880360918A03062E87
:10635000000C770B77FF03C07195619571099091DF
:106360008A0380918403981365C0633008F062C08B
:1063700010928A0380918A0380938403643008F02A
:1063800069C08091C4058111E7C080914415909146
:1063900045158250944341F480911A01882309F4F1
:1063A000EDC0815080931A010E94C379C0903306DA
:1063B000D0903406E0903506F090360681110E94A8
:1063C000E130D701C6013AE0B695A7959795879534
:1063D0003A95D1F7009741E0A407B10520F08FEF7F
:1063E0009FEFA0E0B0E09695879520915301211191
:1063F000D7C03091D40331118EC180914415909152
:1064000045158250944309F46DC18091C6058111F0
:1064100069C18091800390918103A0918203B09122
:106420008303881A990AAA0ABB0AB7FC69C10E94A9
:106430006B1D66C1633009F09DCF80918A0387FD93
:1064400007C081E0880F880F80938A0364E092CFB1
:106450008FEFF8CF8091E30521E030E040E050E09D
:10646000882309F456C0C090DF05D090E005E09085
:10647000E105F090E205C114D104E104F104E9F171
:1064800070E090E080E00E94FFE120E030E040E832
:106490005EE30E9460E22B013C01C501B4016C196E
:1064A0007D098E099F090E94FFE19B01AC01C30198
:1064B000B2010E9474E920E030E04AE754E40E940F
:1064C00060E26B017C0120E030E042E053E40E9496
:1064D00074EA24E630E040E050E087FF12C020E09C
:1064E00030E040EA52E4C701B6010E9474EA2AE0B3
:1064F00030E040E050E087FF04C021E030E040E0C1
:1065000050E08092DF059092E005A092E105B09204
:10651000E205A0918A030A2E000CBB0B0E94E8E85A
:1065200024E030E040E050E00E94C0E88091CE05D9
:106530009091CF05A091D005B091D105820F931F06
:10654000A41FB51F8093CE059093CF05A093D005CF
:10655000B093D10510928A03D501C4018856954C99
:10656000AF4FBF4F8093800390938103A09382032A
:10657000B093830381E08093530107CF8CE0809335
:106580001A0180917E0390917F03009729F0019773
:1065900090937F0380937E0381E08093530104CF27
:1065A000009741F040917E0350917F0348175907AF
:1065B00008F023CF8091D40381111DC0223038F020
:1065C000243008F44CC0243011F41092530180910F
:1065D0008315811105C081E0809383150E94C9C293
:1065E00080914C1590914D150E94A2C281E080933C
:1065F000CA058093D40383E00E94DE1A81E0809371
:106600006A15E0914415F091451509951092CA0557
:106610008091D403811127C01092C4058091441544
:10662000909145158250944309F0EFCE0E9480C1AD
:10663000DC01CB0188199909AA09BB09C0907E0326
:10664000D0907F03F12CE12CC816D906EA06FB0690
:1066500008F0D3CE90937F0380937E03CECE81E06B
:1066600080935301B4CF8AE495E10E940EC691E075
:10667000811101C090E09093D403882369F2809146
:1066800044159091451582509443B9F40E9480C1FD
:10669000DC01CB0188199909AA09BB09C0907E03C6
:1066A000D0907F03F12CE12CC816D906EA06FB0630
:1066B00020F490937F0380937E030F900F900F90B0
:1066C0000F90DF91CF911F910F91FF90EF90DF908E
:1066D000CF90BF90AF909F908F907F906F905F9082
:1066E0004F90089548E9840E4AE3941EA11CB11C02
:1066F0008092800390928103A0928203B0928303E0
:106700008091D4038111D9CF809153018130A9F6B2
:1067100010925301D2CF009709F46DCF43CF8091EF
:10672000EC059091ED05892B79F48091EC05909121
:10673000ED05892B49F42091EC053091ED0581E0C0
:10674000232B19F480E0089581E00895CF92DF9221
:10675000EF92FF926B017C0183E3C816D104E10440
:10676000F10470F082E3C81AD108E108F10862E38D
:1067700070E080E090E00E94E5C00E945386ECCF7C
:10678000C701B6010E94E5C0FF90EF90DF90CF9067
:106790000C9453865E9A809194058E7F8093940525
:1067A0005E9A809194058D7F80939405159A8091CF
:1067B00094058B7F809394055E9A08959091C616F8
:1067C00093FB882780F993FF06C081E09091BB146A
:1067D000911101C080E008950E94B5BA0E94DE3395
:1067E000882351F08091C61682FD06C081EA9CE0A4
:1067F0009093A2058093A1058AE99CE00E947EB552
:106800000C9485904F925F926F927F928F929F929D
:10681000AF92BF92CF92DF92EF92FF920F931F93AE
:10682000CF93DF9300D000D01F92CDB7DEB7109288
:10683000E3058091C4051092C4058823E9F020E0A7
:1068400040E070E060E080E99AE90F900F900F90CF
:106850000F900F90DF91CF911F910F91FF90EF90CC
:10686000DF90CF90BF90AF909F908F907F906F9070
:106870005F904F900C94B01C20911F01309120012B
:106880004091CE055091CF05CA01820F931F243647
:10689000310509F015C44730510544F006978A3098
:1068A00091050CF01CC48AE090E023C406964A3F90
:1068B0005F4FACF38091CA05882309F4C0C12091D1
:1068C0000106309102064091030650910406609142
:1068D000440B7091450B8091460B9091470B0E94A1
:1068E000F1E84B015C0120910506309106064091CC
:1068F0000706509108066091480B7091490B8091F2
:106900004A0B90914B0B0E94F1E869837A838B8349
:106910009C832091090630910A0640910B06509104
:106920000C0660914C0B70914D0B80914E0B909129
:106930004F0B0E94F1E82B013C0120E030E040E2E7
:1069400051E40E9460E220E030E048EC52E40E9412
:1069500060E26B017C0120E030E0A901C301B201DB
:106960000E94FAE120E030E040EA50EC87FD04C0EC
:1069700020E030E040EA50E4C701B6010E94F1E8AF
:1069800020E030E040E251E40E9474E90E94E6E930
:106990002B013C0180E277FE09C070946094509412
:1069A0004094411C511C611C711C8DE28093D503E5
:1069B00060E2F0E14F16F7E25F06610471048CF0CB
:1069C000C301B20120E137E240E050E00E94C0E89C
:1069D000CA01B9012AE030E040E050E00E94C0E87E
:1069E000605D6093D60360E228EE421623E0520613
:1069F000610471048CF0C301B20128EE33E040E081
:106A000050E00E94C0E8CA01B9012AE030E040E04D
:106A100050E00E94C0E8605D6093D703C301B201FB
:106A200024E630E040E050E00E94C0E86AE0C62E74
:106A3000D12CE12CF12CCA01B901A70196010E94C9
:106A4000C0E8605D6093D803C301B201A70196015D
:106A50000E94C0E86D83CA01B901A70196010E9496
:106A6000C0E8CD80CC2009F454C38EE28093D903D2
:106A7000605D6093DA032C2D205D2093DB0365EDD0
:106A800073E082E793E00E944CEB20E030E0A90144
:106A9000C501B4010E94FAE120E030E040E05FEB84
:106AA00087FD04C020E030E040E05FE3C501B401B1
:106AB0000E94F1E80E94E6E9CB010E94DD91BC0151
:106AC0008DE693E00E944CEB20E030E0A901698163
:106AD0007A818B819C810E94FAE120E030E040E0E5
:106AE0005FEB87FD04C020E030E040E05FE36981B8
:106AF0007A818B819C810E94F1E80E94E6E9CB01BA
:106B00000E94DD91BC0188E693E00E944CEB40912D
:106B1000CA034F774983411127C00E94DE3388237F
:106B200019F18091BE169091BF16A091C016B09138
:106B3000C1160097A105B105B9F0BC01CD016D5991
:106B40007F4F8F4F9F4F24E630E040E050E00E949F
:106B500042E86091C2167091C3168091C41690915C
:106B6000C5160E9442E829830E943890B62E872ECF
:106B7000982EA92E6D8380911801C9808C15C1F0C3
:106B8000C092180128E4C29EB001112490E080E078
:106B90000E94FFE12AE037ED43E25CE30E9460E2FD
:106BA0000E94EDE960936703C110C5C210926203B1
:106BB00080911701CD80C81609F441C0B092170129
:106BC0006B2D782D892D9A2D20E13EE040E050E09C
:106BD0000E9442E869012CE3422E512C612C712C59
:106BE0006B2D782D892D9A2DA30192010E9442E8E8
:106BF000CA01B901A30192010E9442E824E6C2162B
:106C0000D10408F0BFC27F936F93DF92CF928DECD7
:106C10009BE09F938F9382E593E09F938F930E94D5
:106C200091E10FB6F894DEBF0FBECDBF85E0982F7F
:106C3000990F990F891B880F8058809351030E94E8
:106C400080C100914D0310914E0320914F0330916C
:106C500050036B017C01C01AD10AE20AF30A9701C2
:106C6000860137FD11C020914C03209520934C03E1
:106C70006A547C4F8F4F9F4F60934D0370934E0328
:106C800080934F0390935003D0904C03D98281E0BE
:106C90000E94DE1A80917E15843158F4809180150F
:106CA000883038F022E53CE04CE068E080E50E9466
:106CB00041C380917E158431A0F48091801582308B
:106CC00080F0E980EE2031F0809137062CE13CE045
:106CD000811102C026EE3BE042E162E088E60E94BC
:106CE00041C380917E158C3108F0D0C0E090A5148E
:106CF000F090A614883028F58091A7149091A814DC
:106D00000E945C92FC01808193E0803229F48181B1
:106D100092E0803209F491E043E050E0491B5109D0
:106D20004E0F5F1F892F880F880F981B892F67E0F0
:106D3000815F0E94272F69E070E080E090E00E9470
:106D4000F32180917E158C3130F58091801584314E
:106D500010F1C7010E945C92FC01808193E08032B7
:106D600029F4818192E0803209F491E043E050E01F
:106D7000491B51094E0F5F1F892F880F880F981BE1
:106D8000892F6CE1815F0E94272F69E070E080E02D
:106D900090E00E94F321E090A905F090AA0580916F
:106DA0007E15883028F58091AB059091AC050E9446
:106DB0005C92FC01808193E0803229F4818192E031
:106DC000803209F491E043E050E0491B51094E0F35
:106DD0005F1F892F880F880F981B892F67E0865ABD
:106DE0000E94272F69E070E080E090E00E94F3218C
:106DF00080917E158C3130F580918015843110F1B1
:106E0000C7010E945C92FC01808193E0803229F4EA
:106E1000818192E0803209F491E043E050E0491B27
:106E200051094E0F5F1F892F880F880F981B892FDC
:106E30006CE1865A0E94272F69E070E080E090E0C4
:106E40000E94F32180917E158C3100F58091801590
:106E50008431E0F0809137068823C1F024E6829FD8
:106E6000C001112481589F4F6FEF70E00E94ACE881
:106E7000CB010E945C92AC016CE187E60E94272F57
:106E800065E270E080E090E00E94F3210E94DE3332
:106E9000882369F180917E15843348F580918015AF
:106EA0008A3228F107E028E04AE26AE28AE495E1C2
:106EB0000E944AC405E022E04CE262E38AE495E1E4
:106EC0000E944AC46AE08AE20E9403C460914C15A1
:106ED00070914D1582E3809366158BE28093671560
:106EE00026E635E142E38AE495E10E949EC2809164
:106EF0007E15853340F480918015813320F06AE45B
:106F000086E30E9403C480917E15843368F48091E7
:106F10008015823348F002E02091670342E367E383
:106F20008AE495E10E944AC480917E158033D8F4AA
:106F3000809180158832B8F080916203882361F0D7
:106F400042E653E060E387E30E94272F65E270E0AA
:106F500080E090E00E94F32142E553E060E38091FD
:106F600051030E94272F80917E15873208F055C06B
:106F7000809180158F3108F450C083E08093811593
:106F800046E24093821568E570E080E090E00E9460
:106F9000F3218BE08093811566E260938215C980AE
:106FA000CC2009F404C18DE693E00E94862388E298
:106FB00080938115F6E2F093821569E570E080E038
:106FC00090E00E94F32180E38093811596E2C92E20
:106FD000C0928215D980DD2009F40AC188E693E0C9
:106FE0000E9486238DE480938115F6E2F09382154A
:106FF0006AE570E080E090E00E94F32185E58093EF
:10700000811586E2C82EC0928215D980DD2009F450
:1070100012C182E793E00E94862380917E1583331C
:1070200038F5809180158B3218F183E00E94DE1ACA
:1070300083E08093811583E38093821566E070E09E
:1070400080E090E00E94F32181E00E94DE1A8091AE
:107050001F01909120010E945C92AC0163E38CE0DF
:107060000E94272F65E270E080E090E00E94F3210B
:1070700080917E15813408F007C180918015863398
:1070800008F402C1109281158EE3809382158BE67D
:1070900092E10E946916898360E870E08BE692E1D4
:1070A0000E942823F981F53108F0EEC060E270E01B
:1070B00080E090E00E94F32129812F5F2983F2CFA5
:1070C000243631054CF48536910504F58A30910556
:1070D00034F48AE090E009C084369105BCF0883E23
:1070E000E3E09E0714F087EE93E02817390709F4D0
:1070F000E1CB9093200180931F011092CE05109256
:10710000CF051092D0051092D105D4CB84E690E043
:10711000F0CF662351F08EE28093D903605D6093D7
:10712000DA0380E28093DB03AACC80E28093DA0367
:107130008093D903F6CF498180E2443628F0842F2A
:1071400064E60E947EE8805D8093D903698190E2C5
:107150006A3040F02AE0862F622F0E947EE80E946B
:107160007EE8905D9093DA0389816AE00E947EE870
:10717000905D9093DB0369ED73E082E693E00E94FB
:107180004CEB16CD7F936F93DF92CF9283EC9BE015
:107190009F938F9382E593E09F938F930E9491E159
:1071A0000FB6F894DEBF0FBECDBF86E040CD87E0BE
:1071B0000E94498580FF13C00DE613E0F80161913C
:1071C0008F01662309F4F3CE6F320CF06FE3062EC5
:1071D000000C770B880B990B0E94F321EFCF809165
:1071E000940580FDE0CE81EE9BE00E942423DFCE5B
:1071F00087E00E944985869580FF13C008E613E06A
:10720000F80161918F01662309F4ECCE6F320CF026
:107210006FE3062E000C770B880B990B0E94F3216D
:10722000EFCF80919405869580FDD8CE81EE9BE0CE
:107230000E942423D7CE87E00E94498586958695B3
:1072400080FF17C082E793E09A838983E981FA81FE
:107250006191FA83E983662309F4DFCE6F320CF083
:107260006FE3062E000C770B880B990B0E94F3211D
:10727000EDCF809194058695869580FDCACE89EDE7
:107280009BE00E942423C9CE0F900F900F900F9087
:107290000F90DF91CF911F910F91FF90EF90DF90B2
:1072A000CF90BF90AF909F908F907F906F905F90A6
:1072B0004F9008950E94DE33882339F08091C616DE
:1072C00082FB882780F991E08927089581E008955D
:1072D0009091C00095FFFCCF8093C6000895CF9396
:1072E000DF93EC018991882319F00E946839FACF65
:1072F0008DE00E9468398AE0DF91CF910C94683963
:10730000CF93DF93EC01FE0184912196882319F03D
:107310000E946839F8CFDF91CF910895E0913E0C3B
:1073200081E6E89FF0011124E056F34F808181113E
:1073300007C081ED95E20E9480398AE00C9468399B
:1073400008950E94683989E394E00C948039AF92E3
:10735000BF92CF92DF92EF92FF920F931F93CF9342
:10736000DF9384E294E00E94803960916B04709115
:107370006C0480916D0490916E0445E00E948D70C4
:1073800081E194E00E948039C0E0D9E0D15021F041
:1073900080E20E946839FACF8C2F0E9492C7CF5F9B
:1073A000C53099F78AE00E94683907E014E0C0E030
:1073B00080E20E9468398C2F0E9492C75801D5E064
:1073C00080E20E946839F501C080D180E280F380BC
:1073D000A7019601C701B6010E94F2EA81112CC0F3
:1073E00020E030E0A901C701B6010E9474EA87FDE0
:1073F00003C08BE20E94683945E0C701B6010E94D4
:107400008D70D15084E1A80EB11CD111D9CF8AE082
:107410000E946839CF5F0C5F1F4FC53049F68AE084
:10742000DF91CF911F910F91FF90EF90DF90CF9060
:10743000BF90AF900C946839F12C80E20E946839BB
:10744000F3948DE3F8E0FF12F9CFDBCFCF92DF9218
:10745000EF92FF926A017B010E94803942E0C701EE
:10746000B601FF90EF90DF90CF900C948D70CF938A
:10747000DF93EB010E948039CE01DF91CF910C9414
:107480002EB78AE094E00C94803984E094E00C9468
:107490008039CF9384E50E945830C0E08823D9F02A
:1074A0000E943430C82F1816B4F40E94453A8DE477
:1074B0000E94683980914503909146030E9499C7C4
:1074C0006C2FCC0F770B8EE395E00E94373A8AE061
:1074D0000E946839CFEF8C2FCF910895EC018B017A
:1074E000F42E0E94DE710E94413A84EE93E00E94E5
:1074F00080390115110511F405E516E2209711F404
:10750000CBEDD3E00E9477201F930F93DF93CF93AF
:107510008BEC93E09F938F93D1E0DF930E945C1FED
:107520000E946B1DC0914B15C695C6958DB79EB731
:1075300007960FB6F8949EBF0FBE8DBF809183153E
:10754000811104C0D09383150E94C9C280914C154B
:1075500090914D150E94A2C2DC2FDD0F1D2F1C0F34
:1075600083E00E94DE1A4BE652E16C2F80E00E941D
:10757000272F10928115D09382158CEB93E00E94F7
:10758000242310928115109382158FEA93E00E94B4
:1075900024238AE495E10E940EC68111E1CF82ED99
:1075A00093E00E947EB589EE93E030E6019729F0E2
:1075B000232F2A950000E9F7F9CFF89489EE93E09C
:1075C00038EE019729F0232F2A950000E9F7F9CF2B
:1075D0000E94DE71FF2021F00E94CA33A895FECFE1
:1075E0005E9AFCCF8091540B9091550B2FEF3FEF9B
:1075F000981751F0E92FF0E0EC5AF44F228130E077
:107600009F5F9F779093550BC90108951F920F922A
:107610000FB60F9211240F900FBE0F901F90189568
:107620001F920F920FB60F9211240BB60F922F9349
:107630003F934F935F938F939F93EF93FF9380912B
:10764000C6004091550B9091540B31E0390F3F77B4
:10765000209121032C3008F072C0E22FF0E0ED5CA5
:10766000F44C0C94DFE83F3B663B753B803B873B2B
:107670009F3B8B3B9F3B8F3B933B9F3B973B80329A
:1076800029F0E8F48A3011F08D30F1F4431731F02D
:10769000E92FF0E0EC5AF44F8283932F9093540B30
:1076A000FF91EF919F918F915F914F913F912F911A
:1076B0000F900BBE0F900FBE0F901F9018958D343A
:1076C00081F021E08E3471F02BE00CC08A3338F465
:1076D0008033E0F68032D1F28D32B1F7D7CF8D34DE
:1076E00099F722E020932103D1CF813329F084330D
:1076F00029F0803249F7CACF23E0F4CF28E0F2CF57
:1077000024E0803379F326E0813361F3DDCF25E097
:107710008833D1F6E7CF27E08233B1F6E3CF29E013
:10772000813391F6DFCF2AE0803371F6DBCF8A30E8
:1077300019F08D3009F0AACF10922103A7CF8A301B
:1077400019F08D3009F0A2CF509184155523A1F383
:10775000273049F02A3059F0253071F71092520144
:1077600010929103E9CF21E020937104E5CF21E04D
:1077700020937004E1CF8EBD0DB407FEFDCF0895B8
:107780008FEF8EBD0DB407FEFDCF8EB5089590919D
:1077900064009B7F90936400982F906A96959CBD9F
:1077A00080FD03C091E0863009F490E09DBD08950E
:1077B000CF92DF92EF92FF92CF936B017C01C42FA7
:1077C0004A3069F4F7FE0BC0F094E094D094C09472
:1077D000C11CD11CE11CF11C8DE20E9468394C2FA8
:1077E000C701B601CF91FF90EF90DF90CF900C943E
:1077F0002BC7CF92DF92EF92FF926A017B010E942A
:1078000080394AE0C701B601FF90EF90DF90CF903A
:107810000C94D83B2F923F924F925F926F927F923F
:107820008F929F92AF92BF92CF92DF92EF92FF9290
:107830000F931F93CF93DF93CDB7DEB7EB970FB6C0
:10784000F894DEBF0FBECDBF85E40E945830882378
:1078500021F00E94741C811183C283E50E9458307C
:10786000882309F45EC00E94741C9A83898383E490
:107870000E945830A5E07A2E882319F00E94741CCB
:10788000782E60E085E50E9473308FAB60E088E47D
:107890009BE00E94751F49815A81BA01550F880BE0
:1078A000990B0E9401E2162F7D838E83292E0E9460
:1078B00080C16B877C878D879E8760915001709116
:1078C00051016F507109072E000C880B990B0E9413
:1078D00001E29B01AC01612F7D818E81922D0E947E
:1078E00074EA18161CF589EF9AE00E948039EB962D
:1078F0000FB6F894DEBF0FBECDBFDF91CF911F91C1
:107900000F91FF90EF90DF90CF90BF90AF909F903E
:107910008F907F906F905F904F903F902F900C943E
:10792000B5BA24EB30E03A832983A1CF8B859C85BF
:10793000AD85BE85805B9C43AF4FBF4F8BAB9CAB8F
:10794000ADABBEAB85EE9AE00E9480390E94DE713D
:107950008FE78093A91481E0809352018B849C84EB
:10796000AD84BE848AA69BA6ACA6BDA61C8E1D8E29
:107970001E8E1F8E18A219A21AA21BA219821A8289
:107980001B821C822FE730E040E050E02F87388BCD
:10799000498B5A8B1F8230E43D8B4CE14E8B56E471
:1079A0005F8B188E198E1A8E1B8EFFE7CF2ED12C6F
:1079B000E12CF12C1EA61FA618AA19AA1AAA1DA20C
:1079C0001EA21FA218A68CA31C8A1B8A312C00E0C1
:1079D0001AAE1BAEA72D770CBB0BB9AFA8AF809129
:1079E0005201882309F48BC00E9480C12B013C0105
:1079F000B0917204B9A7BB2309F46BC00E949172C5
:107A00006091A5147091A614072E000C880B990B99
:107A10000E9401E2362E072F8AAF9BAF288D398D49
:107A20004A8D5B8D0E9474EA181634F4388E098FE3
:107A30002AAD2A8F3BAD3B8F2F813D894E895F89CF
:107A4000632D702F8AAD9BAD0E94FAE187FF06C0BF
:107A50003F820D8B4AAD4E8B5BAD5F8B8CA1232D8E
:107A6000302F4AAD5BAD612F7D81882309F494C12D
:107A70008E81922D0E94FAE187FF2BC0B301A201F3
:107A8000481959096A097B09DB01CA0188589341E1
:107A9000A109B109B7FD1DC08F859889A989BA8947
:107AA0008C199D09AE09BF09B595A795979587953E
:107AB0008093A9144DA35EA36FA378A7188F9D810F
:107AC000998FAE81AA8F2B8E4B865C866D867E86C3
:107AD0001CA220E030E040EF51E4612F7D818E81D7
:107AE000922D0E94F1E8232D302F4AAD5BAD0E940C
:107AF000FAE187FF22C082E79AE00E948039109263
:107B000052010E94DE71F3CE4BEEC42ED12CE12C3B
:107B1000F12C95C184E190E0A0E0B0E08F87988BD4
:107B2000A98BBA8B34E1C32ED12CE12CF12C95C159
:107B3000CF86D88AE98AFA8A90C1D301C2012AA5E0
:107B40003BA54CA55DA5821B930BA40BB50BB7FD04
:107B50004CC080E00E9431718AE00E946839D301F4
:107B6000C2018053984FAF4FBF4F8AA79BA7ACA7C6
:107B7000BDA79EA5911167C02FA538A949A95AA9EB
:107B8000632D702F8AAD9BAD0E9474EA18160CF01D
:107B900046C020E030E040E050E4632D702F8AAD15
:107BA0009BAD0E94F1E86FA778AB89AB9AABA301BC
:107BB0009201205B3C434F4F5F4F2BAB3CAB4DAB37
:107BC0005EAB20E030E040EC50E4612F7D818E819F
:107BD000922D0E94F0E8232D302F4AAD5BAD0E941C
:107BE000FAE1881F8827881F8EA78B859C85AD8525
:107BF000BE8588169906AA06BB0610F4D501C401F5
:107C0000481A590A6A0A7B0A31E843163FE45306C8
:107C100032E16306710480F184E59AE06ECFD3010E
:107C2000C2012BA93CA94DA95EA9821B930BA40BF1
:107C3000B50B41EB51E260EC71E2B7FDD6CF80E0CD
:107C40000E94A972D2CF20E030E040EF51E4612FD2
:107C50007D818E81922D0E94F0E89B01AC01632D05
:107C6000702F8AAD9BAD0E94FAE187FFBECF4DE534
:107C700052E26DE672E2E3CF48AD59AD8B899C8943
:107C8000481759070CF069C003970CF466C087EFDA
:107C900099E00E9480398AED99E00E9480394981FB
:107CA0005A816B817C8183EF99E00E94263A8AE0B9
:107CB0000E9468398AED99E00E94803948A159A153
:107CC0006AA17BA18FEE99E00E94263A8AE00E9489
:107CD00068398AED99E00E9480394C8D5D8D6E8DFA
:107CE0007F8D8BEE99E00E94263A8AE00E946839E7
:107CF0009FA9992309F4FBCD29813A814B815C81AD
:107D00002093AA143093AB144093AC145093AD1449
:107D10002CEA35EC47E25EE368A179A18AA19BA138
:107D20000E9460E26093AE147093AF148093B0141D
:107D30009093B1142CEA35EC47E25EE36C8D7D8DB7
:107D40008E8D9F8D0E9474E96093B2147093B3146A
:107D50008093B4149093B514CACD0E94E7303FCEFF
:107D600084E29BE0EB960FB6F894DEBF0FBECDBF6A
:107D7000DF91CF911F910F91FF90EF90DF90CF9007
:107D8000BF90AF909F908F907F906F905F904F903B
:107D90003F902F900C9480398E81922D0E9474EA2E
:107DA00018160CF096CED301C2012B853C854D856B
:107DB0005E85821B930BA40BB50BAC01BD0148582B
:107DC00053416109710977FD84CE4B895C89452B4C
:107DD00009F4FEC08DA09EA0AFA0B8A4880E991E85
:107DE000AA1EBB1E2DA13EA14FA158A5281B390BD1
:107DF0004A0B5B0BC701B6010E9432E8A501940152
:107E00000E94C0E8CF84D888E988FA88C20ED31EC1
:107E1000E41EF51E54E1C516D104E104F1040CF48E
:107E200079CE8CEEC816D104E104F1040CF06CCECE
:107E300090E8C916D104E104F1040CF479CECF86A0
:107E4000D88AE98AFA8A2EEF30E040E050E02C1917
:107E50003D094E095F0969017A014F855889698991
:107E60007A898DED9AE00E94F93BB701A60188ED71
:107E70009AE00E94F93B4F815D896E897F8981ED8F
:107E80009AE00E94263A488D598D6A8D7B8D8AEC46
:107E90009AE00E94263AAB89BC8913970CF498C0EB
:107EA000C701B6010E9401E220E030E040E850E462
:107EB0000E9460E269837A838B839C832F813D8952
:107EC0004E895F89688D798D8A8D9B8D0E94F0E83F
:107ED0002BED3FE049E450E40E9460E220E030E016
:107EE00040E05FE30E9460E29B01AC0169817A811E
:107EF0008B819C810E9474E96F83788789879A8738
:107F0000C501B4010E9401E22FE632E143E85AE3E1
:107F10000E9460E24B015C012AE939E949E15FE333
:107F20006F81788589859A850E9460E269837A836A
:107F30008B839C839B01AC010E94F1E8A501940115
:107F40000E9474E968A379A38AA39BA329813A813B
:107F50004B815C81C501B4010E9460E220E030E009
:107F600040E05EE30E9460E26C8F7D8F8E8F9F8F7A
:107F70004F81588569857A8584EC9AE00E94263A7B
:107F8000B501A4018EEB9AE00E94263A8AE00E9495
:107F900068398FEA9AE00E94803949815A816B8161
:107FA0007C8189EA9AE00E94263A48A159A16AA1F7
:107FB0007BA183EA9AE00E94263A4C8D5D8D6E8DFE
:107FC0007F8D8DE99AE00E94263A8AE00E94683906
:107FD0008F859889A989BA898C0D9D1DAE1DBF1DFD
:107FE000B595A795979587958093A9142B893C897A
:107FF0002F5F3F4F3C8B2B8B1F833D813D8B4E81F1
:108000004E8B2F8A5301420159A55CA362CDCF93B9
:10801000DF93EB010E948039CE01DF91CF910C9468
:10802000B5CB4F925F926F927F928F929F92AF9259
:10803000BF92CF92DF92EF92FF920F931F93CF9355
:10804000DF9300D01F92CDB7DEB780913D0C803119
:1080500008F0C7C131E6E32E80913D0C803108F075
:10806000F8C08091540B9091550B891B8F7709F4C0
:10807000F0C00E94F23A97FF0BC00E94413A89E794
:1080800093E00E9480398091540B8093550BE4CF8C
:108090008A3019F08D3009F0D3C010923C0C8091D9
:1080A000DA0B9091DB0BFC01EA52F44F1682892B1C
:1080B00019F40E945386D0CF1092DB0B1092DA0B8A
:1080C0000CED1BE0F8018191803209F446C08E343A
:1080D00009F0A1C064E773E0C8010E9477E16C0178
:1080E000892B41F06EE470E0C80104960E9441EBD8
:1080F000009709F4C8014AE050E070E060E00196A2
:108100000E94EEDE4B015C018091D60B9091D70B63
:10811000A091D80BB091D90B0196A11DB11D881665
:108120009906AA06BB0629F060E081E493E0CD2819
:1081300051F16AE270E0C8010E9470EB9C01009767
:1081400029F1982F901BF12C992349F09150F801B7
:10815000E90FF11D8081F826F7CF8F01B3CF4AE0F8
:1081600050E070E060E0C90101960E94EEDE4F2C05
:10817000512C712C612C641575058605970551F0FD
:1081800060E082E293E00E94AEB866CF60E088EFE4
:1081900092E0F9CF8092D60B9092D70BA092D80B99
:1081A000B092D90B8091A4058130E1F067E470E0D2
:1081B000C8010E9441EB0097A9F04AE050E070E04E
:1081C00060E001960E94EEDE623071058105910546
:1081D00048F487E592E00E94803960E08DE492E007
:1081E0000E94751F8091DC0B8B3309F435CF809191
:1081F0003D0C803108F030CF80913F0C8E9DC00146
:1082000011246CED7BE0805C934F0E944CEB80E08E
:108210000E947AB821CF8091C61680FFC3CF6EEF3F
:1082200075E2C8010E9477E1009731F0FC0183817B
:1082300080538A3008F0B6CF60E08EEC92E0A3CF96
:108240002AED3BE04CED5BE06CE37CE00E94DC1649
:1082500003CF8091C61682FFC4C01A82198281E6BC
:10826000F82E90E1B92E29E6A22E80913D0C8031A6
:1082700008F0B7C00E9414178111B3C041E050E06C
:10828000BE016D5F7F4F88EB94E10E9438CD0B817A
:1082900010E0019711F00FEF1FEF8091C014909143
:1082A000C114A091C214B091C3148093C2169093CC
:1082B000C316A093C416B093C5160E9414170F3F9F
:1082C000100749F4811107C00E94413A81E993E007
:1082D0000E948039CACF40913F0C242F30E00A30F1
:1082E00061F00D3051F0882309F46DC089819A81C5
:1082F000009719F001969A83898310922E03898141
:108300009A81F29EF001F39EF00D1124E35CF34F8D
:10831000DF01A80FB91F13961C92892BB9F50E9493
:1083200053860E941417882309F49FCF0E949C77DC
:1083300088EB94E10E94476C8091BD168823F1F18F
:1083400081508093BD168A9DC001112462E0835E36
:108350009A4F0E946FCFE091BD1624E0E29FF0019A
:108360001124E75EFA4F408151816281738140930D
:10837000C2165093C3166093C4167093C51688EB4B
:1083800094E10E9410CC0E94AEC76FCF1A8219826E
:1083900083818D3479F48481823361F485818533DE
:1083A00049F4868180538A3028F08091C6168B7FED
:1083B0008093C61681E00E947AB8B3CF0E949FC70F
:1083C000B092A40552CF4F9DA0011124405C534FA1
:1083D0009E012F5F3F4F6EE273E0802F0E94DC16FC
:1083E00044CF0E9480C14B015C0180913C0390917D
:1083F0003D03A0913E03B0913F030097A105B10555
:1084000051F14091E8055091E9056091EA057091BC
:10841000EB05840F951FA61FB71FA5019401281B0C
:10842000390B4A0B5B0BDA01C901B7FD14C00E947E
:10843000413A6091F1057091F20580E192E00E946D
:1084400007408AE00E94683940E070E060E090E018
:1084500080E00E946E3A80910B0190910C01A091F6
:108460000D01B0910E01892B8A2B8B2B79F0909105
:108470001E1580911F15981709F4FCC08092E8051D
:108480009092E905A092EA05B092EB050E9480C1A6
:108490006B017C0180919103811108C020911E1510
:1084A00090911F1581E0291301C080E02091A5144F
:1084B0003091A61491E089272A3A31050CF480E026
:1084C00091E040912A0350912B0360912C0370910D
:1084D0002D03452B462B472B09F490E0981789F084
:1084E000882309F401C1D701C60180569444A24FE4
:1084F000BF4F80932A0390932B03A0932C03B09338
:108500002D034090500B5090510B6090520B709087
:10851000530B20912603309127034091280350915B
:108520002903C301B2010E94FAE1882319F1809165
:108530002A0390912B03A0912C03B0912D0340921C
:108540002603509227036092280370922903892BF7
:108550008A2B8B2B09F449C0D701C601805694445D
:10856000A24FBF4F80932A0390932B03A0932C0319
:10857000B0932D0380912A0390912B03A0912C039B
:10858000B0912D030097A105B10579F1C81AD90A58
:10859000EA0AFB0AF7FC29C010922A0310922B0367
:1085A00010922C0310922D038BEF91E00E948039E2
:1085B00060E087EE91E00E94751F8091A714909172
:1085C000A8141816190624F490E080E00E9448A030
:1085D0008091AB059091AC051816190634F41092F1
:1085E000AC051092AB050E94686280912F039091B8
:1085F0003003A0913103B0913203A5019401281BEF
:10860000390B4A0B5B0BDA01C901B7FD8FC09091A2
:108610001E1580911F15F0903706981749F0E091CC
:108620001F153BE4E39FF0011124EF56F94FF08052
:108630000E9480C1FF2009F4D1C000912203109153
:1086400023032091240330912503011511052105F1
:10865000310509F04DC06C597F4F8F4F9F4F60938C
:108660002203709323038093240390932503FF2414
:10867000FA9444C00E9480C10091E8051091E90578
:108680002091EA053091EB05C0900B01D0900C01D0
:10869000E0900D01F0900E010C0D1D1D2E1D3F1DD3
:1086A000601B710B820B930B97FF03C01092330377
:1086B000EDCE809133038111E9CE81E080933303C5
:1086C0005E9A809194058E7F809394055E9A809146
:1086D00094058D7F80939405159A809194058B7FE6
:1086E000809394055E9AD2CE80E090E0DC0101CFC9
:1086F000601B710B820B930B97FDB9CF0F2D10E010
:1087000084E00E9438B8F11072C060E084E00E94FA
:1087100089C044E6840E911CA11CB11C80922F03D9
:1087200090923003A0923103B09232030E9453869C
:108730008091A4058823F1F1109108011130B1F165
:108740008091C61680628093C61681E080930801EE
:1087500064EF71E080E090E00E94A6330E94D0D1E7
:108760008091C61683FFA5C0123028F460E080EA2D
:1087700093E00E94751F01E083E0809353010E9403
:1087800080C16C597F4F8F4F9F4F609385037093CB
:1087900086038093870390938803002339F0123077
:1087A00029F481E08093BC160E942BD20E943C9455
:1087B0000E94E7300F900F900F90DF91CF911F91A3
:1087C0000F91FF90EF90DF90CF90BF90AF909F9070
:1087D0008F907F906F905F904F900895109222033A
:1087E00010922303109224031092250387CF0F3F8A
:1087F000110511F461E08ACFE9E3F6E2E491E1507A
:10880000EA3008F051C0F0E0E85FFB4B0C94DFE881
:10881000124417441C4426445444544430443844BD
:1088200040444A4484B5806884BDF7BC72CF84B5A7
:10883000806284BDF8BC6DCF809180008068809399
:108840008000109389000093880063CF809180009E
:1088500080628093800010938B0000938A0059CF30
:108860008091B00080688093B000F092B30051CF47
:108870008091B00080628093B000F092B40049CF44
:1088800080919000806880939000109399000093ED
:1088900098003FCF80919000806280939000109369
:1088A0009B0000939A0035CF003811050CF0A2CF41
:1088B0002CCF00E0112309F479CF5ECF2F923F92A5
:1088C0004F925F926F927F928F929F92AF92BF92E0
:1088D000CF92DF92EF92FF920F931F93CF93DF938C
:1088E000CDB7DEB764970FB6F894DEBF0FBECDBF2D
:1088F0008091FB0A83FDB0C10E94493A898787FDB8
:10890000ABC189E40E945830882309F497C10E94C2
:10891000343090E01816190614F481E090E026E057
:10892000289FF001299FF00D1124E255FA4F808114
:1089300091811B8A0E9448A02091A7143091A8140D
:108940008091A5149091A614821793078CF48AEC59
:1089500099E09F938F9385ED99E09F938F931F925A
:108960000E945C1F0F900F900F900F900F9005C00A
:108970002B898FEB99E0222361F381E080935201F0
:108980001C821D821E821F821A861B861C861D86E3
:108990001F862CE3288B3CE1398B46E44A8B212C43
:1089A000312C50E85A838FEB8B83198291E09E879C
:1089B000812C912C540101C01E860091A7141091A6
:1089C000A814B801012E000C880B990B0E9401E23B
:1089D000D62EE72EF82E988791014A815B810E945E
:1089E000FAE1882391F08091A5149091A6143B8917
:1089F0003111E7C041E04983081719070CF01982CB
:108A00002D2C3E2CFA8258855B830E9480C16B011D
:108A10007C01DC01CB012A853B854C855D85821B71
:108A2000930BA40BB50BB7FD2FC0D701C60188511E
:108A30009C4FAF4FBF4F8A879B87AC87BD87898587
:108A40000E9431718BEB99E00E948039811491046E
:108A5000A104B10409F4E0C0C501B4016053784F2A
:108A60008F4F9F4F6C197D098E099F0928EE33E0C7
:108A700040E050E00E9442E8CA01B9014AE00E9489
:108A8000D83B8AE00E9468390E9411400E9480C150
:108A90006093E8057093E9058093EA059093EB05F0
:108AA0006091A5147091A614072E000C880B990BE9
:108AB0000E9401E26887072F182F9C8B262F372FE3
:108AC000482F592FB1018A819B810E94F0E82B0128
:108AD0003C0120E030E0A9010E9474EA87FF04C055
:108AE00077FA709477F8709481149104A104B1041A
:108AF00009F096C020E030E040E85FE3C301B20136
:108B00000E94FAE187FF10C09E85812C912C5401B0
:108B1000992331F08AE9882E82E0982EA12CB12C7D
:108B20008C0C9D1CAE1CBF1CA981AA2399F12C8121
:108B30003D814E815F81211531054105510541F08F
:108B4000D701C601821B930BA40BB50BB7FD22C046
:108B50002885302F412F5C896F85788989899A898A
:108B60000E94F0E820E030E040EC5FE30E94FAE190
:108B700087FD2AC0D701C601805A9541AF4FBF4F2C
:108B80008C839D83AE83BF8398859F87088B198BC9
:108B9000AC89AA8B809152018823B1F08114910491
:108BA000A104B10409F408CFB0EDCB1AB7E0DB0A99
:108BB000E108F108C818D908EA08FB08F7FCFCCE60
:108BC00003C0081719070CF580915201882309F496
:108BD00043C01092520164960FB6F894DEBF0FBEE8
:108BE000CDBFDF91CF911F910F91FF90EF90DF905C
:108BF000CF90BF90AF909F908F907F906F905F903D
:108C00004F903F902F900C94B5BA2D2C3E2CFA82A9
:108C100088858B831982F9CE8FE30E94683931CF22
:108C200020E030E040E450E4C301B2010E9474EA65
:108C300018160CF079CF4601570176CF83E50E94D4
:108C400058308B8B811105C082E50E9458308823F3
:108C500019F00E94741C6ECE64960FB6F894DEBFB5
:108C60000FBECDBFDF91CF911F910F91FF90EF907D
:108C7000DF90CF90BF90AF909F908F907F906F903C
:108C80005F904F903F902F9008952F923F924F9278
:108C90005F926F927F928F929F92AF92BF92CF928C
:108CA000DF92EF92FF920F931F93CF93DF93CDB795
:108CB000DEB7CB54D1090FB6F894DEBF0FBECDBFDF
:108CC0002C968FAF2C97809147038D3409F481C483
:108CD000843511F40C94C85B873491F4809145037A
:108CE000909146038C31910509F434C208F06AC0B2
:108CF0008430910509F4AEC130F4029708F4F7C04E
:108D00000E94DBBA77C18531910509F473C14B9795
:108D1000B9F70E94E9BA81116DC18CE0EEE5F1E08E
:108D2000DE01119601900D928A95E1F770E060E006
:108D300080E50E94653040E050E068E472E44CA3B6
:108D40005DA36EA37FA340E050E060EA70E448A317
:108D500059A36AA37BA3813009F4B5C1823009F419
:108D6000D1C120E030E040E050E460914C0B7091C4
:108D70004D0B80914E0B90914F0B0E94F1E87B01BF
:108D80008C0120E030E046E953E40E9474EA1816B2
:108D900024F4E12CF12C06E913E4A984BA84CB84F1
:108DA000DC849701A801B501C6010E9474EA181677
:108DB00014F475018601C701D8018C8F9D8FAE8F89
:108DC000BF8FC2C18A35910509F4E6C360F58D31C4
:108DD000910509F43DC38A9709F092CF8091A405CB
:108DE000813009F007C189E40E945830082F10E053
:108DF000882319F00E94741C182F8AE40E945830AE
:108E0000F82E882311F40C942A5C0E94741C002311
:108E100009F421C3153010F40C941C5C8AE595E02C
:108E20000E948039E7C08B35910509F4B8C38C35B1
:108E3000910509F065CF9AE6C92E91E0D92EF12C63
:108E4000E12C00E010E0D6018D916D010E945830B8
:108E5000382E8823E1F10E94781C4B015C0113300D
:108E600059F0F701EF5FF94F208131814281538141
:108E70000E94F0E84B015C01F701EC5BF44F2081AC
:108E8000318142815381C501B4010E94F0E82B0178
:108E90003C012DEB37E346E855EB0E9474EA87FD71
:108EA0000AC02DEB37E346E855E3C301B2010E9447
:108EB000FAE1181664F4133009F075C38092500B70
:108EC0009092510BA092520BB092530B032D1F5F47
:108ED000B4E0EB0EF11C143009F0B5CF002321F003
:108EE00080E59BE00E9481830E94128E83C0809166
:108EF000A405813009F07EC06DEEC62E63E0D62E4B
:108F000074E4E72E7BE0F72EE1E0AE2EE6E0BE2E25
:108F100010E088E5810F0E945830882309F47EC054
:108F20000E94781C2B013C01812F0E94301788235E
:108F300009F46AC0D7012D913D914D915C91C30117
:108F4000B2010E94F1E8D6016D937D938D939C93BD
:108F500013971F5FF4E0CF0ED11C24E0E20EF11C4A
:108F600034E0A30EB11C1330A1F685E40E94583002
:108F7000882309F45EC00E94781C6B017C0183E0A9
:108F80000E943017882371F02091500B3091510BC3
:108F90004091520B5091530BC701B6010E94F1E86A
:108FA0006B017C01C092F903D092FA03E092FB03BB
:108FB000F092FC0386E40E9458308823C9F00E9496
:108FC000781C20E030E0A9010E9474EA181684F4AD
:108FD0000E94781C20E030E040E752E40E9474E9EF
:108FE00060932101709322018093230190932401C7
:108FF0000E945C892C96FFAD2C97F1110C9479514D
:109000000E948E390C947951F50120813181428181
:109010005381C301B2010E94F0E895CFF70180812E
:109020009181A281B381F60180839183A283B3836E
:1090300090CF8091500B9091510BA091520BB09119
:10904000530B8093F9039093FA03A093FB03B0931F
:10905000FC03B0CF80E50E945830C12CD12C7601A2
:10906000882321F00E94541C6B017C0183E50E943F
:109070005830882361F00E94781C20E030E04AE7F5
:1090800054E40E9460E20E94EDE96B017C010E94C1
:109090009C7780916B12811105C060E081E595E0BD
:1090A0000E94751F0E9480C1C60ED71EE81EF91EC1
:1090B0000E9480C16C197D098E099F0997FF9ACF84
:1090C0000E941140F5CFBE01605E7F4FCE01099630
:1090D0000E943286E0904C0BF0904D0B00914E0BAD
:1090E00010914F0B2D813E814F81588569817A8186
:1090F0008B819C81DE0194966D010E947A850E948D
:10910000128E78CF29853A854B855C8560914C0B12
:1091100070914D0B80914E0B90914F0B0E94F1E896
:109120006B017C0120E030E046E953E40E94FAE163
:1091300087FD06C0C12CD12C56E9E52E53E4F52E4F
:10914000CC8EDD8EEE8EFF8EBE01605E7F4FCE0137
:109150004C96BECF87E00E944985882309F464C1FC
:109160000E949C7710922801609101048CE40E9477
:109170007330982E80E00E9498300E9480C16093E6
:10918000E8057093E9058093EA059093EB058091DB
:10919000210190912201A0912301B091240180939B
:1091A000380390933903A0933A03B0933B03809123
:1091B0001F0190912001909337038093360384E63A
:1091C00090E09093200180931F0181E080939205AD
:1091D0000E940F8F8AE50E94231CA82E88E50E941A
:1091E000231C182F89E50E94231CB82E181308C0D1
:1091F000B12EA11205C011E0BB24B394AA24A394FC
:1092000082E50E945830882309F416C10E94781C18
:109210003B01882EC92E20E030E0A9010E94FAE12E
:10922000882309F444C0111103C0BB2009F4D0C045
:10923000D0904C0BE0904D0BF0904E0B00914F0BEB
:109240009301482D5C2D6D2D7E2D8F2D902F0E942A
:1092500074EA181624F0D62CE72CF82C0C2D80E09C
:1092600090E0A0E8B0E48C8F9D8FAE8FBF8F20E0A0
:1092700030E046E953E46D2D7E2D8F2D902F0E9416
:10928000FAE187FD05C0D12CE12C26E9F22E03E49A
:109290008D2D9E2DAF2DB02F89839A83AB83BC83F8
:1092A000BE01645E7F4FCE0101960E94328611237B
:1092B00009F489C0BB2009F483C01092440B1092BA
:1092C000450B1092460B1092470B1092480B1092D0
:1092D000490B10924A0B10924B0B0E945186E6E903
:1092E000F6E1C590D590E590F490EAE9F6E1459075
:1092F000559065907490A7019601C301B2010E9438
:10930000FAE187FFA0C0A7019601C301B2010E9444
:1093100074E99B01AC010E9460E220E030E040E88B
:109320005FE30E94F1E80E94B2EA20E030E048E406
:1093300052E40E9460E269837A838B839C8320914C
:109340004C0B30914D0B40914E0B50914F0B28A779
:1093500039A74AA75BA720E030E040EC5FE3C301F8
:10936000B2010E9460E22B013C0177FA709477F819
:10937000709420E030E040EC5FE3C701B6010E944A
:1093800060E29058AE014F5F5F4F6A01E8A4F9A414
:109390000AA51BA5A30192010E947A850E942A902A
:1093A0001092440B1092450B1092460B1092470BF3
:1093B0001092480B1092490B10924A0B10924B0BD3
:1093C00080E00E94C18CBB2019F081E00E94C18C1A
:1093D000AA2019F082E00E94C18C0E9451868091DF
:1093E000910580939205892D0E94983080913803D1
:1093F00090913903A0913A03B0913B0380932101EE
:1094000090932201A0932301B0932401809136030D
:10941000909137039093200180931F0183E0809304
:1094200053010E94128EE6CD60E08FE40E947330FB
:10943000882309F495CEDECD612C712C30E8832E83
:1094400040E4C42EF0CEA3019201C701B6015FCF64
:109450000E94AB5CCFCD853008F0E0CC90E1E4E435
:10946000FBE0ADEEB3E001900D929A95E1F7002399
:10947000A1F054E01502F0011124E756FA4E4081A4
:109480005181628173814093ED035093EE036093A9
:10949000EF037093F003FF2091F094E08902F00154
:1094A0001124EB57FA4E80819181A281B381809380
:1094B000F1039093F203A093F303B093F40386E4D3
:1094C0000E945830811151C0C12CD12C760180905E
:1094D000210190902201A0902301B090240120E06E
:1094E00030E0A901C701B6010E94FAE1882341F0EA
:1094F000C0922101D0922201E0922301F092240136
:1095000000911F011091200184E690E090932001CA
:1095100080931F01C0905801D0905901E0905A01EA
:10952000F0905B0180E090E0A0E8BFE380935801F9
:1095300090935901A0935A01B0935B010E945C89FA
:109540008092210190922201A0922301B0922401E5
:109550001093200100931F01C0925801D09259012D
:10956000E0925A01F0925B0145CD0E94781C6B019C
:109570007C0120E030E0A9010E9474EA18160CF08A
:10958000A3CF20E030E040E752E4C701B6010E94DB
:1095900074E96B017C019BCF109240032BCD8FE0CF
:1095A0008093400327CDF701EF51FC4F5F01A301EA
:1095B000920160817181828193810E94F1E8D501DD
:1095C0006D937D938D939C931397812F0E94298592
:1095D0007ECC80914503909146038237910511F42A
:1095E0000C94F95408F080C18934910509F445C6FA
:1095F00008F0D9C08831910509F498C408F06CC00E
:109600008231910511F40C94085400F582309105D3
:1096100008F411C4419709F073CB8BE092E00E94EB
:10962000FF1B882309F45BC488E50E94231C811179
:109630005E9889E50E94231C81115E988AE50E944C
:10964000231C882309F4D6CC1598D4CC85319105F8
:1096500009F456C458F5449709F052CB8091C616C8
:1096600083FF47C48EE995E00E9480398091C61639
:1096700083FF17C08EEE94E10E949F6D8BE1EEEEAA
:10968000F4E1DE01119601900D928A95E1F770E008
:1096900060E0CE0101960E9499D0CE0101960E9411
:1096A000A46D8FE895E00E948039A4CC86319105A5
:1096B00009F429C4479709F023CB80914103909185
:1096C0004203FC012191222309F42AC42032D1F75C
:1096D000DF0111971C92F6CF8C31910509F4A5C4D6
:1096E00020F58A31910509F44FC408F42EC483E4AF
:1096F0000E94231C882309F467C489EC95E00E942A
:1097000080398091BB14882309F459C4BE016F5F6E
:109710007F4F88EB94E10E946A6CCE0101960E9413
:10972000B5CB8AE00E94683965CC8E31910509F489
:109730008BC408F482C48F31910509F4F4C4809776
:1097400009F0DECA8091C61682FD0E949C77809146
:10975000C61683FF4FCC60E080E50E947330182F5F
:10976000682F80914103909142030E946FCF83E55F
:109770000E945830882381F00E94641CAB01BC0118
:109780004093C2165093C3166093C4167093C516C7
:1097900088EB94E10E9410CC0E94AEC711112ACC34
:1097A0000E94859027CC8C35910511F40C945C5463
:1097B00008F049C08135910511F40C94E35378F415
:1097C0008C34910509F469C58D34910509F47AC585
:1097D0008B34910509F094CA0E9485900BCC833597
:1097E000910511F40C94005410F40C94F853843542
:1097F000910511F40C9408548535910509F080CA3F
:1098000083E50E94231C882309F4F4CB0E9480C1C5
:109810006093E8057093E9058093EA059093EB0562
:109820000E94781C20E030E04AE754E40E9460E2A5
:109830000E94EDE960933C0370933D0380933E03E7
:1098400090933F03D7CB8C36910509F4D3CBE8F541
:109850008936910509F43EC540F58836910509F031
:109860004FCA8091FB0A83FDC5CB0E94493A87FD10
:10987000C1CB89E40E945830882311F40C94E95B31
:109880000E94343090E01816190614F481E090E03C
:1098900026E0289FF001299FF00D1124E255FA4F90
:1098A000808191810E9448A0A5CB8A36910509F458
:1098B0003AC58B36910509F023CA80E50E943EBB6C
:1098C000811198CB1092370695CB8E36910509F40D
:1098D0005EC508F4FBC48F36910509F46BC580376B
:1098E000910509F487CB0CCA8232E1E09E0711F49E
:1098F0000C94C05708F0AAC18E3B910509F4C7C566
:1099000008F094C08737910511F40C944E5588F4F3
:109910008537910511F40C94015510F00C941355F2
:109920008337910509F0ECC987EB96E00E948039F6
:1099300061CB8937910511F40C945B5510F40C94AC
:1099400052558C38910509F476C58139910509F095
:10995000D7C983E50E945830882311F40C946355CD
:109960000E94741C823010F00C9467558C011127F2
:1099700088E40E9458308823D1F00E94741C8A3AEF
:10998000910514F40C946F550E94741C843B914013
:1099900014F00C9473550E94741C26E0209FF00173
:1099A000219FF00D1124E255FA4F9183808382E4C8
:1099B0000E9458308823C9F00E94741C059714F443
:1099C0000C9477550E94741C8D38910514F00C94FA
:1099D0007B550E94741C26E0209FF001219FF00D12
:1099E0001124E255FA4F9383828386E40E94583013
:1099F000882309F4FFCA0E94741C97FF02C00C94CC
:109A00007F550E94741C8F3F910519F014F00C943F
:109A100083550E94741C26E0209FF001219FF00DC9
:109A20001124E255FA4F95838483E4CA8D3C910555
:109A300011F40C941F5608F070C0893C910511F484
:109A40000C948A5590F5883C910509F059C90E94FB
:109A5000493A182F87FDCECA0091060484E40E947B
:109A60005830F82E8823C1F00E94781C4B015C010D
:109A700020E030E0A9010E94FAE1882311F40C945F
:109A8000875524E01202F0011124EE5FFB4F808223
:109A90009182A282B3820F2D602F83E50E947330E2
:109AA000809306040E94355FA5CA8B3C910511F492
:109AB0000C94B4558C3C910509F022C983E092E0E6
:109AC0000E94FF1B81110C94D7554091300B50918F
:109AD000310B6091320B7091330B8FED97E00E9448
:109AE000263A4091340B5091350B6091360B7091B2
:109AF000370B8CED97E00E94263A4091380B50913D
:109B0000390B60913A0B70913B0B82E198E10E9416
:109B1000263A8AE00E9468396DCA833D910511F4A6
:109B20000C94A05608F04DC045E9E42E45E0F42E13
:109B300010E08E3C910509F0E3C888E5810F0E9492
:109B4000231C882351F00E94781CF70160837183E5
:109B500082839383812F0E9429851F5FF4E0EF0E9B
:109B6000F11C133051F780E192E00E94FF1B81113C
:109B7000BBC94091950550919605609197057091EC
:109B8000980581E298E00E94263A4091990550910B
:109B90009A0560919B0570919C0583E197E20E9474
:109BA000263A40919D0550919E0560919F057091C8
:109BB000A00580E197E20E94263A8AE00E94683977
:109BC00019CA8C3D910511F40C9468578D3D91058F
:109BD00009F096C80E94493A082F87FD0BCA83E511
:109BE0000E945830002E000C110B7801EE0CFF1C67
:109BF000882311F40C94A6570E94741CF701EB5DA6
:109C0000FE4F91838083000F111F000F111F9801D9
:109C1000285A3E4F7901BC01990F880B990B0E947D
:109C200001E22AE037ED43E25CE30E9460E2035088
:109C30001C4FD8012D913D914D915C910E9460E2A5
:109C4000F7016083718382839383D4C98C3A21E0C6
:109C5000920711F40C94DC5A08F083C08F3241E073
:109C6000940711F40C94E15810F58D32A1E09A0795
:109C700011F40C941A5810F00C949B588C329140AB
:109C800009F03EC864E071E083E50E9465308C0114
:109C900068EE73E080E50E9465308938F3E19F0744
:109CA00010F088E893E1B8010E949894A3C98A391A
:109CB000F1E09F0709F49EC938F48039914009F01A
:109CC0001FC80E949C7796C9843A41E0940711F41A
:109CD0000C94E558853A914011F00C94804688E543
:109CE0000E94231CC82E89E40E94231CA82E8823CE
:109CF00011F40C94435A0E94741C082F89E50E94A9
:109D0000231CF82E8AE40E94231CE82E882311F4D9
:109D10000C946E5A0E94741C182F8AE50E94231C12
:109D2000D82EB12C811104C081E50E94231CB82ECD
:109D3000A11001C0E12C8E2D90E0C11001C0F12CCA
:109D40008F0D911D019731F4D1100C94995AB110D7
:109D50000C94995A0E94413A82E299E00E9480391B
:109D600049C9883FA1E09A0711F40C94965B18F555
:109D7000853FE1E09E0711F40C948E5B40F4843F34
:109D8000914011F00C9480460E94677433C9863F5D
:109D900031E0930711F40C94925B873F914011F0EE
:109DA0000C94804661E083E50E94733091E089273E
:109DB0000E9482A01FC9803A53E0950709F4A5C10B
:109DC00078F48C30924011F00C9480468091C61645
:109DD00082FD02C00C94A95B80648093C6160AC9F8
:109DE000873EE3E09E0711F40C94B15B893E9340FB
:109DF00011F00C9480468091BC1681110C94C15BCB
:109E00000E9438906D3371058105910520F085EA37
:109E100099E00E94395C81EA99E00E94395C84EE05
:109E20008093CA038DE899E00E94803989E899E01F
:109E30000E94395CDFC880E50E945830C12CD12CCB
:109E40007601882321F00E94541C6B017C0183E57C
:109E50000E945830882361F00E94781C20E030E096
:109E60004AE754E40E9460E20E94EDE96B017C0144
:109E70000E949C7780914103909142030097E1F00A
:109E80000E9457B881E080939103C114D104E1048A
:109E9000F10431F00E9480C1C60ED71EE81EF91EE3
:109EA000809191038823B1F0C114D104E104F1043D
:109EB00049F40E941140F4CF60E083E795E00E94EE
:109EC000751FE0CF0E9480C16C197D098E099F0922
:109ED00097FDEFCF109291030E94B5BA8BC860E056
:109EE00086E895E00E94751F5E985E9815985E98CA
:109EF00081C80E94453A8FEA95E00E9480397AC86D
:109F00000E94D0D177C88091C61682FD73C80E9486
:109F10009FC78091C616877F80628093C6166AC8E5
:109F200060E00E946FCF1092CA0364C80E94DE33C3
:109F3000882321F00E94AEC70E9485908AE99CE0A8
:109F40000E947EB50E94B5BA55C88091C61682FFA0
:109F500003C08B7F8093C61680910006813069F420
:109F600082E0809300060E9480C16093DD037093BD
:109F7000DE038093DF039093E0030E94B5BA89EB80
:109F800095E00E947EB536C88091C61683FF32C820
:109F900083E50E945830882309F42CC80E94641C71
:109FA000AB01BC014093C2165093C3166093C41614
:109FB0007093C51688EB94E10E9410CC1BC88FEB00
:109FC00095E00E948039ADCB8091C61682FF27C0F4
:109FD000C090C216D090C316E090C416F090C5167B
:109FE00088ED95E00E9480394AE0C701B6010E94E1
:109FF0002BC78FE20E9468396091BE167091BF1620
:10A000008091C0169091C1164AE00E942BC78DE046
:10A010000E9468398AE00E9468390C94FA478AEEF7
:10A0200095E00E9480390C94FA4780914103909109
:10A0300042030E9427CF0C94FA478091C6168E7F68
:10A040008093C6160C94FA478091C61683FD02C011
:10A050000C94FA470E94F6CB8091C61683FD02C08D
:10A060000C94FA474091410350914203BE01645E53
:10A070007F4F80E00E9435B78C01009711F40C945B
:10A08000FA476C8D7D8D19821C8222E0AC01CE01D5
:10A0900001960E94AA6D811119C0F12CCE01019682
:10A0A0000E94A46DB801FF2031F186E196E00E9484
:10A0B00007408AE00E9468391092C2161092C316B7
:10A0C0001092C4161092C5160C94FA47CE01019650
:10A0D0000E94A4CC882309F361E0CE0101960E947E
:10A0E000506C0097D1F225EEDC012C931C820E946B
:10A0F00045C8F82ED3CF8EEF95E00E9407408BEF36
:10A1000095E00E9480390C94FA47209141033091E8
:10A1100042039091C61692609093C616C9010E94A0
:10A1200027CF0C94FA470E9438907B018C0120E8DD
:10A1300031E541E050E00E9442E8C9016DE671E07E
:10A140000E9498E84B015C01C801B70120E13EE0A4
:10A1500040E050E00E9442E8CA01B90128E130E045
:10A1600040E050E00E9442E8762E672EC62ED72EA1
:10A170008CE3282E312C412C512CC801B701A201AF
:10A1800091010E9442E8F62EE72ECA01B901A20110
:10A1900091010E9442E8CB018E010F5F1F4F811495
:10A1A000910431F1EF92FF927F936F936F927F92C0
:10A1B000BF92AF929F928F928CE496E09F938F9381
:10A1C0001F930F930E9491E10FB6F894DEBF0FBE6C
:10A1D000CDBFC8010E9457B80E94453AB80180E639
:10A1E00096E00E9407408AE00E9468390C94FA4782
:10A1F000A114B10489F0EF92FF927F936F936F9255
:10A200007F92BF92AF928CE396E09F938F931F93C0
:10A210000F930E9491E1D8CFCD2879F0EF92FF9271
:10A220007F936F936F927F9280E396E09F938F93DB
:10A230001F930F930E9491E1C7CF892B69F0EF9292
:10A24000FF927F936F9388E296E09F938F931F9383
:10A250000F930E9491E1B8CFEF92FF9284E296E0D3
:10A260009F938F931F930F930E9491E10F900F90F4
:10A270000F900F900F900F90ACCF80E50E94231CA1
:10A28000882311F40C94FA470E943430853608F084
:10A2900084E68093CA030C94FA47809100068130CB
:10A2A00011F00C94FA4782E0809300060E9480C16E
:10A2B0006093DD037093DE038093DF039093E003EC
:10A2C0000C94FA470E94A9900C94FA470E945E44AD
:10A2D0000C94FA470E94493A182F87FD0AC08DE670
:10A2E00096E00E948039812F0E9431718AE00E949D
:10A2F0006839C55BDF4F0FB6F894DEBF0FBECDBF28
:10A30000DF91CF911F910F91FF90EF90DF90CF9051
:10A31000BF90AF909F908F907F906F905F904F9085
:10A320003F902F90089580E50E943EBB81110C94D0
:10A33000FA4781E40E94231C60913706062F10E043
:10A34000811102C00FEF10E089E40E945830882389
:10A3500011F40C94F45B0E94343090E01816190646
:10A3600014F481E090E026E0289FF001299FF00D91
:10A370001124E255FA4F048115810F3F110519F0A0
:10A3800010F00FEF10E0009337060C94FA478EE4BC
:10A390000E945830882311F40C94FA470E94641CE0
:10A3A0006093D60B7093D70B8093D80B9093D90BF7
:10A3B0000C94FA4783E50E94231C882329F083E547
:10A3C0000E943EBB8093FB0A0E94453A8EE796E0CE
:10A3D0000E9480398091FB0A882351F110E000E04F
:10A3E00020E08091FB0A90E0B0E0A0E0002E04C0E5
:10A3F000B695A795979587950A94D2F780FF12C0D6
:10A40000FF24F394F20E222319F08CE20E946839A3
:10A41000F801EE0FFF1FEC58F94F859194910E94BF
:10A4200080392F2D0F5F1F4F05301105D1F679C9E7
:10A4300080E796E0C6CD8091FB0A83FF02C00C94B2
:10A44000FA4789E40E945830882311F40C94005C88
:10A450000E94343090E01816190614F481E090E060
:10A4600026E0289FF001299FF00D1124E255FA4FB4
:10A47000828193818C38910514F08CE890E0909360
:10A48000AC058093AB050E9468620C94FA478091FA
:10A49000FB0A83FF02C00C94FA4789E40E945830FB
:10A4A000882311F40C940B5C0E94343090E0181651
:10A4B000190614F481E090E026E0289FF001299F1E
:10A4C000F00D1124E255FA4F828193811CAA8C3839
:10A4D000910514F08CE890E09093AC058093AB0567
:10A4E0000E9468622091AB053091AC058091A9056E
:10A4F0009091AA05821793070CF03BC188E996E07A
:10A5000060E00E94751F81E0809352011DAA1EAA7F
:10A510001FAA18AE1BAE1CAE1DAE1EAE21961FAEFE
:10A5200021979CE322969FAF2297ACE12496AFAF90
:10A530002497B6E42896BFAF2897312C212CE0E869
:10A54000ECA7FFEBF8AB18A621E02FAF812C912CE4
:10A5500054010091AB051091AC05B801012E000C1F
:10A56000880B990B0E9401E26B017C01232D322D97
:10A570004CA558A90E94FAE1882389F08091A90589
:10A580009091AA053CA93111F7C041E048A70817EE
:10A5900019070CF018A63C2C2D2CECA6F8AA0E944A
:10A5A00080C16B017C01DC01CB012BAD3CAD4DAD1D
:10A5B0005EAD821B930BA40BB50BB7FD2FC0D7016B
:10A5C000C60188519C4FAF4FBF4F8BAF9CAFADAF13
:10A5D000BEAF80E00E94317185E896E00E9480392C
:10A5E00081149104A104B10409F4DBC0C501B401D4
:10A5F00068577C4E8F4F9F4F6C197D098E099F09BC
:10A6000028EE33E040E050E00E9442E8CA01B90180
:10A610004AE00E94D83B8AE00E9468390E941140BB
:10A620000E9480C16093E8057093E9058093EA0574
:10A630009093EB056091A9057091AA05072E000C77
:10A64000880B990B0E9401E269AF7AAF8C019B01E4
:10A65000AC01632D722D8CA598A90E94F0E82B0106
:10A660003C0120E030E0A9010E9474EA87FF04C0A9
:10A6700077FA709477F8709481149104A104B1046E
:10A6800009F093C020E030E040E85FE3C301B2018D
:10A690000E94FAE187FF10C09FADA2E88A2EA6E0D3
:10A6A0009A2EA12CB12C911103C0812C912C540114
:10A6B0008C0C9D1CAE1CBF1CA8A5AA2309F442C08B
:10A6C0002DA93EA94FA958AD2115310541055105C8
:10A6D00041F0D701C601821B930BA40BB50BB7FD4C
:10A6E00031C029AD3AADA80121966FAD21972296D0
:10A6F0007FAD229724968FAD249728969FAD2897FB
:10A700000E94F0E820E030E040E85FE30E94FAE1D8
:10A7100087FD35C0D701C601805A9541AF4FBF4F65
:10A720008DAB9EABAFABB8AF99AD21969FAF2197E4
:10A73000AAAD2296AFAF229724960FAF2497289602
:10A740001FAF2897809152018823C9F0811491048A
:10A75000A104B10461F0B8E8CB1AB3E1DB0AE10867
:10A76000F108C818D908EA08FB08F7FE08C01FAEB0
:10A77000F0CE89E896E0C4CE0817190764F48091FA
:10A780005201882311F40C94FA47109252010E944E
:10A79000B5BA0C94FA473C2C2D2CECA6F8AA18A6B6
:10A7A000FECE8FE30E94683936CF20E030E040E4EF
:10A7B00050E4C301B2010E9474EA18160CF07CCF79
:10A7C0004601570179CF0E94DE710E94AC770E944A
:10A7D000A9901092370668EE73E080E090E00E9446
:10A7E000A63360E087EA96E00E94751F0C94FA4752
:10A7F000809140038F7D8061809340030C94FA47E1
:10A80000809140038F7E8062809340030C94FA47CE
:10A8100083E50E9458308823F1F00E9480C1609344
:10A82000E8057093E9058093EA059093EB050E9493
:10A83000781C20E030E04AE754E40E9460E20E9485
:10A84000EDE960930B0170930C0180930D019093DF
:10A850000E010C94FA478BE092E00E94FF1B8823C4
:10A8600039F10E949C7788E50E94231C882331F0EF
:10A870005E9A809194058E7F8093940589E50E946D
:10A88000231C882331F05E9A809194058D7F8093FC
:10A8900094058AE50E94231C882311F40C94FA473E
:10A8A000159A809194058B7F809394050C94FA47B8
:10A8B0000E94AC770C94FA470E94493A87FF02C085
:10A8C0000C94FA478BE092E00E94FF1B882309F466
:10A8D0008BC0EAE6CE2EE1E0DE2EFCEFEF2EFAE0B2
:10A8E000FF2E10E0F60181916F010E9458308823FD
:10A8F00009F465C0133009F06DC00E94781C4B014B
:10A900005C0120E030E040EA51E40E94FAE187FF78
:10A910004EC0A501940160911C0B70911D0B80919C
:10A920001E0B90911F0B0E9474E92B013C01AC019E
:10A930009B0160911B0670911C0680911D069091F1
:10A940001E060E9460E260931B0670931C068093B3
:10A950001D0690931E06A301920160912C0B70912D
:10A960002D0B80912E0B90912F0B0E9460E2609333
:10A970002C0B70932D0B80932E0B90932F0B6091CB
:10A980002B0670912C0680912D0690912E060E9428
:10A99000FFE1A30192010E9460E20E94EDE9609351
:10A9A0002B0670932C0680932D0690932E06809292
:10A9B0001C0B90921D0BA0921E0BB0921F0B1F5FE1
:10A9C000B4E0EB0EF11C143009F08CCF0E947877C4
:10A9D0000C94FA470E94781CD70154966D937D938E
:10A9E0008D939C935797EBCF81E00E947ABA0C9499
:10A9F000FA470E9415BA80E295E10E94B8730C9460
:10AA0000FA478091410390914203009741F0FC0185
:10AA10002081222321F00E9457B80C94FA470E940B
:10AA2000B5BA0C94FA47009141031091420394E0A7
:10AA3000F12C40E0915009F1D8018C91282F2B7F07
:10AA40002134A1F411962C912133B9F4813419F1F8
:10AA5000853409F441E098012E5F3F4F89012F5F53
:10AA60003F4FD8018C918032C9F3E4CF803529F46F
:10AA7000F801818180538A3070F341110E94453A78
:10AA8000FF2021F087EB97E00E948039C8010E94E7
:10AA90006F390C94FA47FF24F394DDCF0E94F48EB3
:10AAA0000C94FA4781E080939205809391050E946F
:10AAB0000F8F0C94FA4710929205109291050E9404
:10AAC0000F8F0C94FA4790E080E00C94B64C0E94F3
:10AAD000413A8AEB97E00E9480390C94FA478AEA5F
:10AAE00090E00C94CD4C83EB91E00C94CD4C85E040
:10AAF00090E00C94EB4C8CE890E00C94EB4C90E0E4
:10AB000080E00C940B4D8FEF90E00C940B4D80E0A7
:10AB10000C94504D0E94493A87FF02C00C94FA47AA
:10AB20000AE611E06CEFE62E6AE0F62E7EE6C72E0E
:10AB300071E0D72ED8018D918D010E94231C8823AE
:10AB400059F00E94781C0E94EDE9F701608371833F
:10AB5000828393830E942A77F4E0EF0EF11CC016E3
:10AB6000D10641F70C94FA470E94493A87FF02C088
:10AB70000C94FA475AE6E52E51E0F52E10E000E07D
:10AB8000D7018D917D010E94231C882349F00E94EA
:10AB9000781CF801E450F54F64A375A386A397A32E
:10ABA0000C5F1F4F0031110559F70C94FA4783E5EC
:10ABB0000E945830882391F00E94781C6093300BDB
:10ABC0007093310B8093320B9093330B6093380B5F
:10ABD0007093390B80933A0B90933B0B80E50E9466
:10ABE0005830882351F00E94781C6093300B70938A
:10ABF000310B8093320B9093330B82E50E945830D7
:10AC0000882351F00E94781C6093340B7093350BAD
:10AC10008093360B9093370B84E50E94583088233D
:10AC200011F40C94FA470E94781C6093380B7093CF
:10AC3000390B80933A0B90933B0B0C94FA4788E0C6
:10AC400092E00E94FF1B882311F40C94FA4782E4DF
:10AC50000E94231C882351F00E94541C60930C0B0B
:10AC600070930D0B80930E0B90930F0B83E50E9456
:10AC7000231C882351F00E94781C60933C0B709336
:10AC80003D0B80933E0B90933F0B84E50E94231C69
:10AC9000882351F00E94781C6093400B7093410B05
:10ACA0008093420B9093430B88E50E94231C8823DA
:10ACB00051F00E94781C60930F06709310068093E9
:10ACC00011069093120689E50E94231C882351F0F7
:10ACD0000E94781C609313067093140680931506E7
:10ACE000909316068AE50E94231C8823B1F00E94E7
:10ACF000781C60931706709318068093190690933A
:10AD00001A062DEC3CEC4CEC5DE30E94FAE11816BF
:10AD100024F08FEE97E00E94803985E40E94231C86
:10AD2000882311F40C94FA470E94781C60931B0648
:10AD300070931C0680931D0690931E060C94FA4790
:10AD40004090010650900206609003067090040641
:10AD50002091290130912A0140912B0150912C0121
:10AD6000C301B2010E94F1E868A779A78AA79BA74F
:10AD70008090050690900606A0900706B090080601
:10AD800020912D0130912E0140912F0150913001E1
:10AD9000C501B4010E94F1E86CA77DA78EA79FA70B
:10ADA000C0900906D0900A06E0900B06F0900C06C1
:10ADB00020913101309132014091330150913401A1
:10ADC000C701B6010E94F1E868AB79AB8AAB9BABD7
:10ADD0002091350130913601409137015091380171
:10ADE000C301B2010E94F1E82B013C01209139011D
:10ADF00030913A0140913B0150913C01C501B401B1
:10AE00000E94F1E84B015C0120913D0130913E012F
:10AE100040913F0150914001C701B6010E94F1E805
:10AE20006B017C010E94453A8AE398E00E948039D8
:10AE300083E50E94231C882321F00E9448308093E0
:10AE4000270180912701882309F43FC084EB98E013
:10AE50000E94803982E398E00E94803948A559A574
:10AE60006AA57BA583E897E10E94263A4CA55DA5DB
:10AE70006EA57FA583E197E20E94263A48A959A9C9
:10AE80006AA97BA980E197E20E94263A80E398E0D4
:10AE90000E94803988E298E00E948039B301A201C3
:10AEA00083E897E10E94263AB501A40183E197E285
:10AEB0000E94263AB701A60180E197E20E94263A55
:10AEC0008AE00E9468390C94FA4780EB98E0C0CF82
:10AED00082E40E94231C882341F080911F019091FD
:10AEE00020019093100180930F0182E50E94231CA2
:10AEF000882341F080910F019091100190932001DF
:10AF000080931F0183E50E945830882331F00E940E
:10AF1000741C9093200180931F01E0914303F091F2
:10AF200044038081882311F40C94FA4760911F0137
:10AF3000709120018AE498E00E94373A85E20E94ED
:10AF400068398AE00E9468390C94FA470E94453AB1
:10AF500085E40E94683980E3800F0E946839F70118
:10AF6000EB5DFE4F608171818EE498E00E94373A7C
:10AF700085E20E9468398AE00E9468390C94FA4799
:10AF80008AE50E945830882331F10E94781C20E025
:10AF900030E040E050EC0E94FAE187FD3AC00E94A8
:10AFA000781C20E030E040E050E40E9474EA18167B
:10AFB000ACF10E94781C2091180B3091190B409134
:10AFC0001A0B50911B0B0E9460E20E94E6E9CB0134
:10AFD0000E94B9C105C083E50E9458308111D5CFC8
:10AFE00080E192E00E94FF1B81111DC00E94453A42
:10AFF00040916B0450916C0460916D0470916E04EB
:10B0000086E598E00E94263A8AE00E9468390C940E
:10B01000FA4760E070E080E090ECCDCF60E070E057
:10B0200080E090E4C8CF82E50E94231C8111DECF2E
:10B030000C94FA4785E40E943EBB811174C080E500
:10B040000E94231C882351F00E94781C6093AA144C
:10B050007093AB148093AC149093AD1489E40E9468
:10B06000231C882381F00E94781C2CEA35EC47E2EF
:10B070005EE30E9460E26093AE147093AF1480931D
:10B08000B0149093B11484E40E94231C882381F0AF
:10B090000E94781C2CEA35EC47E25EE30E9474E9DA
:10B0A0006093B2147093B3148093B4149093B51456
:10B0B0000E94453A4091AA145091AB146091AC148F
:10B0C0007091AD148BE698E00E94263A2CEA35EC9C
:10B0D00047E25EE36091AE147091AF148091B014BA
:10B0E0009091B1140E9474E9AB01BC0187E698E02D
:10B0F0000E94263A2CEA35EC47E25EE36091B214F6
:10B100007091B3148091B4149091B5140E9460E2D0
:10B11000AB01BC0183E698E00E94263A8AE00E94D7
:10B1200068390C94FA470E94413A8FE698E00E94F1
:10B1300080390C94FA4783E50E94231C182F88233A
:10B1400069F00E94741C9C0190935D0180935C01E6
:10B1500091E0232B09F090E09093480680E50E944F
:10B16000231C882361F020915C0130915D01232B29
:10B1700011F00E944830809348060C94FA47111150
:10B180000C94FA470E94453A8DE998E00E94803974
:10B1900080914806882391F085E898E00E948039E4
:10B1A00060915C0170915D018CE898E00E94373AF3
:10B1B00088E898E00E9480390C94FA4781E898E08A
:10B1C000EDCF0E940A3C0C94FA4783E50E94231CB1
:10B1D000182F30900104882319F00E944830382E2F
:10B1E0002091440B3091450B4091460B5091470BF9
:10B1F00027962CAF3DAF4EAF5FAF27974090480BDF
:10B200005090490B60904A0B70904B0B80914C0B07
:10B2100090914D0BA0914E0BB0914F0B2B968CAF94
:10B220009DAFAEAFBFAF2B97112329F0311003C0F4
:10B2300080E00E94983086E50E94231C21968FAF03
:10B2400021970E94B930882309F4B8C083E40E9492
:10B25000231C882309F49FC00E94781C6B017C0189
:10B26000A7E0B4E0B9ABA8ABB9A7A8A7F5E0FCA7E5
:10B270001AAE1BAE28EC2FAF02EC1CAA212C38EC26
:10B280003DAB42E449AF88A599A523969FAF8EAF09
:10B29000239715E02396AEADBFAD23978D909D907B
:10B2A000AD90BD902396BFAFAEAF23972CA9322DA2
:10B2B0004DA959ADC501B4010E94FAE187FF04C050
:10B2C0008CAA292CADAAB9AE2AAD3BAD4FAD502FFB
:10B2D000C501B4010E9474EA181624F48AAE9BAE2C
:10B2E000AFAE0B2D1150B1F6BCA5B150BCA7E8A56F
:10B2F000F9A57496F9A7E8A7B111C5CF2AAD3BAD62
:10B300004FAD502F6CA9722D8DA999AD0E94F1E817
:10B3100020E030E040E05FE30E9460E2A701960198
:10B320000E94F1E86B017C012DEB37E346E855EB19
:10B330000E9474EA87FD0AC02DEB37E346E855E327
:10B34000C701B6010E94FAE118162CF580E00E94B0
:10B35000983015E0A8A8B9A805E0D5016D917D91B8
:10B360008D919D915D014D01B4E08B1A9108A7016B
:10B3700096010E94F0E8F4016083718382839383D5
:10B38000015059F7115028A939A92C5E3F4F39AB0C
:10B3900028AB1111DFCF21964FAD2197442351F0F7
:10B3A0000E94B930882331F084EE98E00E94803901
:10B3B0000E94A739832D0E9498300DC0311005C01E
:10B3C00021963FAD21973323A9F30E94453A8AEF96
:10B3D00098E00E948039332051F08091010481115E
:10B3E00006C00E94413A85EC98E00E9480390E9494
:10B3F000453A87EB98E00E948039809101048823C8
:10B4000009F43EC084EB98E00E9480398AE00E94F3
:10B4100068392091440B3091450B4091460B509177
:10B42000470B27966CAD7DAD8EAD9FAD27970E94E3
:10B43000FAE181110C9474472091480B3091490B2B
:10B4400040914A0B50914B0BC301B2010E94FAE1AB
:10B4500081110C94744720914C0B30914D0B40910D
:10B460004E0B50914F0B2B966CAD7DAD8EAD9FADBD
:10B470002B970E94FAE181110C9474470C94FA47BF
:10B4800080EB98E0C1CFC11003C00FEF0C947E4E4B
:10B490000E94781C2091010630910206409103061B
:10B4A000509104060E94F0E820E030E040EA51E4C8
:10B4B0000E94F0E820E030E042E052E40E94F1E82F
:10B4C00021EC3FE04CE75CE30E9460E20E94E6E989
:10B4D000062F653010F40C947E4ED7CFF11003C0C8
:10B4E0001FEF0C948D4E0E94781C20910506309120
:10B4F000060640910706509108060E94F0E820E0F9
:10B5000030E040EA51E40E94F0E820E030E044EB13
:10B5100051E40E94F1E821E63BE046EB5CE30E9447
:10B5200060E20E94E6E9162F653010F40C948D4E0F
:10B53000D7CF07FD02C017FF08C00E94413A89E03B
:10B5400099E00E9480390C94FA470E94781CE02E02
:10B55000000FFF08A12F110FBB0B20E030E0A90165
:10B56000BB2091F025E02E9DF0012F9DF00D1124C0
:10B57000EA0FFB1FEE0FFF1FEE0FFF1FE95FFB4FF0
:10B580002081318142815381E5E0EE9D8001EF9D74
:10B59000100D11240A0F1B1F000F111F000F111F88
:10B5A000095F1B4F0E94F1E8D8016D937D938D9345
:10B5B0009C9313970C94FA470E94E9BA81110C945A
:10B5C000FA4795E6C92E96E1D92EE4E4FBE0F9A707
:10B5D000E8A79E012F5F3F4F1901790110E000E0BD
:10B5E000F6016591759185919491A8A5B9A58D9065
:10B5F0009D90AD90BD90B9A7A8A7A50194010E9408
:10B60000F0E82B013C01F701408251826282738293
:10B6100020E030E040EA51EC0E9474EA87FD0AC065
:10B6200020E030E040EA51E4C301B2010E94FAE1B7
:10B63000181684F4F801E954F94DE4911E1654F4F7
:10B64000B7FAB094B7F8B094D7018D929D92AD92AD
:10B65000BC921397F70181909190A190B1907F01D6
:10B6600020E030E040EA51ECC501B4010E9474EAE8
:10B6700087FD3FC020E030E040EA51E4C501B4015D
:10B680000E94FAE11816ACF10F5F1F4FF4E0CF0EE5
:10B69000D11C0330110509F0A3CF85E9E82E85E020
:10B6A000F82E10E0F10181919191A191B1911F01CA
:10B6B000F70181939193A193B1937F01812F0E9410
:10B6C00029851F5F133071F70E94128E60E082E4BB
:10B6D00099E00E94751F63E972E084E690E00E94A1
:10B6E00098946AEB72E084E690E00E9498940C943F
:10B6F000FA470E94413A80E699E00E94803961E071
:10B7000082E599E00E94751F0E946B1D68E270E05F
:10B7100088EC90E00E9498940C94FA470E9456A6F8
:10B720000C94FA470E941A8F0C94FA4781E0809398
:10B730006F040E944AA610926F04882311F40C949F
:10B74000FA470E94453A8EE799E00E9480390C94AE
:10B75000FA4783FD02C00C94FA470E94F6CB0C9482
:10B76000FA4781E08093A4051092961260E083E589
:10B770000E94733081110C94FA470E9491B80C9486
:10B78000FA470E942BD281110C94FA470C94004F77
:10B79000109145030E9480C16093E8057093E9050C
:10B7A0008093EA059093EB05112311F40C94FA476A
:10B7B0000E94453A84E50E946839812F0E9492C711
:10B7C00080E20E94683989EA99E00E9480390C94ED
:10B7D000FA4783E50E945830882311F40C94FA4705
:10B7E0000E94741C0C94524C83E50E9458308823AC
:10B7F00011F40C94BD510E94641C8B010C94BD513A
:10B8000083E50E945830882311F40C94FA470E9473
:10B81000741C0C943A5283E50E9458308CAB811111
:10B8200007C082E50E945830882311F40C94FA472F
:10B830000E94741C0C946752F1100C942B4A90E1F6
:10B84000E4E4FBE0ADEEB3E001900D929A95E1F7F0
:10B850000C94394A80E001110C940A4780E1E4E439
:10B86000FBE0ADEEB3E001900D928A95E1F70C9408
:10B870005F4A4F925F926F927F928F929F92AF92A8
:10B88000BF92CF92DF92EF92FF920F931F93CF93CD
:10B89000DF93CDB7DEB77C014DB65EB66090F105A3
:10B8A0007090F2058DB69EB66AE070E0C7010E9406
:10B8B0003CE16C018C010E191F09892B21F4C70191
:10B8C0000E9447E18C01C80101962DB73EB7281BA5
:10B8D000390B0FB6F8943EBF0FBE2DBF8DB79EB784
:10B8E00001965C01A801B7010E9468E1F501E00F33
:10B8F000F11F1082C5010E942E2F81E00E94454653
:10B90000C114D10451F076019FEFE91AF90A0FB67C
:10B91000F8949EBE0FBE8DBEC5CF0FB6F8949EBEE6
:10B920000FBE8DBEC3010E942E2F0FB6F8945EBECF
:10B930000FBE4DBEDF91CF911F910F91FF90EF9001
:10B94000DF90CF90BF90AF909F908F907F906F903F
:10B950005F904F9008954F925F926F927F928F9277
:10B960009F92AF92BF92CF92DF92EF92FF920F938E
:10B970001F93CF93DF93CDB7DEB728970FB6F89418
:10B98000DEBF0FBECDBF83E50E943EBB863028F0F0
:10B9900087E295E00E94803949C0833009F46EC186
:10B9A000E8F4813071F1823009F45AC084E195E005
:10B9B0000E9480390E94B9308823F1F080910104FF
:10B9C000811117C080EB98E00E9480398AE00E94C4
:10B9D00068390E94A7390E94128E28C0843009F469
:10B9E00093C1853019F780E00E9498300E9488301A
:10B9F000F2CF84EB98E0E8CF86E095E00E948039B2
:10BA0000EACF0E94883010920A01109209018091B9
:10BA1000D203811125C08EE40E94231C81111DC018
:10BA200084EF94E09093A2058093A10528960FB629
:10BA3000F894DEBF0FBECDBFDF91CF911F910F9164
:10BA4000FF90EF90DF90CF90BF90AF909F908F903E
:10BA50007F906F905F904F9008958AEF94E0E2CFCF
:10BA60008091090190910A0197FF03C08BEC94E04B
:10BA700091CF009709F0A8C01D821E821F821886F0
:10BA80008DEC9CECACE4BEE389839A83AB83BC83EE
:10BA9000BE016B5F7F4FCE0101960E94328680917E
:10BAA000090190910A01893191050CF0B3C021E0A0
:10BAB000209328019C012F5F3F4F30930A01209370
:10BAC000090165E00E948AE880FF03C024E0291B89
:10BAD000922F24E09202F0011124E756FA4E808062
:10BAE0009180A280B38094E08902F0011124EB5789
:10BAF000FA4E40805180628073808DEC9CECACE407
:10BB0000BEE38D839E83AF83B88719821A821B821E
:10BB10001C82CE0101966C01E12CF12C00EA10E4AC
:10BB2000A3019201C501B4010E947A8519821A828B
:10BB30001B821C82B601CE0105960E94328680923D
:10BB4000440B9092450BA092460BB092470B40924B
:10BB5000480B5092490B60924A0B70924B0B10921B
:10BB6000D2030091090110910A0189E1E82EF12C1C
:10BB7000093111050CF47801B70184E694E00E94C4
:10BB8000373A69E170E08FE594E00E94373A8AE045
:10BB90000E946839101611060CF01DCF1F9289E122
:10BBA0008F93FF92EF9288E494E09F938F9386E5C2
:10BBB00094E09F938F931F920E945C1F0FB6F8949E
:10BBC000DEBF0FBECDBF07CF815065E00E948AE87F
:10BBD00080FF03C024E0291B922F25E09202F00190
:10BBE0001124E80FF11D87FDFA95EE0FFF1FEE0FF0
:10BBF000FF1FE95FFB4F80914C0B90914D0BA09183
:10BC00004E0BB0914F0B80839183A283B38310922C
:10BC1000280145CF80E090E0A0EAB0E480934C0B8F
:10BC200090934D0BA0934E0BB0934F0B81E291E09C
:10BC30000E945F850E949C778FEF9FEF90930A018F
:10BC40008093090187EB94E00E94803985EA94E0B3
:10BC50000E9457B863E972E084E690E00E949894ED
:10BC60006AEB72E084E690E00E9498948FE994E099
:10BC70000E94395C81E00E94983071CF89E40E9473
:10BC80005830882371F00E94741C182F853068F09A
:10BC900064E070E08CE894E00E94373A89E894E030
:10BCA00079CE8AE40E94A139C1CE8AE40E9458303C
:10BCB0008823B9F30E94741C082F853048F064E093
:10BCC00070E086E794E00E94373A83E794E062CE22
:10BCD0008AE50E9458308823A9F00E94781C25E04C
:10BCE0001202F0011124E00FF11D07FDFA95EE0F8D
:10BCF000FF1FEE0FFF1FE95FFB4F6083718382839D
:10BD0000938369CE8AE5CECF8AE50E945830882396
:10BD1000C9F30E94781C60936B0470936C04809349
:10BD20006D0490936E0457CECF93DF93C0913E0C79
:10BD300081E6C89FE0011124C05CD34F8091FB0ACB
:10BD400080FF05C00E94453ACE010E946F39CE01A6
:10BD50000E942E2F80E0DF91CF910C9445460F93E7
:10BD60001F93CF93DF93CDB7DEB760970FB6F894EC
:10BD7000DEBF0FBECDBF8C01DC01ED91FC910280D6
:10BD8000F381E02DBE016F5F7F4F0995882309F491
:10BD900064C08981807CC9F56F81637070E0762F03
:10BDA0006627770F770F8885B4E08B9FC001112439
:10BDB000682B792B89858295869586958370682B6B
:10BDC0006F5F7F4F90E080E02A852370220F3B85D4
:10BDD00037FB332730F9232B3E813F70230F332766
:10BDE000331F2750310904C0660F771F881F991F22
:10BDF0002A95D2F760960FB6F894DEBF0FBECDBF7E
:10BE0000DF91CF911F910F910895803419F56885C6
:10BE10006695669570E090E080E0CB017727662715
:10BE20002A85622B098510E0102F0027012E000CB7
:10BE3000220B330B602B712B822B932B6F5F7F4F69
:10BE40008F4F9F4F4AE0660F771F881F991F4A95B3
:10BE5000D1F7D0CF8BE0F801848360E070E0CB01B4
:10BE6000C9CF0895FC0182810895CF92DF92EF92AD
:10BE7000FF9280910604882309F457C0C090020401
:10BE8000D0900304E0900404F090050420E030E03A
:10BE9000A901C701B6010E94FAE1882309F445C04F
:10BEA00020E030E040E05FE3C701B6010E9460E2BD
:10BEB0009B01AC010E9460E22BED3FE049E450E4BD
:10BEC0000E9460E29B01AC0160E070E080E89FE3CB
:10BED0000E9474E96B017C01C092FD03D092FE03C5
:10BEE000E092FF03F0920004609125017091260119
:10BEF000072E000C880B990B0E9401E22AE037ED17
:10BF000043E25CE30E9460E2A70196010E9460E2C6
:10BF1000609358017093590180935A0190935B018B
:10BF2000FF90EF90DF90CF900895C12CD12C80E846
:10BF3000E82E8FE3F82ED0CF2F923F924F925F9250
:10BF40006F927F928F929F92AF92BF92CF92DF9229
:10BF5000EF92FF920F931F93CF93DF93CDB7DEB78E
:10BF600066970FB6F894DEBF0FBECDBFDC01CD9053
:10BF7000DD90ED90FC90139714962D913D914D918D
:10BF80005C9117972B873C874D875E8720E030E0D8
:10BF900040EA51E4C701B6010E94F0E821EC3FE01D
:10BFA0004CE75CE30E9460E20E94E6E964300CF436
:10BFB00028C163E0662E660F7708F301EE0FFF1FBE
:10BFC000EE0FFF1FE756FA4E80809180A280B3806B
:10BFD000F3013196FA83E98320E030E040EA51E44E
:10BFE0006B857C858D859E850E94F0E821E63BE08F
:10BFF00046EB5CE30E9460E20E94E6E964300CF4E8
:10C0000004C163E0062F660F110BF801EE0FFF1F4E
:10C01000EE0FFF1FE756FA4E208131814281538196
:10C020002B833C834D835E83A8014F5F5F4F5E8B04
:10C030004D8BA5E0A69DC001A79D900D1124988B66
:10C040008F87FC01E00FF11FEE0FFF1FEE0FFF1FA8
:10C05000E95FFB4F20813181428153812F833887F3
:10C0600049875A87E981FA81EE0FFF1FEE0FFF1F04
:10C07000E756FA4EA5019401608171818281938116
:10C080000E94F0E8698B7A8B8B8B9C8BA5019401C5
:10C09000C701B6010E94F0E82B013C0185E049810F
:10C0A0005A81849F1001859F300C1124F101E00F0B
:10C0B000F11FEE0FFF1FEE0FFF1FE95FFB4F2F81F8
:10C0C000388549855A8560817181828193810E947A
:10C0D000F0E829893A894B895C890E9474E9A301B7
:10C0E00092010E9460E22F81388549855A850E941D
:10C0F000F1E86B017C01EF85F889AD89BE89EA0F13
:10C10000FB1FEE0FFF1FEE0FFF1FE95FFB4F80804D
:10C110009180A280B380FD01E20DF31DEE0FFF1FA1
:10C12000EE0FFF1FE95FFB4FA50194016081718154
:10C13000828193810E94F0E829893A894B895C8940
:10C140000E9474E9A30192010E9460E2A50194019A
:10C150000E94F1E8A70196010E94F0E84B015C0102
:10C16000ED89FE89EE0FFF1FEE0FFF1FE756FA4E17
:10C170002B813C814D815E816081718182819381BF
:10C180000E94F0E89B01AC01C501B4010E9474E972
:10C190004B015C012B813C814D815E816B857C85EF
:10C1A0008D859E850E94F0E89B01AC01C501B4011C
:10C1B0000E9460E2A70196010E94F1E820916B04C1
:10C1C00030916C0440916D0450916E040E94F1E82E
:10C1D00066960FB6F894DEBF0FBECDBFDF91CF914C
:10C1E0001F910F91FF90EF90DF90CF90BF90AF9095
:10C1F0009F908F907F906F905F904F903F902F9087
:10C20000089567FFD7CE60E0D5CE67FFFBCE60E034
:10C21000F9CE8F929F92AF92BF92CF92DF92EF9220
:10C22000FF92FC01C080D180E280F38020E030E00A
:10C2300040E251E4C701B6010E9460E220E030E034
:10C2400040E251E40E9460E24B015C0120E030E0FA
:10C25000A901C701B6010E94FAE120E030E040EAFE
:10C2600050E487FF04C020E030E040EA50ECC50114
:10C27000B4010E94F1E820E030E040E251E40E9485
:10C2800074E90E94E6E99B018BE237FF05C0222793
:10C290003327261B370B8DE28093D603C90168EE46
:10C2A00073E00E94ACE8CB01EAE0F0E0BF010E943D
:10C2B000ACE8805D8093D703C90164E670E00E941A
:10C2C000ACE8CB01BF010E94ACE8805D8093D8034D
:10C2D000C901BF010E94ACE8282FCB01BF010E9419
:10C2E000ACE8805D8093D9038EE28093DA03205D11
:10C2F0002093DB0386ED93E0FF90EF90DF90CF90EB
:10C30000BF90AF909F908F90089524E6829FC001C8
:10C31000112481589F4F6FEF70E00E94ACE8262FE8
:10C3200081E3643609F080E28093D80390E22A30FA
:10C3300040F03AE0822F632F0E947EE80E947EE860
:10C34000905D9093D903822F6AE00E947EE8905D11
:10C350009093DA0385E28093DB0388ED93E0089500
:10C360006091250170912601072E000C880B990B16
:10C370000E9401E22AE037ED43E25CE30E9460E2C2
:10C380002091FD033091FE034091FF035091000482
:10C390000E9460E2609358017093590180935A01A2
:10C3A00090935B0108958091E505811104C080910F
:10C3B000C0058093370608958091BB168823C1F08D
:10C3C00081508093BB16EEEEF4E1882351F081504A
:10C3D000990B2BE1289FF001299FF00D1124E355C3
:10C3E000FA4E8BE1A3EDB4E101900D928A95E1F74D
:10C3F0002091BB16211105C08091C61680628093E2
:10C40000C61681E090E0A0E0B0E0211103C080E01A
:10C4100090E0DC018093CE059093CF05A093D005EA
:10C42000B093D1051092C70581E08093DE0583E0CB
:10C43000809353010895CF93DF93EC01CB01BA01B0
:10C440000E9401E220E030E0A9010E94F1E80E9490
:10C45000E6E979836883DF91CF910895CF93DF93E5
:10C46000EC01CB01BA010E9401E229EC38EC48EC66
:10C470005EE30E9474E920E030E040E05FE30E9468
:10C48000F1E80E94EDE96883DF91CF9108950E9461
:10C4900001E229EC38EC48EC5EE30E9474E920E00C
:10C4A00030E040E05FE30E94F1E80E94EDE9862F72
:10C4B0000C948561E091E50586E0E802F001112425
:10C4C000E255FA4F8091C00590E0958384830895EA
:10C4D0002091AB053091AC0521153105E9F0809133
:10C4E000A9059091AA050296245031098217930755
:10C4F0009CF49093100580930F050E9480C1605EAC
:10C5000070448D4F9F4F6093110570931205809377
:10C5100013059093140508951092110510921205B9
:10C5200010921305109214050895CF93DF93EC0138
:10C530008D810E94C73B60E08B81DF91CF910C948D
:10C5400089C0DF92EF92FF920F931F93CF93DF93F7
:10C550008C01C62FD22FF32EE42ED52E0E94956289
:10C560000E94FFC18C2F80640E94BB3B8D2D0E94D6
:10C57000BB3B8E2D0E94BB3B8F2D0E94BB3B8D2F62
:10C580000E94BB3B87E8C11101C085E90E94BB3B0B
:10C59000CC3011F40E94C03BC0E00E94C03BF801C7
:10C5A000868387FF04C0CF3F11F0CF5FF6CFDF91C6
:10C5B000CF911F910F91FF90EF90DF90089561E070
:10C5C000FC0183810E9489C08FEF0C94BB3B0F93C9
:10C5D0001F93CF938C010E9495620E94FFC1C82FC8
:10C5E000882371F08DEF0E94BB3B0E94FFC1C82FD2
:10C5F000C8010E94DF628C2FCF911F910F91089587
:10C6000082E1F8018483F4CF8F929F92AF92BF9220
:10C61000CF92DF92EF92FF920F931F93CF93DF930E
:10C62000EC016A017B01590120E030E0A90167E3D8
:10C630000E94A162A501980167E1CE010E94A1625A
:10C64000811127C08F81833039F089E0CC0CDD1C4B
:10C65000EE1CFF1C8A95D1F7A701960169E1CE0176
:10C660000E94A16211E0882319F010E087E08C831A
:10C67000CE010E94DF62812FDF91CF911F910F9138
:10C68000FF90EF90DF90CF90BF90AF909F908F90F2
:10C69000089589E08C8310E0EBCFCF93DF93EC011A
:10C6A0006EBDFA01CA019E5F0DB407FEFDCF208169
:10C6B0002EBD0DB407FEFDCF21812EBD3296E817A9
:10C6C000F90791F70DB407FEFDCF8FEF0E94BB3B3A
:10C6D0008FEF0E94BB3B0E94C03B8E838F718530E1
:10C6E00049F083E18C83CE010E94DF6280E0DF911C
:10C6F000CF91089581E0FBCF0F931F93CF93DF93EA
:10C70000EC018B010E9495620E94FFC181110CC057
:10C7100085E18C8310E0CE010E94DF62812FDF91E2
:10C72000CF911F910F910895A8016CEFCE010E9447
:10C730004D63182F882361F3EECF0F931F93CF9390
:10C74000DF93EC0189018F81833039F089E0440F58
:10C75000551F661F771F8A95D1F79A01AB0168E1D3
:10C76000CE010E94A16281112AC0A8016EEFCE0104
:10C770000E944D63182F8823B1F00E94FFC1182F2B
:10C780008823D1F020E030E0A9016DE0CE010E94C5
:10C79000A162882321F086E18C8310E004C00E940E
:10C7A000C03B8111F8CFCE010E94DF62812FDF9163
:10C7B000CF911F910F91089587E18C83F4CF86E08C
:10C7C000EBCF1F93CF93DF93EC010E94956220E0A3
:10C7D00030E0A9016CE0CE010E94A16211E0882343
:10C7E00019F010E083E08C83CE010E94DF62812F7C
:10C7F000DF91CF911F9108951F93CF93DF93EC01A9
:10C800008F81833039F089E0440F551F661F771FF1
:10C810008A95D1F79A01AB0162E1CE010E94A16233
:10C8200011E0882319F010E085E08C83CE010E948E
:10C83000DF62812FDF91CF911F9108958F929F9298
:10C84000AF92BF92EF92FF920F931F93CF93DF931C
:10C850008C01EB017A010E9480C14B015C012CE24A
:10C86000820E21E0921EA11CB11C0E94C03BF80167
:10C8700086838F3F69F40E9480C1681979098A090B
:10C880009B0997FDF2CF81E1F8018483C0E021C0CC
:10C890008E3F71F5F1E0EF1AF1088FEF8EBDFE01CA
:10C8A0002FEF0DB407FEFDCF8EB581932EBDCF01C6
:10C8B0008C1B9D0B8E159F05A0F30DB407FEFDCFBD
:10C8C0008EB5CE0DDF1D88830E94C03B0E94C03B09
:10C8D000C1E0C8010E94DF628C2FDF91CF911F91D0
:10C8E0000F91FF90EF90BF90AF909F908F90089521
:10C8F0008FE0CACF0F931F93CF93DF93EC018B018F
:10C900000E94956240E052E0B801CE01DF91CF91E4
:10C910001F910F910C941E640F931F93CF93DF937D
:10C92000EC0189018F81833039F089E0440F551F74
:10C93000661F771F8A95D1F79A01AB0161E1CE019D
:10C940000E94A16281110AC040E052E0B801CE010C
:10C95000DF91CF911F910F910C941E6484E08C8322
:10C96000CE010E94DF6280E0DF91CF911F910F9195
:10C9700008958F929F92AF92BF92CF92DF92EF92E3
:10C98000FF920F931F93CF93DF93EC01162F1F821B
:10C990001C824B830E9480C16B017C0120EDC20E82
:10C9A00027E0D21EE11CF11CA89561E08B810E945A
:10C9B00089C08B810E9438B8249A2C9A279A26988D
:10C9C000259A81E00E94C73B85E08D830E94C73B8A
:10C9D0000AE08FEF0E94BB3B0150D9F7A89520E0F9
:10C9E00030E0A90160E0CE010E94A1628E83813017
:10C9F00081F00E9480C16C197D098E099F0997FD05
:10CA0000EECF81E08C83CE010E94DF621A8280E04B
:10CA10006AC0A8952AEA31E040E050E068E0CE0123
:10CA20000E94A162853041F581E08F83A8958F81B6
:10CA3000812C912C5401823029F4812C912CA12C31
:10CA400080E4B82E20E030E0A90167E3CE010E9427
:10CA5000A162A501940169E2CE010E94A1628E83C8
:10CA60008823F1F00E9480C16C197D098E099F090D
:10CA700097FDE8CF8AE0C6CF04E00E94C03B8E83DA
:10CA80000150D9F78A3A11F482E0CFCF0E9480C1D9
:10CA90006C197D098E099F0997FDBCCF82E0B2CF4A
:10CAA0008F818230C1F420E030E0A9016AE3CE0139
:10CAB0000E94A162882311F088E0A4CF0E94C03BAD
:10CAC000807C803C11F483E08F830E94C03B0E94F5
:10CAD000C03B0E94C03BCE010E94DF6281E08A839E
:10CAE000173070F41D83DF91CF911F910F91FF904C
:10CAF000EF90DF90CF90BF90AF909F908F90089570
:10CB000088E18C8384CF0F931F93CF93DF93EC0145
:10CB10008B0120E030E0A90169E00E94A16281114F
:10CB20000AC040E150E0B801CE01DF91CF911F91E2
:10CB30000F910C941E6480E18C83CE010E94DF6211
:10CB400080E0DF91CF911F910F910895CF93C82F6F
:10CB5000CB010E9480398CEF95E10E9480398DEEE7
:10CB600095E1CC2311F082EF95E10E9480398AE0B3
:10CB7000CF910C9468390C948CC10C948CC1409169
:10CB80006F0421E042276CE070E00C94DFB9409123
:10CB90006F0421E0422764E070E00C94DFB940911B
:10CBA0006F0421E0422761E070E00C94DFB940910E
:10CBB0006F0421E0422762E070E00C94DFB94091FD
:10CBC0006F0421E0422761E070E00C94DFB94091EE
:10CBD0006F0421E0422768E070E00C94DFB94091D7
:10CBE0006F0421E042276CE070E00C94DFB941E073
:10CBF00061E070E00C94DFB940916F0421E04227BE
:10CC00000C94DFB962E070E00C9418C16CE070E045
:10CC10000C9418C164E070E00C9418C161E070E0FD
:10CC20000C9418C161E070E00C9418C16CE070E0E5
:10CC30000C9418C10F931F93CF93811113C0C42F6D
:10CC40008B010E94453A8AEE96E10E948039C80124
:10CC50000E948039CC2331F08AE0CF911F910F914F
:10CC60000C946839CF911F910F910895CF93DF9362
:10CC700080911E1590911F15891B80958F7019F456
:10CC80000E941140F5CF80911E158F5F8F70A0918B
:10CC90001E159BE4A99FD0011124FD01E55BF94F0E
:10CCA000EF0119929A95E9F798E09083A05AB94F4D
:10CCB00090E1E0E2F5E101900D929A95E1F7209183
:10CCC0001E1590911F15291303C094E690931B1510
:10CCD00080931E15DF91CF910C94E13020E040E06D
:10CCE00070E060E086E397E60E94B01C81E08093EC
:10CCF000C6051092EF051092EE05089520E040E081
:10CD000070E060E08CE499E60C94B01C80914806D9
:10CD1000811114C080915C0190915D010197209177
:10CD2000A5143091A6142817390744F420E040E0F8
:10CD300070E060E081E599E60C94B01C0C947E668E
:10CD400021E02093C605FC0180819181A281B381FD
:10CD500080931B0190931C01A0931D01B0931E01B1
:10CD600020E040E070E060E08091BE059091BF055A
:10CD70000C94B01CCF93DF9300D000D0CDB7DEB7BA
:10CD80008DEC9CECACECBCE389839A83AB83BC83D5
:10CD9000CE0101960E94A0660F900F900F900F9009
:10CDA000DF91CF910895CF93DF9300D000D0CDB71E
:10CDB000DEB78DEC9CECACECBDE389839A83AB834E
:10CDC000BC83CE0101960E94A0660F900F900F9039
:10CDD0000F90DF91CF910895CF93DF9300D000D0D3
:10CDE000CDB7DEB780E090E0A0E8BFE389839A8307
:10CDF000AB83BC83CE0101960E94A0660F900F907A
:10CE00000F900F90DF91CF910895CF93DF9300D0D3
:10CE100000D0CDB7DEB780E090E0A0E2B1E4898336
:10CE20009A83AB83BC83CE0101960E94A0660F90CB
:10CE30000F900F900F90DF91CF91089581E0809334
:10CE4000C6051092940510927E0420E040E070E048
:10CE500060E087EE9BE60E94B01C87E495E190932A
:10CE6000A2058093A10508950C94841D8F929F9232
:10CE7000AF92BF92CF92DF92EF92FF92CF938091C9
:10CE8000C4051092C405882369F01092C605CF919D
:10CE9000FF90EF90DF90CF90BF90AF909F908F90DA
:10CEA0000C94841D4091CE055091CF056091D00522
:10CEB0007091D105411551056105710599F01092E8
:10CEC000CE051092CF051092D0051092D10581E0C9
:10CED000809353012AE0249FC001259F900D1124C7
:10CEE0000E94B9C180915301882309F4AEC06091BA
:10CEF000EE057091EF05072E000C880B990B0E9430
:10CF000001E2209140063091410640914206509145
:10CF100043060E9460E26B017C0120E030E040E2C9
:10CF200051E40E9460E220E030E04AE754E40E94CD
:10CF300060E24B015C0120E030E0A901C701B601CD
:10CF40000E94FAE120E030E040EA50E487FF04C0AC
:10CF500020E030E040EA50ECC501B4010E94F1E865
:10CF600020E030E040E251E40E9474E90E94E6E9EA
:10CF70006B017C018BE2F7FE09C0F094E094D09441
:10CF8000C094C11CD11CE11CF11C8DE28093D5031F
:10CF9000C701B60120E137E240E050E00E94C0E85E
:10CFA0008AE0882E912CA12CB12CCA01B901A501CF
:10CFB00094010E94C0E8605D6093D603C701B6018A
:10CFC00028EE33E040E050E00E94C0E8CA01B90119
:10CFD000A50194010E94C0E8605D6093D7038EE2D2
:10CFE0008093D803C701B60124E630E040E050E06A
:10CFF0000E94C0E8CA01B901A50194010E94C0E8DD
:10D00000605D6093D903C701B601A50194010E9438
:10D01000C0E8C62FCA01B901A50194010E94C0E869
:10D02000605D6093DA03C05DC093DB0365ED73E080
:10D0300089EA95E1CF91FF90EF90DF90CF90BF907C
:10D04000AF909F908F900C948A23CF91FF90EF9098
:10D05000DF90CF90BF90AF909F908F9008956FEF2B
:10D060008091C0050C943FC04F925F926F927F9267
:10D070008F929F92AF92BF92CF92DF92EF92FF92E8
:10D080000F931F93CF93DF930091C0050E9493BD30
:10D09000C091C70510E0000F111F08581A4E95E007
:10D0A000592E5C0E2EE5E22E25E1F22ED3E0DC1B9C
:10D0B0003FE2C32E38E6D32E40E5A42E45E1B42E40
:10D0C00082E0782E7C1A55E8852E55E1952E81E078
:10D0D000682E6C1A4C2E4194C11137C08091C9053D
:10D0E0008823B1F080915301882359F081E0909119
:10D0F000C905911180E024E04CE655E1642D0E94C1
:10D1000067BCCF5F5C12E8CF84E08093C8050CC099
:10D110008091C4051092C405882321F30E94841DC8
:10D120008091DE058823F1F2DF91CF911F910F915D
:10D13000FF90EF90DF90CF90BF90AF909F908F9037
:10D140007F906F905F904F900895C13059F5F8012E
:10D15000859194919093E7058093E6058091C905A8
:10D16000813081F080915301882359F21F929F9260
:10D170008F926F9281E09091C905913009F474C04B
:10D1800080E072C08091C4051092C405882351F3D9
:10D190008091C005682F0E943FC08091DE058823E2
:10D1A00009F3C2CFC23009F042C0F80185919491D1
:10D1B0009093E7058093E6058091C9058230D1F010
:10D1C00080915301882309F49CCFDF92CF92BF92C4
:10D1D000AF927F9281E09091C905923009F080E092
:10D1E0008F930E94A21C0F900F900F900F900F90A2
:10D1F0000F9087CF8091C4051092C405882301F356
:10D200000E942F688091DE058823D1F28DCF809116
:10D21000C4051092C4058823C1F06091C0058FEF4A
:10D220000E943FC08091DE05882379F07DCFC33016
:10D2300009F067CFF801859194919093E705809369
:10D24000E6058091C905833011F38091530188234D
:10D2500009F457CF1F92FF92EF92DF9381E09091F4
:10D26000C905933009F08CCF8F930E94A21C0F90B8
:10D270000F900F900F900F9044CF6CEC7BE682E004
:10D280000C946CD461ED7BE681E00C946CD466ED7B
:10D290007BE680E00C946CD463E879E683E00C9440
:10D2A0006CD4EF92FF920F931F9385EFE82E84E1E9
:10D2B000F82E07EF14E124E337E64EE756E667E081
:10D2C00075E18CE095E10E949EC41F910F91FF9043
:10D2D000EF900895EF92FF920F931F9387E3E82E4C
:10D2E00084E1F82E0AEA14E124E337E64CED5FE12D
:10D2F00069E374E18EE394E10E949EC41F910F9153
:10D30000FF90EF900895CF93DF9300D000D0CDB77A
:10D31000DEB78091C4051092C405882359F010929D
:10D32000C6050E94841D0F900F900F900F90DF9103
:10D33000CF9108956091CE057091CF058091D00571
:10D340009091D105611571058105910561F10E94EA
:10D3500001E220911B0130911C0140911D0150916F
:10D360001E010E9460E22091500B3091510B4091C0
:10D37000520B5091530B0E94F1E86093500B709345
:10D38000510B8093520B9093530B83E00E944120EA
:10D3900081E0809353011092CE051092CF05109238
:10D3A000D0051092D10580915301882309F4BBCF99
:10D3B0002091BA053091BB054091BC055091BD0547
:10D3C0006091500B7091510B8091520B9091530BC7
:10D3D0000E94F0E869837A838B839C83CE01019657
:10D3E0000E940961BC0188E896E20E948A239BCFD3
:10D3F0002F923F924F925F926F927F928F929F9265
:10D40000AF92BF92CF92DF92EF92FF921F93CF9392
:10D41000DF93CDB7DEB72C970FB6F894DEBF0FBE03
:10D42000CDBF1C01162F8091C4051092C40588231E
:10D43000E1F01092C6050E94841D2C960FB6F89458
:10D44000DEBF0FBECDBFDF91CF911F91FF90EF9058
:10D45000DF90CF90BF90AF909F908F907F906F9014
:10D460005F904F903F902F9008958091CE059091BE
:10D47000CF05A091D005B091D1058D839E83AF8358
:10D48000B887892B8A2B8B2B09F460C080912701E8
:10D49000882309F4BDC0809128018111B9C0613091
:10D4A00009F494C0623009F4A2C0809029019090E0
:10D4B0002A01A0902B01B0902C01C0903501D09092
:10D4C0003601E0903701F0903801612E712C6D81AA
:10D4D0007E818F8198850E9401E220911B0130910D
:10D4E0001C0140911D0150911E010E9460E2D30178
:10D4F000AA0FBB1FAA0FBB1FBC87AB87AC5BB44F87
:10D50000BA87A9872D913D914D915C910E94F1E8D8
:10D510002B013C018D819E81AF81B885B7FF8FC003
:10D52000A5019401C301B2010E94FAE187FD7FC009
:10D53000EB85FC85EC5BF44F408251826282738202
:10D54000812F0E94412081E0809353011092CE05EB
:10D550001092CF051092D0051092D1058091530101
:10D56000882309F46ACFF4E01F9FC0011124FC0155
:10D57000EC5BF44F8F5F994FDC012D913D914D9104
:10D580005C9160817181828193810E94F1E86B01DD
:10D590007C01C982DA82EB82FC822DEC3CEC4CEC03
:10D5A0005DE360911B0170911C0180911D019091C0
:10D5B0001E010E9474EA87FD52C0CE0101960E94AE
:10D5C0000961BC01C1010E948A2337CF80902D01DF
:10D5D00090902E01A0902F01B0903001C0903901A1
:10D5E000D0903A01E0903B01F0903C016ECF8090EA
:10D5F000310190903201A0903301B0903401C0907D
:10D600003D01D0903E01E0903F01F09040015DCFA0
:10D61000812C30E5932E33ECA32E37ECB32EC12CA6
:10D6200040E5D42E43ECE42E47E4F42E4ECFA985FA
:10D63000BA858D929D92AD92BC92139781CFA7012E
:10D640009601C301B2010E9474EA18160CF070CF63
:10D65000E985FA85C082D182E282F38271CF20E02F
:10D6600030E040E251E4C701B6010E9460E220E0F0
:10D6700030E04AE754E40E9460E24B015C0120E0A4
:10D6800030E0A901C701B6010E94FAE120E030E0D4
:10D6900040EA50E487FF04C020E030E040EA50EC6C
:10D6A000C501B4010E94F1E820E030E040E251E41D
:10D6B0000E9474E90E94E6E96B017C01F7FC62C0FC
:10D6C00020EA36E841E050E00E94C0E8CA01B90112
:10D6D0002AE030E040E050E00E94C0E8605D6093E6
:10D6E000D503C701B60120E137E240E050E00E94D7
:10D6F000C0E88AE0882E912CA12CB12CCA01B90176
:10D70000A50194010E94C0E8605D6093D603C70143
:10D71000B60128EE33E040E050E00E94C0E8CA01C4
:10D72000B901A50194010E94C0E8605D6093D70330
:10D730008EE28093D803C701B60124E630E040E0D2
:10D7400050E00E94C0E8CA01B901A50194010E94FD
:10D75000C0E8605D6093D903C701B601A5019401DB
:10D760000E94C0E8162FCA01B901A50194010E94C8
:10D77000C0E8605D6093DA03105D1093DB0385ED14
:10D7800093E01FCFF094E094D094C094C11CD11CBE
:10D79000E11CF11C6DE2A3CF62E081E996E20C94FA
:10D7A000F86961E088E996E20C94F86960E08FE935
:10D7B00096E20C94F8696BE172E681E992E90C94C7
:10D7C000CA246EE272E687E492E60C94CA24809141
:10D7D0005301882331F041E06DE673E182E00E945D
:10D7E0000ABC80917E048770873041F420E040E0DD
:10D7F00070E060E08DE690EA0C94B01C08950F9301
:10D800001F93CF93DF93CDB7DEB72A970FB6F89467
:10D81000DEBF0FBECDBF809153018823F1F01F9270
:10D8200089E18F938091D30390E001969F938F932A
:10D830008AE493E19F938F938E010F5F1F4F1F9395
:10D840000F930E9491E1B8018FE393E10E948A2334
:10D850000FB6F894DEBF0FBECDBF84E080935301B6
:10D860008091D203811108C020E040E070E060E0C8
:10D8700089E094E20E94B01C2A960FB6F894DEBFAD
:10D880000FBECDBFDF91CF911F910F910895CF9320
:10D89000DF93EC010E94C1CB1B82DF91CF910895F1
:10D8A000CF93DF93EC01462F41706C857D858E858B
:10D8B0009F850E948EC8882351F0888920E2829F2C
:10D8C000C001112489569D4EDF91CF91089590E0BB
:10D8D00080E0FACFCF93DF93EB01FC01238121118C
:10D8E00004C080E0DF91CF9108952250223028F4C7
:10D8F0008FE28883198281E0F5CF60E00E94506C4E
:10D90000009779F3DC0160E080E09EE22D91203207
:10D9100099F0883031F49E01260F311DF901908372
:10D920006F5F9E01260F311DAD0141505109FA0173
:10D930004081F90140836F5F8F5F8B3039F7FE01C3
:10D94000E60FF11D1082D7CF3F924F925F926F92F8
:10D950007F928F929F92AF92BF92CF92DF92EF927F
:10D96000FF920F931F93CF93DF93CDB7DEB72C9722
:10D970000FB6F894DEBF0FBECDBF5C01DC01599637
:10D980008D909C90F40181859285A385B4859C013E
:10D99000AD012F5F3F4F4F4F5F4F29873A874B872E
:10D9A0005C87D50114964D905D906D907C90179793
:10D9B000411451046104710409F459C0BFEF4B1ABA
:10D9C0005B0A6B0A7B0A312C730162011D821E8285
:10D9D0001F821886F40181859285A385B4852D81E7
:10D9E0003E814F815885281739074A075B0708F0A1
:10D9F00056C089859A85AB85BC858C159D05AE057D
:10DA0000BF0550F482E0C82ED12CE12CF12C92E01D
:10DA1000492E512C612C712C9E012F5F3F4FB70175
:10DA2000A601C4010E94C8CA8823C9F189819A81CC
:10DA3000AB81BC81892B8A2B8B2B01F1260137010D
:10DA40009FEF491A590A690A790A2D813E814F814F
:10DA500058852F5F3F4F4F4F5F4F2D833E834F833E
:10DA600058873FEFC31AD30AE30AF30AB3CF4080C3
:10DA700051806280738033243394A6CFC414D504BC
:10DA8000E604F70411F70FEF1FEF2FEF3FE0B701A8
:10DA9000A601C4010E9436CA782E81111AC0712CC9
:10DAA000872D2C960FB6F894DEBF0FBECDBFDF9149
:10DAB000CF911F910F91FF90EF90DF90CF90BF908B
:10DAC000AF909F908F907F906F905F904F903F901E
:10DAD0000895F5014481558166817781411551058D
:10DAE0006105710539F097018601C4010E9436CAAB
:10DAF0008823A9F2D5011496CD92DD92ED92FC9285
:10DB00001797332051F0D701C6010196A11DB11D11
:10DB1000F40180839183A283B383F501858996897B
:10DB2000A789B08D892B8A2B8B2B09F0B9CFC58A99
:10DB3000D68AE78AF08E818180688183B1CF40E008
:10DB400050E0BA010C9410CCFC01238121110C94FB
:10DB5000476C08952F923F924F925F926F927F92FF
:10DB60008F929F92AF92BF92CF92DF92EF92FF92ED
:10DB70000F931F93CF93DF93CDB7DEB7C354D10973
:10DB80000FB6F894DEBF0FBECDBF4C015B016A013A
:10DB9000222E19821C821C8E1F8E6115710521F5A3
:10DBA00010E0CE014C960E94A46DCE0101960E9419
:10DBB000A46D812FCD5BDF4F0FB6F894DEBF0FBE93
:10DBC000CDBFDF91CF911F910F91FF90EF90DF902C
:10DBD000CF90BF90AF909F908F907F906F905F900D
:10DBE0004F903F902F900895FC0183818111D8CFF1
:10DBF000FA0180818F32A1F18B01CE0101967C0167
:10DC00003C0180E2382E2E019CE1490E511C2396E6
:10DC1000EFAE23972496FFAE249722963FAE22972D
:10DC200021963FAE21973FAE3EAE3DAE3CAE3BAE01
:10DC30003AAE39AE38AE3FAA960190E047E0D9013E
:10DC40008D91882309F447C08F3209F444C08E3285
:10DC500009F54A3009F4A4CF98E04AE09D01EFCFDE
:10DC6000FB01838182508B01823060F0618D728D67
:10DC7000CE014C960E9480D18E01045E1F4F8823F6
:10DC800009F48ECFC6016C010196F60120812F3276
:10DC9000D1F3B3CFE7ECF2E22491222321F03196C5
:10DCA0008213FACF7DCF491708F47ACF813208F476
:10DCB00077CF8F3709F474CF3FE9380F3A3108F442
:10DCC00020EEE7E3F0E0EC0FFD1FE90FF11D820FFE
:10DCD00080839F5FC3CF8FA9803209F461CF690130
:10DCE000F90180812F5F3F4F8F32C9F3882301F103
:10DCF00021E0AE01495C5F4FB801C7010E949ED28E
:10DD0000882309F44DCF0A151B0519F0C8010E949C
:10DD1000476C942D852D6E147F0431F023969FADB2
:10DD2000239724968FAD24978701E92EF82E75CF7F
:10DD3000222DAE01495C5F4FB801C4010E949ED202
:10DD4000182F2FCF2F923F924F925F926F927F9218
:10DD50008F929F92AF92BF92CF92DF92EF92FF92FB
:10DD60000F931F93CF93DF93CDB7DEB7ED970FB629
:10DD7000F894DEBF0FBECDBF8091CA05882369F13C
:10DD80008091C61600E010E083FF23C083ED94E18C
:10DD90000E949F6D8BE1E3EDF4E1DE01919601902D
:10DDA0000D928A95E1F710E000E0BE016F5F7F4FB2
:10DDB000CE0181960E9431CE18163CF4CE01019618
:10DDC0000E9414C8080F111DF0CFCE0181960E9449
:10DDD000A46D00937304109374040E9493BD10917A
:10DDE000C7051CAF85E0810F8DAF312E31948CEDCE
:10DDF000C82E81E6D82E93EEA92E94E1B92E81E0AB
:10DE0000782E711A27EE822E24E1922E111113C062
:10DE10008091C905882391F180915301882359F09D
:10DE200081E09091C905911180E024E040EF54E138
:10DE3000632D0E9467BC8091C61685FF55C01130C6
:10DE4000D9F48091C9058130F1F180915301882383
:10DE500009F45BC11F929F928F927F9281E0909113
:10DE6000C905913009F080E08F930E94A21C0F90A9
:10DE70000F900F900F900F9082E066C08091C405C4
:10DE80001092C405882341F20E94841D8091DE0512
:10DE9000882311F2ED960FB6F894DEBF0FBECDBF0A
:10DEA000DF91CF911F910F91FF90EF90DF90CF9076
:10DEB000BF90AF909F908F907F906F905F904F90AA
:10DEC0003F902F9008958091C4051092C405882337
:10DED00009F4BBCF1092C7050E94D0D18091DE0516
:10DEE000882309F4B2CFD6CF83FF2DC0113021F69D
:10DEF0008091C9058130D1F080915301882309F4C4
:10DF000004C1DF92CF92BF92AF927F9281E0909155
:10DF1000C905913009F080E08F930E94A21C0F90F8
:10DF20000F900F900F900F900F90A6CF8091C40587
:10DF30001092C405882301F30E94DC618091DE0504
:10DF40008823D1F2A7CF81E090915301992309F45E
:10DF5000DDC0582E082FF12CE12C412E9CAD491A22
:10DF6000802F2091730430917404E216F30608F0B8
:10DF7000CDC00113A5C083ED94E10E949F6D202EBA
:10DF800025188BE1E3EDF4E1DE01919601900D920D
:10DF90008A95E1F7612CBE016F5F7F4FCE018196BC
:10DFA0000E9431CE18167CF4CE0101960E9414C84E
:10DFB000882389F326106BC0BE016F5F7F4F83EF0C
:10DFC00095E00E942FC8CE0181960E94A46D809199
:10DFD000C6169091C90584FF78C0911366C08091E0
:10DFE000C4051092C405882309F45FC019821C82FD
:10DFF0008091D6146EEE74E1882311F063ED74E124
:10E0000021E043EF55E0CE0101960E94AA6D8823DE
:10E0100009F43FC08BE1FE013196A3EDB4E101901C
:10E020000D928A95E1F78091C6168F7D8093C61672
:10E03000A091BB16AA3080F481E08A0F8093BB16B2
:10E040008BE18A9FD0011124A355BA4EE3EDF4E190
:10E0500001900D928A95E1F7CE0101960E94A46D80
:10E060001092C70582E090E0A0E0B0E08093CE057A
:10E070009093CF05A093D005B093D10581E0809314
:10E08000DE051092D40383E08093530103CF6394A1
:10E0900082CF0E94453A63EF75E08DEC94E10E94D7
:10E0A00007408AE00E946839D7CF809153018823C6
:10E0B00039F081E0911380E041E0642D0E94A8BC1A
:10E0C0008FEFE81AF80A0F5F4BCF911759F0809144
:10E0D00053018823A9F381E09091C905911380E051
:10E0E00040E0EBCF8091C4051092C405882379F3FA
:10E0F00083EF95E00E94B6C70E946B1D0E94B5BADF
:10E100008091DE05882319F3C5CE82E01F5F9DADA7
:10E1100091137CCE8093C805BDCE8F929F92AF9213
:10E12000BF92CF92DF92EF92FF92CF936B017C016F
:10E13000B42E20E030E0A9010E94FAE187FF07C079
:10E140008DE20E946839F7FAF094F7F8F094C0E095
:10E1500060E070E080E09FE3CB1541F02DEC3CECFB
:10E160004CEC5DE30E9460E2CF5FF6CFA701960121
:10E170000E94F1E86B017C010E94EDE94B015C011A
:10E180004AE00E942BC7CC2379F1C501B4010E945B
:10E19000FFE19B01AC01C701B6010E94F0E86B01F1
:10E1A0007C018EE20E946839C150F0F020E030E03E
:10E1B00040E251E4C701B6010E9460E26B017C01BC
:10E1C0000E94EDE94B015C014AE00E942BC7C501AA
:10E1D000B4010E94FFE19B01AC01C701B6010E949E
:10E1E000F0E86B017C01E0CFCF91FF90EF90DF90E2
:10E1F000CF90BF90AF909F908F900895EF92FF9235
:10E200000F931F93CF937C018B01C2E44F3F09F022
:10E21000C4E580E20E9468398C2F0E9468398AE345
:10E220000E946839F701608171818281938142E0A7
:10E230000E948D708BEB92E20E948039F801608120
:10E2400071818281938142E00E948D7062E070E072
:10E2500080E090E0CF911F910F91FF90EF900C9490
:10E26000E5C01F93CF93DF93CDB7DEB728970FB6E6
:10E27000F894DEBF0FBECDBF182F6091A714709128
:10E28000A814072E000C880B990B0E9401E26D83E5
:10E290007E838F8398876091A5147091A614072EB2
:10E2A000000C880B990B0E9401E269837A838B83AF
:10E2B0009C834AEFBE016B5F7F4FCE0101960E94A7
:10E2C000FE706091AB057091AC05072E000C880BB9
:10E2D000990B0E9401E26D837E838F839887609102
:10E2E000A9057091AA05072E000C880B990B0E94B6
:10E2F00001E269837A838B839C834FEFBE016B5F5E
:10E300007F4FCE0101960E94FE706091AD051F3FC8
:10E3100039F085E11802F0011124EF55FB4E6085BC
:10E3200070E083EC92E20E94373A6091AD0570E0B4
:10E330008EEB92E20E94373A28960FB6F894DEBF31
:10E340000FBECDBFDF91CF911F9108950F930FB7EF
:10E350000F9300916E000B7F00936E0078940F93E3
:10E360000BB70F930CB70F921F922F933F934F93BE
:10E370005F936F937F938F939F93AF93BF93EF932D
:10E38000FF9311240E94637AFF91EF91BF91AF91A7
:10E390009F918F917F916F915F914F913F912F91BD
:10E3A0001F900F900CBF0F910BBF0F910460F8945A
:10E3B00000936E000F910FBF0F911895CF93DF93CD
:10E3C000C1EAD4E11F821E820E948CC118865D982A
:10E3D000C5EAD5E01F821E820E94686218865C989A
:10E3E000DF91CF910895109237060E94DE710C9450
:10E3F0006B1D4F925F926F927F928F929F92AF921E
:10E40000BF92EF92FF920F931F93CF93DF93B0E2EF
:10E41000A0E06A2F70E0AB014B0F511D5595479559
:10E42000411117C0EFEDF1E285919491282F822FD1
:10E43000DF91CF911F910F91FF90EF90BF90AF9020
:10E440009F908F907F906F905F904F900895B42F22
:10E45000E2CFA41711F0B41303C0EBE5F2E2E4CF6E
:10E460009A0121503109220F331F220F331FF90166
:10E47000E352FE4DE590F490F901EF51FE4D059108
:10E4800014918E159F051CF3A42F081719070CF47F
:10E49000C0CFBC01F901E152FE4DC591D491F90103
:10E4A000ED51FE4DA590B4906E197F09072E000C1A
:10E4B000880B990B0E9401E22B013C01B5016C1BFA
:10E4C0007D0B072E000C880B990B0E9401E29B012B
:10E4D000AC01C301B2010E9460E24B015C01B801D2
:10E4E0006E197F09072E000C880B990B0E9401E220
:10E4F0009B01AC01C501B4010E9474E94B015C01B0
:10E50000BE01DD0F880B990B0E9401E29B01AC015B
:10E51000C501B4010E94F1E80E94E6E9262F972F79
:10E5200086CFCF93DF93C1EAD4E18A819B810E9499
:10E5300096B69D838C83C5EAD5E08A819B810E9433
:10E54000F9719D838C83A89510927204DF91CF910D
:10E550000895EF92FF920F931F93CF93DF93C82FED
:10E560007B018A018091A4058130A1F40E94413A87
:10E57000C7010E94803983E991E20E948039C7FD7A
:10E5800033C08C2F0C2E000C990B0E942EB78AE002
:10E590000E9468390E94DE71A8958091F50481116E
:10E5A00032C081E08093F50480E88093A4050E9446
:10E5B000DE71D5E1D150149AE1F069E170E080E0BC
:10E5C00090E00E94E5C0A895149868E270E080E0B1
:10E5D00090E00E94E5C0A89568E270E080E090E0DD
:10E5E0000E94E5C0A895E6CF8FE891E20E948039AD
:10E5F000CECF68E871E2CF3F11F06CE871E240E005
:10E60000C8010E946E3ADF91CF911F910F91FF9048
:10E61000EF9008954F925F926F927F928F929F92A8
:10E62000AF92BF92CF92DF92EF92FF920F931F9320
:10E63000CF93DF93EC016B014A01B22EFA014080C7
:10E64000518062807380A30192016D817E818F81F0
:10E6500098850E94FAE18823A1F04D825E826F8244
:10E660007886AA24A39420E030E0A901F401608117
:10E670007181828193810E9474EA18160CF0A12C9A
:10E68000AC828C818230A1F0833009F45AC0813091
:10E69000C9F52D813E814F815885F60160817181D8
:10E6A000828193810E94FAE187FD2CC082E08C83F5
:10E6B000B701FF0C880B990B0E9401E29B01AC0192
:10E6C0006D817E818F8198850E94F0E89B01AC016D
:10E6D000F60160817181828193810E9474EA87FDD5
:10E6E00022C00E9480C16B017C019801A8EEB3E0BA
:10E6F0000E946FE8C60ED71EE81EF91EC882D98296
:10E70000EA82FB82DF91CF911F910F91FF90EF90F2
:10E71000DF90CF90BF90AF909F908F907F906F9041
:10E720005F904F9008950E9480C1088119812A81CD
:10E730003B81601B710B820B930B97FDE3CF83E052
:10E740008C834DE552E26DE672E28B2DDF91CF9125
:10E750001F910F91FF90EF90DF90CF90BF90AF90FF
:10E760009F908F907F906F905F904F900C94A972C4
:10E77000CF93DF93EC01488159816A817B818EE7D9
:10E7800091E20E94F93B4C815D816E817F8185E23F
:10E7900097E20E94F93B488559856A857B8581E22D
:10E7A00097E20E94F93B8AE0DF91CF910C9468399F
:10E7B000BC012091D6043091D7044091D6045091E9
:10E7C000D7042417350731F481E02617370709F0FD
:10E7D00080E008959A01F1CF0F930FB70F93009146
:10E7E0006E000F930B7F00936E0000916F000D7F02
:10E7F00000936F000F930BB70F930CB70F921F92FC
:10E800002F933F934F935F936F937F938F939F9338
:10E81000AF93BF93EF93FF9311240E94F87BFF9176
:10E82000EF91BF91AF919F918F917F916F915F9188
:10E830004F913F912F911F900F900CBF0F910BBFE5
:10E840000F910260F89400936F000F9100936E0097
:10E850000F910FBF0F9118950000000000000000FD
:10E860008091930580FF27C0459A8FEF80938C0499
:10E8700080919305869580FF21C0479A8FEF809302
:10E880008D04809193058695869580FF1AC02A98FD
:10E890008FEF80938E04809193058695869586955B
:10E8A00080FF12C0289A8FEF80938F040000000031
:10E8B000000000000895459881E0D8CF479881E096
:10E8C000DECF2A9A81E0E5CF289881E0EDCFCF9284
:10E8D000DF92EF92FF920F931F93CF93DF93CDB709
:10E8E000DEB7C658D1090FB6F894DEBF0FBECDBF54
:10E8F000C358DF4F188219821A821B82CD57D0402D
:10E900008091140290911502A0911602B091170205
:10E91000CF57DF4F88839983AA83BB83C158D040E8
:10E9200084E690E090930E0680930D061092B71443
:10E930001092B61410928B0464E070E0CE018F57F1
:10E940009F4F0E9418C180910D0690910E0602966D
:10E9500090930E0680930D061092B7141092B61481
:10E9600081E0CA57DF4F8883C658D040CE018A570E
:10E970009F4F0E94126668E470E08CEF9AE00E945C
:10E9800018C160E170E08FE096E00E9418C18AE053
:10E9900097EDA3EABCE3C358DF4F88839983AA832A
:10E9A000BB83CD57D040CE0183589F4F0E940A664B
:10E9B00085E995E00E9416667E018DE6E80EF11C61
:10E9C0008FEFD7018C93C7010E94126619821A82B9
:10E9D0001B821C828E010F5F1F4FC8010E940A66B6
:10E9E00019821A821B821C82C8010E940A6685E075
:10E9F0008983F70180838BE694E00E940A66C80150
:10EA00000E941266C7010E94126664E670E087E009
:10EA100094E00E9418C18CE0D8011D928A95E9F714
:10EA2000C8010E941666C358DF4F188219821A82E5
:10EA30001B82CD57D0403AE0D32EDA94DD2031F05E
:10EA4000CE0183589F4F0E940A66F7CF88E0F701F6
:10EA5000982F11929A95E9F7D8011D928A95E9F7B6
:10EA600083E0CB57DF4F8883C558D040EA968FAFFD
:10EA7000EA97CE018B579F4F0E941266CE018758AE
:10EA80009F4F0E94126668E070E0C8010E9418C1A2
:10EA900068E070E0C7010E9418C1C358DF4F1882B8
:10EAA00019821A821B82CD57D0402AE0C22ED12C67
:10EAB000B1E0CB1AD10831F0CE0183589F4F0E94AC
:10EAC0000A66F6CF19828FEFF7018083C8010E9492
:10EAD0000E66C7010E94126680E1D82ED801ED2D86
:10EAE0001D92EA95E9F760E170E0C8010E9418C143
:10EAF0001982C8010E940E666CE070E08EEA95E013
:10EB00000E9418C1198A1A8A1B8A1C8A80E090E028
:10EB1000A0E8BFE38D879E87AF87B88B8091AA144A
:10EB20009091AB14A091AC14B091AD1489839A83E9
:10EB3000AB83BC832CEA35EC47E25EE36091AE1414
:10EB40007091AF148091B0149091B1140E9474E947
:10EB50006D837E838F8398872CEA35EC47E25EE3F2
:10EB60006091B2147091B3148091B4149091B51463
:10EB70000E9460E269877A878B879C8764E170E0F6
:10EB8000C8010E9418C184E190E09A838983C8017A
:10EB90000E9402668CE0E6E9F1E0D80101900D9256
:10EBA0008A95E1F7C8010E9406668CE0E6E9F1E08B
:10EBB000D80101900D928A95E1F7C8010E9406667E
:10EBC0001982C8010E9412668FE790E09A838983B8
:10EBD000C8010E94026685E0E2EAF1E0D8010190F6
:10EBE0000D928A95E1F765E070E0C8010E9418C1B6
:10EBF0001982C8010E940E6680E2E7EAF1E0D801BE
:10EC000001900D928A95E1F760E270E0C8010E94E0
:10EC100018C1D7011C92C7010E940E6686E094E0DD
:10EC20000E940E6682E094E00E940A66C358DF4F9D
:10EC3000188219821A821B82CD57D040CE01835888
:10EC40009F4F0E940A6680E2F80111928A95E9F7C7
:10EC500060E270E0C8010E9418C1FE01F99688E0E8
:10EC6000DF011D928A95E9F744E650E060E070E02C
:10EC700049835A836B837C834D835E836F8378875C
:10EC800083E090E0A0E0B0E089879A87AB87BC87FB
:10EC90004D875E876F87788B498B5A8B6B8B7C8B0C
:10ECA0008D8B9E8BAF8BB88F898F9A8FAB8FBC8FDC
:10ECB0008D8F9E8FAF8FB8A38EE190E0A0E0B0E083
:10ECC00089A39AA3ABA3BCA38DA39EA3AFA3B8A70C
:10ECD00089A79AA7ABA7BCA78DA79EA7AFA7B8ABDC
:10ECE00089AB9AABABABBCAB8DAB9EABAFABB8AFAC
:10ECF00060E470E0C8010E9418C1F8018D2D1192E6
:10ED00008A95E9F760E170E0C8010E9418C1D80156
:10ED10001D92DA94E9F760E170E0C8010E9418C121
:10ED2000C358DF4F188219821A821B82CD57D040F8
:10ED3000CE0183589F4F0E940A669CE0D92EF801AD
:10ED40008D2D11928A95E9F76CE070E0C8010E9460
:10ED500018C18CE6D8011D928A95E9F76CE670E03F
:10ED6000C8010E9418C18FE794E00E940666F7016F
:10ED700010821182128213821482158216821782E7
:10ED800068E070E0C7010E9418C1F7011192DA949F
:10ED9000E9F7CB57DF4F1882C558D04080E090E0AC
:10EDA000A0E4B0E4ED968CAF9DAFAEAFBFAFED97F2
:10EDB000C7010E941666CE018B579F4F0E941266B4
:10EDC000CE0187589F4F0E940A6680918B04811163
:10EDD00024C000910D0610910E068091B6149091FA
:10EDE000B714D7018D939C9384E690E090930E0620
:10EDF00080930D0664E070E083ED91E00E9418C1FD
:10EE0000C7010E94026691E00D34134009F490E0BE
:10EE100080918B04892B80938B0480918B048111CA
:10EE200005C060E086EC96E10E94751F90918B040E
:10EE300081E08927CA57DF4F0FB6F894DEBF0FBEB7
:10EE4000CDBFDF91CF911F910F91FF90EF90DF9099
:10EE5000CF900895AF92BF92CF92DF92EF92FF9240
:10EE60000F931F93CF93DF93CCEFDAE00FE116E01F
:10EE70008CE0A82E8BE0B82EC12CD12C7601C39447
:10EE800069917991899199910E94FFE12889398945
:10EE90004A895B890E9460E20E94EDE9F801619372
:10EEA0007193819391938F01C616D706E806F906F0
:10EEB00010F46B017C01AC16BD0611F76FEF7FEF0C
:10EEC000CB01A70196010E9442E820932F063093C0
:10EED00030064093310650933206DF91CF911F9157
:10EEE0000F91FF90EF90DF90CF90BF90AF9008957B
:10EEF0000F931F93CF93DF9300E11BE0C8E3D6E0AD
:10EF0000F80121913191419151918F0160E070E0C0
:10EF100080E89FE30E9474E96993799389939993B8
:10EF2000F6E0C834DF0761F70E9499B9DF91CF910D
:10EF30001F910F910C942A7790911E1580911F15A7
:10EF4000981306C08091490690914A06892B19F0C2
:10EF50000E941140F1CF089590911E1580911F15C8
:10EF6000981308C08091490690914A06892B11F4A4
:10EF70000C94CA330E941140EFCFCF93DF932091BE
:10EF80000104222379F0EC010E949C5F9B01AC01FB
:10EF9000688579858A859B850E94F0E868877987EE
:10EFA0008A879B87DF91CF910895CF93DF9320913C
:10EFB0000104222379F0EC010E949C5F9B01AC01CB
:10EFC000688579858A859B850E94F1E868877987BD
:10EFD0008A879B87DF91CF9108954F925F926F92BE
:10EFE0007F928F929F92AF92BF92CF92DF92EF92D9
:10EFF000FF920F931F93CF93DF93CDB7DEB76A973E
:10F000000FB6F894DEBF0FBECDBF9A8F898F5B011C
:10F010008A01DC01D6966D917D918D919C91D99755
:10F020000E94FFE16B017C01F50120813181428169
:10F0300053810E9460E20E945DE92B013C01D801EE
:10F040002D913D914D915C91C701B6010E9460E206
:10F050000E945DE94B015C01C301B2010E94EDE930
:10F06000698B7A8B8B8B9C8B683771058105910539
:10F0700040F428E730E040E050E0298B3A8B4B8B9E
:10F080005C8BC501B4010E94EDE96D877E878F8797
:10F09000988B683771058105910540F488E790E009
:10F0A000A0E0B0E08D879E87AF87B88BE98DFA8DA1
:10F0B000EE5BFF4F208131814281538129833A8366
:10F0C0004B835C83CA01B9010E9401E22B013C0120
:10F0D00069897A898B899C890E94FFE169877A878F
:10F0E0008B879C8720E030E0A901C301B2010E9418
:10F0F000FAE1882309F43BC1A7019601C701B601D3
:10F100000E9460E24B015C0129853A854B855C8554
:10F11000CA01B9010E9460E29B01AC01C501B401C2
:10F120000E94F0E84B015C01A3019201C301B2010E
:10F130000E94F1E89B01AC01C501B4010E9474E991
:10F140000E945DE90E94EDE96D837E838F8398873D
:10F1500069817A818B819C8190958095709561956C
:10F160007F4F8F4F9F4F0E9401E24B015C016D85E5
:10F170007E858F8598890E94FFE169837A838B83DE
:10F180009C8320E030E0A901C501B4010E94FAE1AE
:10F19000882309F4F0C029813A814B815C81CA013E
:10F1A000B9010E9460E26D8B7E8B8F8B988FA701D7
:10F1B0009601C701B6010E9460E29B01AC016D8916
:10F1C0007E898F89988D0E94F0E86B017C01A501F2
:10F1D0009401C501B4010E94F1E89B01AC01C70193
:10F1E000B6010E9474E90E941CEAA98DBA8D959619
:10F1F0008D909D90AD90BC909897750164012D8184
:10F200003E814F815885C21AD30AE40AF50A0E944A
:10F21000EDE9C61AD70AE80AF90AF7FE6EC020E03F
:10F2200030E0A901C301B2010E94FAE1882309F488
:10F23000A6C0C501B4010E94FFE16B017C01A301DE
:10F240009201C301B2010E94F1E89B01AC01C70128
:10F25000B6010E9460E26B017C0129853A854B85ED
:10F260005C85CA01B9010E9460E29B01AC01C70143
:10F27000B6010E94F0E86B017C0129813A814B8143
:10F280005C81CA01B9010E9460E29B01AC01C70127
:10F29000B6010E94F1E86B017C0120E030E040E81B
:10F2A00050E4C301B2010E9460E29B01AC01C701BE
:10F2B000B6010E9474E90E945DE96B017C0120E0C7
:10F2C00030E0A9010E9474EA18161CF0C12CD12C60
:10F2D0007601C701B6010E94EDE96D837E838F83BD
:10F2E000988786169706A806B90620F48D829E8216
:10F2F000AF82B886C12CD12C76018D819E81AF81E1
:10F30000B885E98DFA8D81A792A7A3A7B4A7C80EE7
:10F31000D91EEA1EFB1EC5A6D6A6E7A6F0AA298915
:10F320003A894B895C8922AF33AF44AF55AFFE9623
:10F330002D853E854F8558892083318342835383B1
:10F340006A960FB6F894DEBF0FBECDBFDF91CF91A6
:10F350001F910F91FF90EF90DF90CF90BF90AF90F3
:10F360009F908F907F906F905F904F90089560E096
:10F3700070E0CB01E5CE60E070E0CB0134CF60E01F
:10F3800070E0CB0198CF90916F0081E091FD02C0B9
:10F3900080E0089590916F009D7F90936F00089595
:10F3A000CF93C82F0E94C37994E0C99F9001112484
:10F3B000F901E752FB4F2B513B4FD9014D915D9124
:10F3C0006D917C91408351836283738391E090932C
:10F3D000D804882319F0CF910C94E130CF9108958F
:10F3E000CF92DF92EF92FF9280917D04329B60C0BA
:10F3F000816080937D0480917D04339B5BC082603B
:10F4000080937D0480917D04349B56C084608093FA
:10F410007D04C090C904C0FE10C08091930580FF98
:10F420000CC080917D0480FF08C08091A30581609D
:10F430008093A30580E00E94D079D12CF12CE12C9F
:10F44000D701C601B695A7959795879580FF11C0FE
:10F4500080919305869580FF0CC080917D0481FF8B
:10F4600008C08091A30582608093A30581E00E947B
:10F47000D07982E0F694E794D794C7948A95D1F72F
:10F48000C0FE1CC0809193058695869580FF16C0AE
:10F4900080917D0482FF12C08091A30584608093D7
:10F4A000A30582E0FF90EF90DF90CF900C94D0798D
:10F4B0008E7F9FCF8D7FA4CF8B7FA9CFFF90EF90C2
:10F4C000DF90CF9008950F931F93CF93DF93809198
:10F4D00047018F3708F447C08F579091A914909334
:10F4E0001805992309F43DC05D9A9091AD0590935C
:10F4F0001705992309F441C05C9A8F5F80934701F7
:10F500008091160591E089278093160581110E944C
:10F51000F01F80914601C1E0C80F85300CF0C0E0BB
:10F52000823009F4D3C05CF5882309F43EC08130F1
:10F5300009F4C1C0C09346018091920581110E94D7
:10F54000F0798091490690914A06009729F0019739
:10F5500090934A0680934906DF91CF911F910F91B6
:10F5600008955D98C2CF90911805891708F05D98AD
:10F5700090911705891708F4C0CF5C98BECF8430EE
:10F5800009F4BBC00CF4B5C08530A1F69091150507
:10F59000911102C0809315058091150581508093CB
:10F5A0001505882339F2C5E0C5CF809145018F5FED
:10F5B00080311CF480934501BDCF109245018091AC
:10F5C0007204811113C08091A1149091A2149093A0
:10F5D000A4148093A3148091A5059091A6059093FF
:10F5E000A8058093A70581E0809372041092A2146D
:10F5F0001092A1141092A6051092A5050091A314D3
:10F600001091A4148091A7149091A814D1E0181619
:10F6100019062CF08091A914811101C0D0E08091CD
:10F620004C0190914D01081719073CF44DE752E247
:10F630006AE872E280E00E94A972DD2371F0809195
:10F640004A0190914B01801791073CF44CE952E23A
:10F6500069EA72E280E00E94A9720091AB05109104
:10F66000AC052091A7053091A80580918F05909158
:10F670009005281739073CF44DE752E26AE872E238
:10F680008FEF0E94A972101611060CF053CF209133
:10F69000A7053091A80580914801909149018217F2
:10F6A00093070CF047CF4CE952E269EA72E28FEF20
:10F6B0000E94A9723FCF10927B0087E480937C0068
:10F6C00080917A00806480937A0034CF80917A00B0
:10F6D00086FD26C020917800309179008091A11498
:10F6E0009091A214820F931F9093A2148093A1145F
:10F6F00021CF10927B0086E4E1CF80917A0086FDD5
:10F7000011C020917800309179008091A5059091E9
:10F71000A605820F931F9093A6058093A5050ACF97
:10F72000C2E008CFC4E006CF0E94C379109233062E
:10F7300010923406109235061092360681110C9400
:10F74000E13008950F931F9380911E1590911F151E
:10F75000891B8F7009F449C090911B15992361F0A2
:10F76000833040F48FEF890F29F080931B1590E0D0
:10F7700080E038C010921B1580911F152BE4829FEA
:10F78000C0011124855B994FFC01208120FDEFCF42
:10F7900040913306509134066091350670913606DB
:10F7A000E95BFF4F0081118122813381401B510BA6
:10F7B000620B730B40933306509334066093350607
:10F7C0007093360620911F152F5F2F7020931C1504
:10F7D00030911F1520911D15321304C020911C1566
:10F7E00020931D151F910F9108950E94947BBFCF08
:10F7F0002F923F924F925F926F927F928F929F9241
:10F80000AF92BF92CF92DF92EF92FF920F931F932E
:10F81000CF93DF9300D000D0CDB7DEB78FEF9FEF4F
:10F8200090938900809388000AE00983312C212C71
:10F8300078948091D2049091D304A091D404B09193
:10F84000D504892B8A2B8B2B09F0C4C18091D80455
:10F850008823E1F08091D6049091D7041092D804C7
:10F86000892B09F4B7C11092D7041092D6041092D4
:10F87000C90490911E1580911F15981709F4AAC10B
:10F8800080911F158F5F8F7080931F158091D60414
:10F890009091D704892B09F49DC14091CE045091D9
:10F8A000CF046091D0047091D1048091CA049091EA
:10F8B000CB04A091CC04B091CD040091BC0410E025
:10F8C00030E020E0841B950BA60BB70B0817190737
:10F8D0002A073B0710F4D901C8018A83840F951FBA
:10F8E000A61FB71F8093CE049093CF04A093D0049B
:10F8F000B093D104E1E0C0909404D0909504E090DE
:10F900009604F09097048091A4049091A504A0918E
:10F91000A604B091A704C80ED91EEA1EFB1EC09211
:10F92000A404D092A504E092A604F092A704F7FCE8
:10F9300033C040918C04042E000C550B660B770BE2
:10F940008091E5049091E604A091E704B091E80469
:10F95000840F951FA61FB71F8093E5049093E604BC
:10F96000A093E704B093E8048091900490919104EF
:10F97000A0919204B0919304A7019601281B390B22
:10F980004A0B5B0BDA01C9018093A4049093A50490
:10F99000A093A604B093A704009198041091990431
:10F9A00020919A0430919B048091A8049091A9041D
:10F9B000A091AA04B091AB04080F191F2A1F3B1F86
:10F9C0000093A8041093A9042093AA043093AB04D5
:10F9D00037FD33C080918D04082E000C990BAA0BC3
:10F9E000BB0B4091E9045091EA046091EB047091E3
:10F9F000EC04840F951FA61FB71F8093E904909312
:10FA0000EA04A093EB04B093EC04809190049091ED
:10FA10009104A0919204B0919304B901A801481BEC
:10FA2000590B6A0B7B0BDB01CA018093A8049093EE
:10FA3000A904A093AA04B093AB0440919C045091F4
:10FA40009D0460919E0470919F048091AC049091FC
:10FA5000AD04A091AE04B091AF04480F591F6A1FC6
:10FA60007B1F4093AC045093AD046093AE0470933D
:10FA7000AF0477FD33C080918E04082E000C990BE3
:10FA8000AA0BBB0B8090ED049090EE04A090EF04C5
:10FA9000B090F004880D991DAA1DBB1D8093ED0444
:10FAA0009093EE04A093EF04B093F004809190043F
:10FAB00090919104A0919204B09193042A013B018A
:10FAC000481A590A6A0A7B0AD301C2018093AC041E
:10FAD0009093AD04A093AE04B093AF048090A004C3
:10FAE0009090A104A090A204B090A3048091B004CF
:10FAF0009091B104A091B204B091B304880D991D06
:10FB0000AA1DBB1D8093B0049093B104A093B204CE
:10FB1000B093B304B7FD33C040908F04042C000CA5
:10FB20005508660877088090F1049090F204A09040
:10FB3000F304B090F404840C951CA61CB71C8092AE
:10FB4000F1049092F204A092F304B092F404809035
:10FB5000900490909104A0909204B09093042C0192
:10FB60003D01481859086A087B08530142018092F8
:10FB7000B0049092B104A092B204B092B304E11127
:10FB800004C0E0918400F0918500F7FE5F9A37FF92
:10FB9000469A77FF2B9AB7FF299AE0918400F0915B
:10FBA0008500E0918400F0918500F7FE5F9837FFB3
:10FBB000469877FF2B98B7FF29985A80552021F057
:10FBC00080918400909185000A8101500A83E0E0D1
:10FBD000011191CE8090540190905501A090560152
:10FBE000B090570181149104A104B10409F047C0F9
:10FBF0008091EC059091ED05009709F42FC023B199
:10FC00002470159800000000000000001816190666
:10FC10000CF0D7C02A9A00000000000000002B9AC8
:10FC200034E03A950000E9F72B980000000000004E
:10FC30000000222309F4C7C02A9A00000000000037
:10FC40000000181619060CF0C0C08091EC059091C8
:10FC5000ED0501979093ED058093EC050E948F339D
:10FC6000882309F4B8C080ED97E0A0E0B0E080936D
:10FC7000540190935501A0935601B0935701809180
:10FC8000D2049091D304A091D404B091D504892BCF
:10FC90008A2B8B2B09F053C4E091D604F091D70442
:10FCA000309709F427C58091CE049091CF04A0919C
:10FCB000D004B091D1044091CA045091CB0460911A
:10FCC000CC047091CD0484179507A607B70708F4F4
:10FCD00086C01092D7041092D6041092C904909155
:10FCE0001E1580911F15981709F404C580911F15E2
:10FCF0008F5F8F7080931F1580EDC82E87E0D82E00
:10FD0000E12CF12C8091D6049091D704892B09F035
:10FD10000EC40E94A27B9093D7048093D604892BB3
:10FD200009F405C44090D6045090D7045C824B82FD
:10FD3000D2018C9183FFB3C2F201858D968DA78D80
:10FD4000B0A1418D528D638D748D058916892789E7
:10FD5000308D0093E5041093E6042093E70430937C
:10FD6000E8044093E9045093EA046093EB04709331
:10FD7000EC048093ED049093EE04A093EF04B09311
:10FD8000F00481A192A1A3A1B4A18093F104909366
:10FD9000F204A093F304B093F4041092D7041092E9
:10FDA000D6041092C90490911E1580911F159817C2
:10FDB00009F4AFCF80911F158F5F8F7080931F154F
:10FDC000A8CF2A9828CF2A9838CF8091EC05909117
:10FDD000ED0501963FCF8FEF9FEFDC0148CF4091BB
:10FDE000C5045091C6046091C7047091C8044817B7
:10FDF00059076A077B0708F4DEC08091C10490911F
:10FE0000C204A091C304B091C40441A952A963A93A
:10FE100074A91127859F412C969F9001A69F300DB4
:10FE2000A59F200D311D869F400C211D311F959FE0
:10FE3000400C211D311FA49F400C211D311F949F98
:10FE4000410C211F311F4694211F311F789F200D27
:10FE5000311D799F300D112442AD53AD64AD75ADA8
:10FE6000420F531F611D711D4093BD045093BE048A
:10FE70006093BF047093C00406A917A920AD31ADEB
:10FE8000041715072607370740F40093BD041093A5
:10FE9000BE042093BF043093C0044090BD04509032
:10FEA000BE046090BF047090C0042EE531E201E012
:10FEB0000A83F90145915591659174914415550551
:10FEC0006605770570F476946794579447941A8181
:10FED000110F1A832C5F3F4F4AE751E24217530735
:10FEE00041F75A815093BC0460E246165104610404
:10FEF000710428F410E2412E512C612C712C70E217
:10FF0000471A5108610871084114E8E05E0661046F
:10FF1000710408F42EC0F4E05F9E90011124225A6F
:10FF2000324EF901329645915491042DEE27059FEA
:10FF3000B001049F610D7E1F06946E1F7E1F112469
:10FF4000AB0170E060E0F901C590D490F12CE12C98
:10FF5000C41AD50AE60AF70A8C0D9D1DAE1DBF1DF9
:10FF60008093C1049093C204A093C304B093C404CB
:10FF7000C9CEB301A20176956795579547959A0129
:10FF80002C7F225A364EF901C590D490F901329651
:10FF900045915491142D1770149F9001159F300DA9
:10FFA0001124F3E036952795FA95E1F7C21AD30AA2
:10FFB000F12CE12CD1CF4091B8045091B90460915B
:10FFC000BA047091BB04481759076A077B0708F009
:10FFD000D4C08091B4049091B504A091B604B091BE
:10FFE000B70441A952A963A974A92227859F312D7D
:10FFF000969F8001A69F100DA59F000D111D869F45
:020000021000EC
:10000000300D011D121F959F300D011D121FA49F61
:10001000300D011D121F949F310D021F121F3695C6
:10002000021F121F789F000D111D799F100D1124C2
:1000300030E020E04091BD045091BE046091BF04C7
:100040007091C004FE9640805180628073800417D6
:1000500015072607370758F4401B510B620B730B2B
:10006000441655066606770610F42A013B012EE574
:1000700031E241E04A83F9014591559165917491CE
:10008000441555056605770570F476946794579482
:1000900047945A81550F5A832C5F3F4F6AE771E2AC
:1000A0006217730741F77A817093BC04E0E24E1641
:1000B00051046104710428F400E2402E512C612C9B
:1000C000712CF0E24F1A510861087108411408E0E0
:1000D00050066104710408F42EC014E0519E900192
:1000E0001124225A324EF901329645915491F42D41
:1000F000EE27F59FB001F49F610D7E1F06946E1FE1
:100100007E1F1124AB0170E060E0F901C590D4902E
:10011000F12CE12CC41AD50AE60AF70A8C0D9D1DB4
:10012000AE1DBF1D8093B4049093B504A093B60494
:10013000B093B704E7CDB301A201769567955795C3
:1001400047959A012C7F225A364EF901C590D490DA
:10015000F901329645915491042D0770049F900146
:10016000059F300D112413E0369527951A95E1F778
:10017000C21AD30AF12CE12CD1CF80914101909188
:100180004201A0914301B0914401B7FF5DC0C6A8F0
:10019000D7A8E0ACF1AC8EE591E221E0FC014591FD
:1001A0005591659174914C155D056E057F0558F468
:1001B000F694E794D794C794220F04964AE751E245
:1001C0004817590759F72093BC0450E2C516D104CB
:1001D000E104F10428F470E2C72ED12CE12CF12CBB
:1001E00060E2C61AD108E108F108C11478E0D70628
:1001F000E104F10408F431C0A4E0DA9EC001112446
:10020000825A924EFC01329625913491BC2D66277C
:10021000B39FA001B29F410D561F0694461F561F63
:10022000112470E060E0FC0185919491B0E0A0E0C1
:10023000841B950BA60BB70B809341019093420151
:10024000A0934301B0934401C0904101D09042017A
:10025000E0904301F090440155CDD701C601B69519
:10026000A795979587958C7F825A964EFC0125918C
:100270003491FC01329645915491EC2DE770E49F46
:10028000C001E59F900D112463E0969587956A95CE
:10029000E1F7281B390BC901B0E0A0E0CDCFAB815D
:1002A000BC8155960D911D912D913C91589781E0FF
:1002B000011511052105310509F480E0EB81FC8170
:1002C000C18CD28CE38CF48CC114D104E104F10410
:1002D00009F08260AB81BC815D964D915D916D911D
:1002E0007C919097411551056105710509F0846075
:1002F0008093C9041092B4041092B5041092B6040D
:100300001092B7041092C1041092C2041092C30458
:100310001092C404EB81FC8185A196A1A7A1B0A590
:100320008093CA049093CB04A093CC04B093CD04E3
:10033000442455243201481A590A6A0A7B0A409219
:10034000A4045092A5046092A6047092A70440925F
:10035000A8045092A9046092AA047092AB0440923F
:10036000AC045092AD046092AE047092AF0440921F
:10037000B0045092B1046092B2047092B30441A0F0
:1003800052A063A074A0440C551C661C771C000F7F
:10039000111F221F331F0093940410939504209380
:1003A000960430939704CC0CDD1CEE1CFF1CC0920D
:1003B0009804D0929904E0929A04F0929B04440F1E
:1003C000551F661F771F40939C0450939D046093B4
:1003D0009E0470939F044092A0045092A1046092E6
:1003E000A2047092A304880F991FAA1FBB1F8093B9
:1003F000900490939104A0939204B093930410926C
:10040000CE041092CF041092D0041092D10481A592
:1004100092A5A3A5B4A58093C5049093C604A09308
:10042000C704B093C80485A596A5A7A5B0A98093D5
:10043000B8049093B904A093BA04B093BB0485A9FF
:1004400090919305891721F0809393050E942C7455
:100450008091920581110E94F07944244A94542C91
:1004600032014092410150924201609243017092E8
:100470004401AB81BC81DA964D915D916D917C9187
:10048000DD974093BD045093BE046093BF04709306
:10049000C0048EE591E2A1E0FC0105911591259142
:1004A0003491041715072607370758F47695679592
:1004B00057954795AA0F0496EAE7F1E2E817F9077E
:1004C00059F7A093BC04403251056105710520F431
:1004D00040E250E060E070E040525109610971096A
:1004E0004115F8E05F076105710508F4DAC004E022
:1004F000509FC0011124825A924EFC0132962591E0
:100500003491AA27439FF001429FE10DFA1F069400
:10051000EA1FFA1F1124AF0170E060E0FC01C590F2
:10052000D490F12CE12CC41AD50AE60AF70AC0923D
:10053000D204D092D304E092D404F092D504892856
:100540008A288B28C9F48091D2049091D304A09179
:10055000D404B091D5048A3F9105A105B10560F49A
:100560002AEF30E040E050E02093D2043093D304EF
:100570004093D4045093D5044091540150915501B7
:1005800060915601709157010091D2041091D304EB
:100590002091D4043091D5044F3F8FEF580768075E
:1005A000780799F0D901C801B695A79597958795D1
:1005B000481759076A077B0740F4809354019093CA
:1005C0005501A0935601B0935701409154015091A9
:1005D000550160915601709157014F3F9FEF5907A8
:1005E0006105710508F07DC04B835A83F62FE72F14
:1005F0008B819A81AF2FBE2F081719072A073B0757
:1006000010F4D901C801081B190B2A0B3B0B0093EE
:10061000D2041093D3042093D4043093D5044F3FD5
:10062000EFEF5E076E077E0761F0481B590B6A0B00
:100630007B0B409354015093550160935601709386
:100640005701F8942091840030918500205F3F4F3E
:10065000098101500983002309F44AC0280E391E7C
:100660002216330610F40C94187C309289002092E4
:10067000880078940F900F900F900F90DF91CF919A
:100680001F910F91FF90EF90DF90CF90BF90AF90B0
:100690009F908F907F906F905F904F903F902F90A2
:1006A0000895DB01CA01B695A795979587958C7F2C
:1006B000825A964EFC01C590D490FC013296259149
:1006C00034914770429FC001439F900D1124A3E0D5
:1006D00096958795AA95E1F7C81AD90AF12CE12CCD
:1006E00026CFAFEFAB83BFEFBA83F0E0E0E080CF7F
:1006F0001901BBCF80EDC82E87E0D82EE12CF12C5C
:1007000008CBFC01208131814281538160911C0B17
:1007100070911D0B80911E0B90911F0B0E9460E247
:100720000E9479EA60932C1570932D1580932E15F5
:1007300090932F1590911E1580911F1598130C946E
:1007400036660E949C770E94C37940912C15509187
:100750002D1560912E1570912F154093F104509333
:10076000F2046093F3047093F40481110C94E1306B
:1007700008954F925F926F927F928F929F92AF9265
:10078000BF92CF92DF92EF92FF920F931F93CF937E
:10079000DF93EC018B015A01F90120911C0B309180
:1007A0001D0B40911E0B50911F0B60817181828146
:1007B00093810E9460E20E9479EA6B017C012091A2
:1007C000180B3091190B40911A0B50911B0BF5012E
:1007D00060817181828193810E9460E20E9479EA46
:1007E0004B015C012091140B3091150B4091160BBD
:1007F0005091170BF80160817181828193810E9471
:1008000060E20E9479EA2B013C012091100B3091AB
:10081000110B4091120B5091130B688179818A81E1
:100820009B810E9460E20E9479EA60932015709398
:1008300021158093221590932315409224155092F0
:100840002515609226157092271580922815909292
:100850002915A0922A15B0922B15C0922C15D09272
:100860002D15E0922E15F0922F1590911E15809166
:100870001F15981791F0DF91CF911F910F91FF9065
:10088000EF90DF90CF90BF90AF909F908F907F9030
:100890006F905F904F900C9436660E949C770E94F8
:1008A000C379409128155091291560912A157091AE
:1008B0002B150091241510912515209126153091A6
:1008C0002715C0902015D0902115E0902215F090AA
:1008D0002315C092E504D092E604E092E704F0927A
:1008E000E8040093E9041093EA042093EB043093A6
:1008F000EC044093ED045093EE046093EF04709386
:10090000F00440912C1550912D1560912E15709189
:100910002F154093F1045093F2046093F304709305
:10092000F404882391F0DF91CF911F910F91FF90F4
:10093000EF90DF90CF90BF90AF909F908F907F907F
:100940006F905F904F900C94E130DF91CF911F91A9
:100950000F91FF90EF90DF90CF90BF90AF909F905E
:100960008F907F906F905F904F900895CF92DF921D
:10097000EF92FF92CF93DF93C82F0E94C37994E048
:10098000C99FE0011124FE01EB51FB4FC080D180D3
:10099000E280F38081110E94E130C85CD94FC70129
:1009A000B6010E9401E2288139814A815B810E945F
:1009B00060E2DF91CF91FF90EF90DF90CF900895AC
:1009C000CF92DF92EF92FF92CF93DF93C82F0E94D6
:1009D000C37994E0C99FE0011124FE01E752FB4F67
:1009E000C080D180E280F38081110E94E130C85C38
:1009F000D94FC701B6010E9401E2288139814A819D
:100A00005B810E9460E2DF91CF91FF90EF90DF90D9
:100A1000CF900895CF930E94C379C82F80911F155E
:100A200080931E1580931D1580931C1584E680937A
:100A30001B150E94947B80ED93E090934A0680936F
:100A40004906C1110E94E13081E08093D804CF9122
:100A50000895CF93DF9324E0829FC0011124EC011D
:100A6000CF5FD94FFC01EB56FA4F8F519C4FDC0101
:100A70002D913D914D915C91608171818281938135
:100A80000E94F1E8688379838A839B83DF91CF9109
:100A9000089580FF04C090917E0490FD8E7F81FFB9
:100AA00005C090917E04969590FD8D7F82FF06C0D3
:100AB00090917E049695969590FD8B7F0895CF92A8
:100AC000DF92EF92FF920F931F93C12CD12C7601EE
:100AD0008C0120E53BE04CE45BE068E47BE084E4EF
:100AE0009BE00E9437B91F910F91FF90EF90DF902C
:100AF000CF9008954F925F926F927F928F929F92C4
:100B0000AF92BF92CF92DF92EF92FF920F931F931B
:100B1000CF93DF93CDB7DEB72C970FB6F894DEBF37
:100B20000FBECDBF2B013C0129873A874B875C87DD
:100B300047015801F601E080F1800281138120E035
:100B400030E0A901B701C8010E94FAE1882309F445
:100B500084C05E2D4F2D302F212F852F942FA32F52
:100B6000B22F89839A83AB83BC8320E030E0A90154
:100B7000B701C8010E94FAE1811104C0E12CF12CF7
:100B800008E413E4C701D8018D839E83AF83B8873F
:100B9000A501940160914C0B70914D0B80914E0B0F
:100BA00090914F0B0E94FAE187FF0CC080924C0B92
:100BB00090924D0BA0924E0BB0924F0BCE0101962E
:100BC0000E945F854092440B5092450B6092460B09
:100BD0007092470B89859A85AB85BC858093480BBD
:100BE0009093490BA0934A0BB0934B0BCE01059603
:100BF0000E945F85A501940160914C0B70914D0B93
:100C000080914E0B90914F0B0E9474EA181664F479
:100C100080924C0B90924D0BA0924E0BB0924F0BCA
:100C2000CE0101960E945F850E949C772C960FB69C
:100C3000F894DEBF0FBECDBFDF91CF911F910F9112
:100C4000FF90EF90DF90CF90BF90AF909F908F90EC
:100C50007F906F905F904F90089550E040E030E8B3
:100C600020E47BCFCF92DF92EF92FF920F931F93FE
:100C70006B01FC01E080F18002811381E4E4FBE080
:100C80002481358146815781608171818281938180
:100C90000E947A851F910F91FF90EF90DF90CF9087
:100CA00008950C9499B92F923F924F925F926F9250
:100CB0007F928F929F92AF92BF92CF92DF92EF92EC
:100CC000FF920F931F93CF93DF93CDB7DEB76C974F
:100CD0000FB6F894DEBF0FBECDBF809171048111B5
:100CE00050C18091700481113CC1809172048111C6
:100CF00019C06C960FB6F894DEBF0FBECDBFDF9162
:100D0000CF911F910F91FF90EF90DF90CF90BF9008
:100D1000AF909F908F907F906F905F904F903F909B
:100D20002F9008950E9491720E9480C14B015C0136
:100D30000091A5141091A614809150019091510139
:100D4000801791070CF448C26091A7147091A81401
:100D5000072E000C880B990B0E9401E26D837E83A5
:100D60008F839887B801110F880B990B0E9401E2BD
:100D700069837A838B839C832AE0E22EF12C0CE337
:100D800010E020E0AE014B5F5F4FBE016F5F7F4F11
:100D900089E095E10E940A730091A5141091A614B0
:100DA00080914E0190914F01801791070CF4F0C093
:100DB00060E06093A91480919D1490919E14A0917D
:100DC0009F14B091A0140097A105B10539F1A501B8
:100DD0009401281B390B4A0B5B0BDA01C901B7FDE3
:100DE0001DC080919B1490919C14081719070CF456
:100DF00013C28091A7149091A814009739F00E5F48
:100E00001F4F0497081719070CF41CC210929D1469
:100E100010929E1410929F141092A0148091A90514
:100E20009091AA05873991050CF0E2C180911105D6
:100E300090911205A0911305B09114050097A1059A
:100E4000B10561F1A5019401281B390B4A0B5B0B1D
:100E5000DA01C901B7FD22C08091A9059091AA05C8
:100E600020910F0530911005821793070CF4CCC127
:100E70002091AB053091AC052115310539F0029672
:100E800024503109821793070CF4EFC11092110519
:100E900010921205109213051092140580910B0503
:100EA00090910C05A0910D05B0910E05A50194013E
:100EB000281B390B4A0B5B0BDA01C901B7FD19CFAF
:100EC00038E8830E33E1931EA11CB11C80920B0500
:100ED00090920C05A0920D05B0920E056091AB05A5
:100EE0007091AC05072E000C880B990B0E9401E253
:100EF0006D837E838F8398876091A9057091AA0581
:100F0000072E000C880B990B0E9401E269837A83FB
:100F10008B839C8382E0E82EF12C02E310E02FEF1C
:100F2000AE014B5F5F4FBE016F5F7F4F82E195E186
:100F30000E940A738091A9059091AA059C012550F1
:100F400031092239310508F05BC12091AB053091A0
:100F5000AC05821793070CF467C180E08093AD0560
:100F6000C8CE109270040E940A850E949C770E944D
:100F7000D2B80E94518680917204882309F4B9CEB8
:100F8000D1CE41E070E060E08FEC91E20E946E3AD9
:100F90008091500190915101081719070CF008CF6A
:100FA000E090A714F090A814B801012E000C880B53
:100FB000990B0E9401E21B012C01E114F10409F4D8
:100FC0003CC1B701601B710B072E000C880B990BFD
:100FD0000E9401E26B017C0120E030E040E251EC34
:100FE0000E94FAE187FD29C120E030E040E251E4AF
:100FF000C701B6010E9474EA18160CF449C1809129
:101000000A05811149C120910205309103054091E3
:1010100004055091050529873A874B875C878091A5
:10102000060590910705A0910805B09109058D87E7
:101030009E87AF87B88BA20191016091F6047091F1
:10104000F7048091F8049091F9040E94F0E820914F
:10105000B2143091B3144091B4145091B5140E945D
:1010600060E229853A854B855C850E94F0E820ED99
:101070003CEC4CE45DE30E9460E229853A854B85B7
:101080005C850E94F1E8698B7A8B8B8B9C8B6093DB
:101090000205709303058093040590930505209144
:1010A000AE143091AF144091B0145091B1142D8B07
:1010B0003E8B4F8B588F2D853E854F855889C701B4
:1010C000B6010E94F1E8762E672E89879D8720E081
:1010D00030E0A9010E94FAE187FDE9C02D893E892F
:1010E0004F89588D60E070E08FE793E40E9474E9C7
:1010F000698F7A8F8B8F9C8F272D362D49855D8543
:101100000E94FAE187FF06C0798C6A8C3B8D398793
:101110004C8D4D87872D962DA985BD85809306051D
:1011200090930705A0930805B09309052091AA1490
:101130003091AB144091AC145091AD14C701B6017D
:101140000E9460E26B017C01C092FA04D092FB0421
:10115000E092FC04F092FD04272D362D49855D8533
:101160006D897E898F89988D0E9460E29B01AC0118
:101170002093FE043093FF04409300055093010533
:10118000C701B6010E94F1E829893A894B895C8937
:101190000E94F1E820E030E0A9010E94F1E86B0133
:1011A0007C0120E030E0A9010E94FAE187FD48C0FF
:1011B00020E030E04FE753E4C701B6010E9474EA33
:1011C0001816A4F56FE72092F6043092F7044092C7
:1011D000F8045092F904EDCD4DE752E26AE872E26C
:1011E00080E00E94A9720091A5141091A614ACCDC4
:1011F0004DE752E26AE872E28FEF0E94A97216CEC2
:101200001092AD055C9875CD41EB51E260EC71E256
:101210008FEF0E94A97242CE41EB51E260EC71E285
:1012200080E00E94A972FACD8FE798CEC701B6017F
:101230000E94E6E975956795C6CF81E080930A051F
:1012400060E0C1CF10939C1400939B140E9480C156
:10125000605B7C438F4F9F4F60939D1470939E14EF
:1012600080939F149093A014D9CD909310058093F0
:101270000F050E9480C1605E70448D4F9F4F609348
:10128000110570931205809313059093140506CEF3
:1012900081E080930A0596CF10920A051D861E866E
:1012A0001F86188A19861A861B861C86C4CE712C46
:1012B000612C19861D862ECF2F923F924F925F92FE
:1012C0006F927F928F929F92AF92BF92CF92DF9256
:1012D000EF92FF920F931F93CF93DF93CDB7DEB7BB
:1012E000A6970FB6F894DEBF0FBECDBF8091270141
:1012F000882309F4CDC080917E04C82ED12CF12C16
:10130000E12C80FF3CC08090290190902A01A090A0
:101310002B01B0902C012091ED033091EE03409110
:10132000EF035091F003C501B4010E9474EA18164E
:1013300044F48092ED039092EE03A092EF03B092FA
:10134000F0038090350190903601A0903701B09065
:1013500038012091ED033091EE034091EF0350915D
:10136000F003C501B4010E94FAE187FF08C0809232
:10137000ED039092EE03A092EF03B092F003D70139
:10138000C601B695A7959795879580FF3CC080903C
:101390002D0190902E01A0902F01B090300120914E
:1013A000F1033091F2034091F3035091F403C5012E
:1013B000B4010E9474EA181644F48092F1039092EA
:1013C000F203A092F303B092F4038090390190905D
:1013D0003A01A0903B01B0903C012091F103309183
:1013E000F2034091F3035091F403C501B4010E944C
:1013F000FAE187FF08C08092F1039092F203A09275
:10140000F303B092F40392E0F694E794D794C79470
:101410009A95D1F7C0FE3CC0C0903101D090320106
:10142000E0903301F09034012091F5033091F60300
:101430004091F7035091F803C701B6010E9474EA86
:10144000181644F4C092F503D092F603E092F70325
:10145000F092F803C0903D01D0903E01E0903F0132
:10146000F09040012091F5033091F6034091F7038D
:101470005091F803C701B6010E94FAE187FF08C046
:10148000C092F503D092F603E092F703F092F803CE
:101490008091FB0A83FD7EC02091500B3091510B4F
:1014A0004091520B5091530B6091F9037091FA03E4
:1014B0008091FB039091FC030E94FAE1882309F4D8
:1014C00069C010914806111161C080915C01909132
:1014D0005D0101972091A5143091A61428173907B2
:1014E0003CF40E94453A8AE496E10E94803911E07A
:1014F0002091500B3091510B4091520B5091530B56
:101500006091F9037091FA038091FB039091FC03C1
:101510000E94F0E86B017C0120E030E0A9010E940C
:1015200074EA87FF04C0F7FAF094F7F8F09420917A
:1015300058013091590140915A0150915B01C70106
:10154000B6010E9460E220E030E84BE354E40E94E0
:1015500074EA1816ECF40E94453A8BE296E10E9478
:1015600080398091F9039091FA03A091FB03B09127
:10157000FC038093500B9093510BA093520BB093AC
:10158000530B89EF93E00E94818304C010E0B0CF39
:101590001111E7CF2AE037ED43E25CE360912101CE
:1015A0007091220180912301909124010E9460E2B8
:1015B0006B017C0160911F0170912001072E000CCE
:1015C000880B990B0E9401E29B01AC01C701B60197
:1015D0000E9460E2698B7A8B8B8B9C8B80910104DB
:1015E000882309F46CC02091440B3091450B409145
:1015F000460B5091470B6091ED037091EE03809183
:10160000EF039091F0030E94F0E86D8B7E8B8F8B3F
:10161000988F2091480B3091490B40914A0B509183
:101620004B0B6091F1037091F2038091F303909161
:10163000F4030E94F0E8698F7A8F8B8F9C8F209142
:101640004C0B30914D0B40914E0B50914F0B6091D4
:10165000F5037091F6038091F7039091F8030E94CF
:10166000F0E86D8F7E8F8F8F98A32091500B309173
:10167000510B4091520B5091530B6091F9037091B3
:10168000FA038091FB039091FC030E94F0E86B0148
:101690007C0120E030E0A9016D897E898F89988DD9
:1016A0000E94FAE181110FC020E030E0A901698DAC
:1016B0007A8D8B8D9C8D0E94FAE1811104C0C12C22
:1016C000D12C76012CC12D893E894F89588DCA01B4
:1016D000B9010E9460E24B015C01298D3A8D4B8D6E
:1016E0005C8DCA01B9010E9460E29B01AC01C50199
:1016F000B4010E94F1E84B015C012D8D3E8D4F8DB0
:1017000058A1CA01B9010E9460E29B01AC01C50168
:10171000B4010E94F1E84B015C01A7019601C701E9
:10172000B6010E9460E29B01AC01C501B4010E94B8
:10173000F1E80E94B2EA4B015C012DEB37E346E889
:1017400055E30E94FAE187FF0FC020E030E0A901D5
:10175000C701B6010E9474EA4601570187FF04C021
:10176000B7FAB094B7F8B0942DEB37E346E855E3F9
:10177000C501B4010E94FAE187FDDEC020E030E03F
:1017800040EA51E4C501B4010E9474E90E94EDE908
:101790001B01672B19F422242394312CB10190E012
:1017A00080E00E94FFE19B01AC0160E070E080E816
:1017B0009FE30E9474E92B013C01AC019B01C50130
:1017C000B4010E9460E24B015C01A30192016D89AA
:1017D0007E898F89988D0E9460E26D8B7E8B8F8BC6
:1017E000988FA3019201698D7A8D8B8D9C8D0E94BB
:1017F00060E2698F7A8F8B8F9C8FA30192016D8D30
:101800007E8D8F8D98A10E9460E26D8F7E8F8F8F6D
:1018100098A3A3019201C701B6010E9460E269A3E7
:101820007AA38BA39CA380E1E4E4FBE08E010F5F2D
:101830001F4FD80101900D928A95E1F70E9480C157
:101840002B013C0128EC420E511C611C711C0DA3A4
:101850001EA381E0281A310809F45FC00E9480C1EC
:101860008B019C01041915092609370937FD86C02B
:101870002B013C0128EC420E511C611C711C0E9482
:1018800011402D893E894F89588D69817A818B81DC
:101890009C810E94F1E869837A838B839C83298DE4
:1018A0003A8D4B8D5C8D6D817E818F8198850E94F4
:1018B000F1E86D837E838F8398872D8D3E8D4F8DCC
:1018C00058A169857A858B859C850E94F1E8698796
:1018D0007A878B879C8729A13AA14BA15CA16D8552
:1018E0007E858F8598890E94F1E86D877E878F8736
:1018F000988B750164018E010F5E1F4F9E01235F5F
:101900003F4FAE01475F5F4FBE016B5F7F4F8DA1C1
:101910009EA10E9437B981119CCF750164018E018F
:101920000F5E1F4F29EF33E045EF53E061EF73E0A7
:101930008DEE93E00E9437B980E1EDEEF3E0A4E490
:10194000BBE001900D928A95E1F7A6960FB6F89448
:10195000DEBF0FBECDBFDF91CF911F910F91FF90E2
:10196000EF90DF90CF90BF90AF909F908F907F903F
:101970006F905F904F903F902F9008950E945386F4
:1019800080CF2F923F924F925F926F927F928F9271
:101990009F92AF92BF92CF92DF92EF92FF920F93FE
:1019A0001F93CF93DF93CDB7DEB761970FB6F8944F
:1019B000DEBF0FBECDBF898BE82EF12CF701E954B5
:1019C000F94D6491062E000C770B880B990B0E9441
:1019D00001E24B015C011701220C331C220C331C69
:1019E000F101EE55F94E2591359145915491C5017E
:1019F000B4010E9460E22B013C01F101EA56F94E6C
:101A0000659175918591949120E030E040EC5FE321
:101A10000E9460E2A50194010E9460E2AB01BC015A
:101A200000E010E0980189890E9445BB20E030E089
:101A3000A901C301B2010E94FAE1882309F441C05F
:101A4000B301A201705800E010E0980189890E945A
:101A500045BBA3019201C301B2010E94F1E82B0131
:101A60003C01F701ED56F94E1491111107C00E9487
:101A7000453A81E796E10E9480391AE089898230EF
:101A800008F0CBC060E070E88BE395E420E030E044
:101A900040E752E40E9474E96B017C01612F70E021
:101AA00090E080E00E94FFE19B01AC01C701B6011C
:101AB0000E9474E98B019C01B301A20189890E94F3
:101AC00045BB81E090E0A0E0B0E0098804C0880F49
:101AD000991FAA1FBB1F0A94D2F720919405282BA7
:101AE0002093940520917E04822B80937E04F10143
:101AF000EB59F94E85919591A591B49181010C5BBB
:101B0000144FF80180839183A283B383F101EF51D5
:101B1000FC4F108211821282138289890E942985CA
:101B20000E945186F801C080D180E280F380F101EB
:101B3000E351FC4FC082D182E282F3828CE0E7EC79
:101B4000F1E0DE01119601900D928A95E1F7E1E056
:101B5000F0E0EC0FFD1FE20DF31D4080518062802C
:101B6000738020E030E0A901C301B2010E94FAE1D4
:101B70008823D1F120E030E0A901C301B2010E9425
:101B800074EA87FF04C077FA709477F87094810143
:101B90000C5B144FA3019201C501B4010E9460E2E5
:101BA0009B01AC01C701B6010E94F0E8F801608317
:101BB000718382839383F98960E070E88BE395E415
:101BC000F23020F060E070E080E793E420E030E065
:101BD00040E752E40E9474E96D877E878F87988B77
:101BE000CE010D960E945F8561960FB6F894DEBF18
:101BF0000FBECDBFDF91CF911F910F91FF90EF905E
:101C0000DF90CF90BF90AF909F908F907F906F901C
